:100000000C94B3400C94E4400C94E4400C94E44011
:100010000C94E4400C94E4400C94E4400C94E440D0
:100020000C94E4400C94E4400C94E4400C94E440C0
:100030000C94E4400C94E4400C94E4400C94E440B0
:100040000C94E4400D94521A0C94E4400C94E44057
:100050000C94E4400C94E4400D94569E0D94317D34
:100060000C94E4400C94F5960C94E4400C94E44019
:100070000C94E4400C94E4400C94E4400C94E44070
:100080000D9403230C94E4400C94E4400C94E4405D
:100090000C94E4400C94E4400C94E4400C94E44050
:1000A0000C94E4400C94E4400D94D5220C94E4406C
:1000B0000C94E4400C94E4400C94E4400D94A7228A
:1000C0000C94E4400C94E4400C94E4400C94E44020
:1000D0000C94E4400C94E4400C94E4400C94E44010
:1000E0000C94E44028972E973F974A97529767972A
:1000F000569767975A975E9767976497C801DC0190
:10010000940244020A026C012E027202F801AA0251
:100110006002AA02AA02AA02AA02AA02AA02AA02C9
:10012000AA02AA02AA02AA02AA02AA02AA02AA026F
:10013000AA02AA02AA02AA02AA02AA02AA02AA025F
:10014000AA02AA02AA02B402AA02AA02AA02AA0245
:10015000AA02AA02AA02AA02F201AA02AA02AA02F8
:10016000AA02AA02AA02AA02AA02AA02AA02C20118
:100170008A02C2029E01EA01460268024E0284021D
:100180002C021C0258017201A402C00282028002E9
:100190005A01F001380278016401B8018E018A0128
:1001A000D20274029201C402900108022802BC0229
:1001B0009802D202340274010C025202A001FE0124
:1001C00070029202CC01F601BA02FA017E027C02B0
:1001D0008201CC02AE01CC01C6013602F401084A0C
:1001E000D73B3BCE016E84BCBFFDC12F3D6C74314B
:1001F0009ABD56833DDA3D00C77F11BED9E4BB4CA2
:100200003E916BAAAABE000000803F05A84CCDB26B
:10021000D44EB93836A9020C50B9918688083CA64C
:10022000AAAA2ABE000000803F07634236B79BD8C7
:10023000A71A39685618AEBAAB558C1D3CB7CC57C7
:1002400063BD6DEDFD753EF6177231BF0000008095
:100250003F08000000BE922449123EABAAAA2ABE63
:10026000CDCCCC4C3E00000080BEABAAAAAA3E007A
:10027000000000BF000000803F00000000000841B7
:1002800078D3BB4387D1133D190E3CC3BD4282AD29
:100290002B3E68EC8276BED98FE1A93E4C80EFFF01
:1002A000BE01C4FF7F3F0000000000000D940E035C
:1002B0000D948E9A0D941AA30D9444000D94EE049F
:1002C0000C94C3D60C9449C80D947EA90C9460FF7D
:1002D0000C9493D70C94C8D60D941D4D0D94F5AD88
:1002E0000C9452970D942CA20D94ACA90D94320D40
:1002F0000D947BA90D947B020C9439CA0C9493DD68
:100300000C9443CA0D9471AD0D946C040D940FB709
:100310000C9466D30D9477A90C94ACFE0D9471A93E
:100320000D9490A90D9486A90C9443D30C9434D0C9
:100330000C945E970D944D020C9492DD0D947C9A72
:100340000D9420AD0D9403B10C947FD50D946DB236
:100350000D94DF040C943ED40C948DFC0D948AAD66
:100360000D94EE000C943BC00C9456FC0C9420D3DE
:100370000D946DA90D94DB270D944A020C94E9E2CB
:100380000C94BEBE0D9466800C9412860D9494ADB0
:100390000D94DF480C944FC80D94B2AD0C94FEE45C
:1003A0000D94FC780C942BD70D9469060C9480E086
:1003B0000C941CE40C9464970D941C490C94F9FC67
:1003C0000C94BAFF0D94E9040D949E250D940C2A0B
:1003D0000C944FE00D947F9A0D944B740C942E97CF
:1003E0000D941FA30D9422800D94A8AD0D9443ADE0
:1003F0000D948B7E0D9453AD0D94DE260D9425AD9A
:100400000D94E8000C9458BD0D94EB000C943BA5A2
:100410000D9494A90D94124D0D94B0A90D9466B944
:100420000C949EFD0C9493F90C94C6D60C9454D85D
:100430000C94BFE80D9447020D948B9A0C94CEF85F
:100440000D94CE7C0C94FFC80C9406FF0D946AB2F8
:100450000D949AA90D94A47C0D94A29A0D942D4DFF
:100460000D941E7E0D943A770D94A8A90D949EAD1F
:100470000D941CA20D94D5040D94FC7C0C943F9714
:100480000C9467970D9437610D94CC4B0D94829A20
:100490000C944A970D9464020C9455C80D94919A4B
:1004A0000D941E2C0D941BAD0D94E4040C9448CABD
:1004B0000D94CE740D9470B20C945A970D943E2600
:1004C0000D944F800C943ECB0C94F9C80C9444FDD1
:1004D0000D94859A0C942AE10C94F8FD0C94FCC8B8
:1004E0000D942FAD0D9413800D9482A90D94C973B2
:1004F0000C94DEFB0C941DFB0D9467AD0D945DAD6B
:100500000D943EA30D9432A30D94889A0D949202FB
:100510000D94FE7C0D94C17E0D94F3040C9452FE58
:100520000C9458FA0D9439AD0D940F4A0D94F7AD13
:100530000D94A2A90D94DC020D94E60C0C9428975E
:100540000D94BC750C94ECD20D9402A30D94ED2681
:100550000D94B6800D94C47E0D941D7E0C94DABA71
:100560000D9450630C9412E60D9449800C945697A8
:100570000C943ECA0D944BAD0D949EA90C94C0D61C
:100580000D9407A30D94969A0D948CA90C94A3D95D
:100590000D94E50C0D94A9020D9480AD0C944BE7DD
:1005A0000C94B4DD0D94B5A90C9449CE0D94DA04E5
:1005B0004E414E494E495459494E46CDCCCC3D0A48
:1005C000D7233C17B7D13877CC2B329595E6241F2B
:1005D000B14F0A000020410000C84200401C4620E4
:1005E000BCBE4CCA1B0E5AAEC59D7400407A10F3B7
:1005F0005A00A0724E18090010A5D4E80000E87651
:1006000048170000E40B54020000CA9A3B000000A7
:10061000E1F505000080969800000040420F0000C0
:1006200000A08601000000102700000000E8030081
:100630000000006400000000000A0000000000014B
:1006400000000000002C76D888DC674F0823DFC14B
:10065000DFAE59E1B1B796E5E3E453C63AE6519906
:100660007696E8E6C28426EB898C9B62ED407C6F2F
:10067000FCEFBC9C9F40F2BAA56FA5F490055A2AE6
:10068000F75C936B6CF9676DC11BFCE0E40D47FEF2
:10069000F520E6B500D0ED902E03009435770500E7
:1006A00080841E080000204E0A000000C80C33336E
:1006B00033330F986E12831141EF8D2114893BE67D
:1006C0005516CFFEE6DB18D1844B381BF77C1D9006
:1006D0001DA4BBE424203284725E228100C9F1246F
:1006E000ECA1E53D27434F4D4D554E4943415449FB
:1006F0004F4E0044525952554E004552524F52539C
:1007000000494E464F004543484F0047322F47337C
:100710002062616420706172616D65746572730A34
:1007200000536C6565702E2E2E00205A3A20002052
:10073000593A200042656420583A20004D6573689C
:1007400020706F696E742063616E6E6F74206265D5
:10075000207265736F6C7665640A00436C69636B25
:1007600020746F20726573756D652E2E2E004E6F8E
:10077000206D6F76652E00456E642066696C65207D
:100780006C6973740A00426567696E2066696C65FE
:10079000206C6973740A004D31323500286E6F2069
:1007A00066696C65290043757272656E74206669AE
:1007B0006C653A200046696C652064656C657465FB
:1007C000643A0044656C6574696F6E206661696C9B
:1007D00065642C2046696C653A2000256973002504
:1007E000696D20256973002569682025696D2025BC
:1007F000697300256964202569682025696D2025B5
:100800006973002569792025696420256968202598
:10081000696D20256973005072696E742074696D6A
:10082000653A20006F6E2E0A006F66662E0A00473A
:100830003236204465627567200006070107FA0614
:10084000F306E5066F66660044454255473A004D9B
:100850003131332053006F6B00466F726D626F74DD
:10086000204F66662E00544845524D414C5F505211
:100870004F54454354494F4E004155544F524550F3
:100880004F52545F53445F53544154555300454DA8
:10089000455247454E43595F5041525345520043DC
:1008A0004153455F4C494748545F42524947485479
:1008B0004E45535300544F47474C455F4C494748BA
:1008C000545300534F4654574152455F504F57457C
:1008D00052004255494C445F50455243454E5400E6
:1008E0004C4556454C494E475F44415441005A5F80
:1008F00050524F4245004155544F4C4556454C00CF
:100900005052494E545F4A4F420050524F47524551
:100910005353004155544F5245504F52545F544524
:100920004D5000564F4C554D455452494300454596
:1009300050524F4D0053455249414C5F584F4E5F06
:10094000584F4646004649524D574152455F4E4129
:100950004D453A4D61726C696E20627567666978C3
:100960002D312E312E782028476974687562292030
:10097000534F555243455F434F44455F55524C3AA0
:1009800068747470733A2F2F6769746875622E6388
:100990006F6D2F4D61726C696E4669726D77617211
:1009A000652F4D61726C696E2050524F544F434F0A
:1009B0004C5F56455253494F4E3A312E30204D41EF
:1009C0004348494E455F545950453A466F726D62EF
:1009D0006F742045585452554445525F434F554E0D
:1009E000543A3220555549443A6365646532613260
:1009F000662D343161322D343734382D396231323D
:100A00002D6335356336326633363766660A002F16
:100A10002F20004D31343520533C696E6465783E9B
:100A2000206F7574206F662072616E6765202830B4
:100A30002D31290A00205400205200416363656C67
:100A400065726174696F6E3A2050003F4A206F757D
:100A500074206F662072616E67652028302E3031F9
:100A600020746F20302E33290A0020466C6F773AAD
:100A7000200000013637260302FFFF353C3D38FFDA
:100A80000FFFFF312E303E12FFFFFFFF28FFFF0850
:100A9000090CFFFF1A1C18FFFF2A24221EFFFF2C3F
:100AA00008440A0643072D452A2B2CFF206F757436
:100AB000206F662072616E67650A00536572766FFB
:100AC00020003A200020536572766F200050726F2C
:100AD0006265205A204F66667365743A2000432988
:100AE0000A0061626C656420286D696E2074656D12
:100AF000702000436F6C6420657874727564657350
:100B000020617265200020643A0020693A0020705C
:100B10003A0043617365206C696768743A206F66B8
:100B2000660A0043617365206C696768743A206FD8
:100B30006E0A00454550524F4D204F4B0A003F5A18
:100B4000206F7574206F662072616E676520282D96
:100B5000323020746F203230290A003A200050725F
:100B60006F6265205A204F666673657400656E710A
:100B700075657565696E672022000000A04200005F
:100B8000A04200008040000000005761726E696E54
:100B9000673A20486F6D696E672042756D7020441A
:100BA000697669736F72203C20310A0002020400EA
:100BB00000A0400000A040000000400000F64300FC
:100BC00000C8430000FA43FF01FF4D3630303A20A1
:100BD000546F6F20636F6C6400486F74656E64209F
:100BE000746F6F20636F6C640A002F2F61637469E8
:100BF0006F6E3A70617573650A007C3C3E5E2B3DFA
:100C00003F2F5B5D3B2C2A225C002C2065653D005C
:100C10002C207A653D002C2079653D002075626CA2
:100C20002E6C696E655F746F5F64657374696E6165
:100C300074696F6E5F63617274657369616E287841
:100C4000653D0020746F6F206C6F6E67206578744F
:100C5000727573696F6E2070726576656E74656407
:100C60000A0020636F6C6420657874727573696F15
:100C70006E2070726576656E7465640A00627573C5
:100C8000793A2070617573656420666F7220696EB1
:100C90007075740A00627573793A207061757365B6
:100CA0006420666F7220757365720A0062757379CD
:100CB0003A2070726F63657373696E670A004B49FF
:100CC0004C4C45442E20004B494C4C2063617573BD
:100CD0006564206279204B494C4C20627574746FB6
:100CE0006E2F70696E0A004B494C4C45442E200013
:100CF0004B494C4C206361757365642062792074A4
:100D00006F6F206D75636820696E616374697665C5
:100D10002074696D65202D2063757272656E742074
:100D2000636F6D6D616E643A20004D363030005057
:100D30006C65617365207265736574005052494E2D
:100D40005445522048414C544544005072696E74D9
:100D500065722068616C7465642E206B696C6C2808
:100D6000292063616C6C6564210A0050726F6269AE
:100D70006E67206661696C65640A0050726F626913
:100D80006E67206661696C656400205A3A20002015
:100D9000593A200042656420583A2000486F6D653A
:100DA0002058592066697273740A00486F6D652077
:100DB00058592066697273740043616E6E6F7420B7
:100DC0006F70656E20737562646972200050726F77
:100DD0007465637465642050696E0A005374616EB3
:100DE0006461726420446576696174696F6E3A204B
:100DF000002052616E67653A2000204D61783A20EC
:100E000000204D696E3A20004D65616E3A20004623
:100E1000696E6973686564210A002072616E676596
:100E20003A2000206D61783A2000206D696E3A20EA
:100E300000207369676D613A2000206D65616E3A2C
:100E400020003A207A3A2000206F662000205A00C5
:100E5000205900205800476F696E6720746F3A0070
:100E6000436C6F636B776973650A00436F756E74CB
:100E700065722D0020446972656374696F6E3A2053
:100E800000202020616E676C653A20005374617207
:100E900074696E67207261646975733A2000506FDF
:100EA000736974696F6E696E67207468652070720B
:100EB0006F62652E2E2E0A003F4E756D62657220A0
:100EC0006F66206C65677320696E206D6F76656D47
:100ED000656E74206E6F7420706C61757369626CDE
:100EE000652028302D3135292E0A003F2028582C26
:100EF0005929206F7574206F6620626F756E647358
:100F00002E0A003F53616D706C652073697A65200D
:100F10006E6F7420706C61757369626C6520283423
:100F20002D3530292E0A004D3438205A2D50726F3D
:100F30006265205265706561746162696C6974797B
:100F400020546573740A003F2856296572626F73D6
:100F500065206C6576656C20697320696D706C61C5
:100F6000757369626C652028302D34292E0A00457E
:100F700072726F722077726974696E6720746F2065
:100F8000454550524F4D210A00454550524F4D2086
:100F90006461746173697A65206572726F722E0A7A
:100FA00000290A002062797465733B206372632014
:100FB0000053657474696E67732053746F7265644F
:100FC00020280055424C2053797374656D2072655A
:100FD00073657428290A00206C6F6164656420665B
:100FE000726F6D2073746F726167652E0A004D65B4
:100FF000736820002E0A003F43616E277420656EDF
:1010000061626C65200020696E697469616C697A3F
:1010100065642E0A0A00290A002062797465733B10
:101020002063726320002073746F7265642073659F
:101030007474696E6773207265747269657665642D
:10104000202800202863616C63756C6174656429D5
:10105000210A0020213D2000454550524F4D20439C
:101060005243206D69736D61746368202D2028736D
:10107000746F7265642920002053697A653A2000F4
:10108000496E6465783A2000204D61726C696E3D4E
:10109000563535290A0028454550524F4D3D0045EB
:1010A0004550524F4D2076657273696F6E206D69A1
:1010B000736D6174636820001000AA03F0013A01A7
:1010C0009002220130031001D00302017004F700E6
:1010D0001005ED00B005E5005006DD00F006D70074
:1010E0009007D1003008CC00D008C7007009C300B9
:1010F000100ABE00B00ABB00500BB700F00BB300E3
:10110000900CB000D00DAA00100FA5005010A00048
:1011100090119B00D0129600B014900090168B0096
:1011200070188500501A8000301C7B00B01E7500BE
:1011300030216F00B02369003026640010285F0062
:10114000902A5A00702C5500F02E4F007031480044
:10115000B0324500F03341007036390010373700A7
:101160005038330090392D00D03A2700B03C1C0095
:10117000503D1700F03D1100903E0900D03FE5FFC3
:101180002000A401C1005E01CC005901D900540126
:10119000E7004F01F5004A01060145011701400132
:1011A0002A013B013E013601540131016C012C0141
:1011B00086012701A3012201C2011D01E4011801DA
:1011C0000902130131020E01670209018E020401B6
:1011D000C302FF00FD02FA003C03F5008303F000A8
:1011E000D003EB002404E6008104E100E804DC0005
:1011F0005905D700D505D2005E06CD00F506C8001A
:101200009B07C3005208BE001B09B900F909B400CE
:10121000EB0AAF00F50BAA00180DA500550EA000B3
:10122000AE0F9B0024119600B712910068148C0039
:101230003716870022188200281A7D00461C780085
:10124000791E7300BD206E000B2369005E256400CB
:10125000AF275F00F8295A00332C5500582E500054
:10126000BA304B009932460016344100B8353C0084
:101270003437370088383200B6392D00BE3A28009E
:10128000A43B2300693C1E00113D19009E3D140043
:10129000163E0F00763E0A00C63E0500083F0000DD
:1012A0003C3FFBFF663FF6FF873FF1FFA13FECFFAE
:1012B000B53FE7FFC53FE2FFD03FDDFFD93FD8FF95
:1012C000E03FD3FFE43FCEFF24F404D9201BC40C3D
:1012D0005C0E9804C4095F0265077101F405F9000A
:1012E000FB04B30048048700C1036900580355009C
:1012F00003034500BE023A008402310053022A0073
:101300002902250004022000E4011C00C801190084
:10131000AF0117009801140084011300710110003F
:101320006101100051010E0043010D0036010B0058
:101330002B010B0020010B00150109000C01090015
:1013400003010800FB000800F3000800EB000700A1
:10135000E4000600DE000600D8000600D200060009
:10136000CC000500C7000500C2000500BD00040058
:10137000B9000400B5000400B1000400AD00040091
:10138000A9000400A5000300A20003009F000400C0
:101390009B000300980003009500020093000300E7
:1013A000900003008D0002008B0003008800020003
:1013B0008600020084000300810002007F0002001A
:1013C0007D0002007B00020079000200770001002E
:1013D0007600020074000200720001007100020039
:1013E0006F0002006D0001006C0002006A00010045
:1013F000690002006700010066000100650001004D
:101400006400020062000100610001006000010050
:101410005F0002005D0001005C0001005B00010054
:101420005A00010059000100580001005700010056
:101430005600010055000100540001005300000057
:101440005300010052000100510001005000010052
:101450004F0001004E0000004E0001004D00010051
:101460004C0001004B0000004B0001004A0001004D
:101470004900010048000000480001004700010049
:101480004600000046000100450000004500010044
:10149000440001004300000043000100420000003E
:1014A0004200010041000000410001004000010035
:1014B0003F0000003F0001003E0000003E00010030
:1014C0003D0000003D0001003C0000003C00000029
:1014D0003C0001003B0000003B0001003A0000001E
:1014E0003A00010039000000390001003800000016
:1014F000380000003800010037000000370001000C
:101500003600000036000000360001003500000003
:1015100035000000350001003400000034000000F8
:1015200034000100330000003300000033000100EC
:1015300032000000320000003200010031000000E3
:1015400031000000310001003000000030000000D8
:10155000300001002F0000002F0000002F000000CD
:101560002F0001002E0000002E0000002E000100C0
:101570002D0000002D0000002D0000002D000100B6
:101580002C0000002C0000002C0000002C000100AA
:101590002B0000002B0000002B0000002B0001009E
:1015A0002A0000002A0000002A0000002A00010092
:1015B0002900000029000000290000002900000087
:1015C0002900010028000000280000002800000079
:1015D000280000002800010027000000270000006C
:1015E000270000002700000027000100260000005F
:1015F0002600000026000000260000002600010052
:101600002500000025000000250000002500000046
:101610002500000025000100240000002400000037
:10162000240000002400000024000100230000002A
:10163000230000002300000023000000230000001E
:10164000230000002300010022000000220000000F
:101650002200000022000000220000002200010001
:1016600021000000210000002100000021000000F6
:1016700021000000210000002100010020000000E6
:1016800020000000200000002000000020000000DA
:101690002000000020000000200001001F000000CA
:1016A0001F0000001F0000001F0000001F000000BE
:1016B0001F0000001F0001001E0000001E000000AF
:1016C0001E0000001E00000024F4D43050C38E2001
:1016D000C2A24017828B7011127A910D816CD90AC7
:1016E000A861E108C7586607615143061E4B5D05B6
:1016F000C145A7041A411104093D9803713931030A
:101700004036DB0265339102D4305402802E1D0234
:10171000632CEE01752AC501B028A00110278101B4
:101720008F2564012B244B01E0223401AC211F01E1
:101730008D200D01801FFC00841EED00971DDF0031
:10174000B81CD200E61BC600201BBC00641AB20005
:10175000B219A8000A19A0006A189900D1179100BF
:1017600040178B00B516840031167E00B315790042
:101770003A157300C7146F0058146A00EE13660020
:101780008813630025135E00C7125B006C125700BC
:1017900015125400C111510070114F0021114B005E
:1017A000D61049008D104700461044000210420038
:1017B000C00F4000800F3E00420F3C00060F3B0070
:1017C000CB0E3800930E37005C0E3500270E340028
:1017D000F30D3200C10D3100900D3000600D2E0070
:1017E000320D2D00050D2C00D90C2B00AE0C29005C
:1017F000850C29005C0C2700350C27000E0C2600F8
:10180000E80B2400C40B2400A00B23007D0B230055
:101810005A0B2100390B2100180B2000F80A1F0079
:10182000D90A1E00BB0A1E009D0A1D00800A1D0069
:10183000630A1C00470A1B002C0A1B00110A1A002D
:10184000F7091A00DD091900C4091900AB091900CC
:10185000920917007B091800630917004C0916004C
:1018600036091600200916000A091500F5081500AA
:10187000E0081400CC081400B8081400A4081400F0
:10188000900813007D0812006B081300580812001E
:101890004608120034081100230811001208110034
:1018A00001081100F0071000E0071000D007100039
:1018B000C0071000B0070F00A107100091070E002D
:1018C00083070F0074070F0065070E0057070E000F
:1018D00049070E003B070D002E070E0020070D00E4
:1018E00013070D0006070D00F9060C00ED060D00AC
:1018F000E0060C00D4060C00C8060C00BC060C0068
:10190000B0060C00A4060B0099060C008D060B0017
:1019100082060B0077060B006C060B0061060A00BE
:1019200057060B004C060A0042060A0038060A0059
:101930002E060A0024060A001A060A0010060900EC
:1019400007060A00FD050900F4050900EB0509007A
:10195000E2050900D9050900D0050900C7050900FD
:10196000BE050900B5050800AD050800A50509007C
:101970009C050800940508008C05080084050800F3
:101980007C050800740508006C0507006505080063
:101990005D050700560508004E05070047050700CE
:1019A0004005080038050700310507002A05070033
:1019B000230507001C050600160507000F05070094
:1019C0000805060002050700FB040600F5040700F1
:1019D000EE040600E8040600E2040700DB0406004B
:1019E000D5040600CF040600C9040600C30406009F
:1019F000BD040600B7040600B1040500AC040600EF
:101A0000A6040600A00405009B040600950405003A
:101A1000900406008A040500850405008004060081
:101A20007A04050075040500700405006B040500C8
:101A300066040500610405005C0405005704050008
:101A4000520405004D040500480405004304050048
:101A50003E0404003A040500350405003004040087
:101A60002C04050027040400230405001E040400C0
:101A70001A04040016040500110404000D040400F7
:101A8000090405000404040000040400FC0304002D
:101A9000F8030400F4030400F0030400EC03040062
:101AA000E8030400E4030400E0030400DC03040092
:101AB000D8030400D4030400D0030400CC030400C2
:101AC000C8030300C50303000A4D657368206F6EE9
:101AD0006C79207061727469616C6C7920706F70C0
:101AE000756C617465642E0A0024F404D9201BC44B
:101AF0000C5C0E9804C4095F0265077101F405F9D6
:101B000000FB04B30048048700C103690058035573
:101B10000003034500BE023A008402310053022A4A
:101B2000002902250004022000E4011C00C801195C
:101B300000AF011700980114008401130071011017
:101B4000006101100051010E0043010D0036010B30
:101B5000002B010B0020010B00150109000C0109ED
:101B60000003010800FB000800F3000800EB000779
:101B700000E4000600DE000600D8000600D20006E1
:101B800000CC000500C7000500C2000500BD000430
:101B900000B9000400B5000400B1000400AD000469
:101BA00000A9000400A5000300A20003009F000498
:101BB000009B0003009800030095000200930003BF
:101BC00000900003008D0002008B000300880002DB
:101BD000008600020084000300810002007F0002F2
:101BE000007D0002007B0002007900020077000106
:101BF0000076000200740002007200010071000211
:101C0000006F0002006D0001006C0002006A00011C
:101C10000069000200670001006600010065000124
:101C20000064000200620001006100010060000128
:101C3000005F0002005D0001005C0001005B00012C
:101C4000005A00010059000100580001005700012E
:101C5000005600010055000100540001005300002F
:101C6000005300010052000100510001005000012A
:101C7000004F0001004E0000004E0001004D000129
:101C8000004C0001004B0000004B0001004A000125
:101C90000049000100480000004800010047000121
:101CA000004600000046000100450000004500011C
:101CB0000044000100430000004300010042000016
:101CC000004200010041000000410001004000010D
:101CD000003F0000003F0001003E0000003E000108
:101CE000003D0000003D0001003C0000003C000001
:101CF000003C0001003B0000003B0001003A0000F6
:101D0000003A0001003900000039000100380000ED
:101D100000380000003800010037000000370001E3
:101D200000360000003600000036000100350000DB
:101D300000350000003500010034000000340000D0
:101D400000340001003300000033000000330001C4
:101D500000320000003200000032000100310000BB
:101D600000310000003100010030000000300000B0
:101D700000300001002F0000002F0000002F0000A5
:101D8000002F0001002E0000002E0000002E000198
:101D9000002D0000002D0000002D0000002D00018E
:101DA000002C0000002C0000002C0000002C000182
:101DB000002B0000002B0000002B0000002B000176
:101DC000002A0000002A0000002A0000002A00016A
:101DD000002900000029000000290000002900005F
:101DE0000029000100280000002800000028000051
:101DF0000028000000280001002700000027000044
:101E00000027000000270000002700010026000036
:101E10000026000000260000002600000026000129
:101E2000002500000025000000250000002500001E
:101E3000002500000025000100240000002400000F
:101E40000024000000240000002400010023000002
:101E500000230000002300000023000000230000F6
:101E600000230000002300010022000000220000E7
:101E700000220000002200000022000000220001D9
:101E800000210000002100000021000000210000CE
:101E900000210000002100000021000100200000BE
:101EA00000200000002000000020000000200000B2
:101EB000002000000020000000200001001F0000A2
:101EC000001F0000001F0000001F0000001F000096
:101ED000001F0000001F0001001E0000001E000087
:101EE000001E0000001E00000024F4D43050C38EF9
:101EF00020C2A24017828B7011127A910D816CD989
:101F00000AA861E108C7586607615143061E4B5D88
:101F100005C145A7041A411104093D9803713931DF
:101F2000034036DB0265339102D4305402802E1D0B
:101F300002632CEE01752AC501B028A0011027818B
:101F4000018F2564012B244B01E0223401AC211FB9
:101F5000018D200D01801FFC00841EED00971DDF08
:101F600000B81CD200E61BC600201BBC00641AB2DD
:101F700000B219A8000A19A0006A189900D1179197
:101F80000040178B00B516840031167E00B315791A
:101F9000003A157300C7146F0058146A00EE1366F8
:101FA000008813630025135E00C7125B006C125794
:101FB0000015125400C111510070114F0021114B36
:101FC00000D61049008D1047004610440002104210
:101FD00000C00F4000800F3E00420F3C00060F3B48
:101FE00000CB0E3800930E37005C0E3500270E3400
:101FF00000F30D3200C10D3100900D3000600D2E48
:1020000000320D2D00050D2C00D90C2B00AE0C2933
:1020100000850C29005C0C2700350C27000E0C26CF
:1020200000E80B2400C40B2400A00B23007D0B232D
:10203000005A0B2100390B2100180B2000F80A1F51
:1020400000D90A1E00BB0A1E009D0A1D00800A1D41
:1020500000630A1C00470A1B002C0A1B00110A1A05
:1020600000F7091A00DD091900C4091900AB0919A4
:1020700000920917007B091800630917004C091624
:102080000036091600200916000A091500F5081582
:1020900000E0081400CC081400B8081400A40814C8
:1020A00000900813007D0812006B081300580812F6
:1020B000004608120034081100230811001208110C
:1020C0000001081100F0071000E0071000D0071011
:1020D00000C0071000B0070F00A107100091070E05
:1020E0000083070F0074070F0065070E0057070EE7
:1020F0000049070E003B070D002E070E0020070DBC
:102100000013070D0006070D00F9060C00ED060D83
:1021100000E0060C00D4060C00C8060C00BC060C3F
:1021200000B0060C00A4060B0099060C008D060BEF
:102130000082060B0077060B006C060B0061060A96
:102140000057060B004C060A0042060A0038060A31
:10215000002E060A0024060A001A060A00100609C4
:102160000007060A00FD050900F4050900EB050952
:1021700000E2050900D9050900D0050900C70509D5
:1021800000BE050900B5050800AD050800A5050954
:10219000009C050800940508008C050800840508CB
:1021A000007C050800740508006C0507006505083B
:1021B000005D050700560508004E050700470507A6
:1021C000004005080038050700310507002A05070B
:1021D00000230507001C050600160507000F05076C
:1021E000000805060002050700FB040600F50407C9
:1021F00000EE040600E8040600E2040700DB040623
:1022000000D5040600CF040600C9040600C3040676
:1022100000BD040600B7040600B1040500AC0406C6
:1022200000A6040600A00405009B04060095040512
:1022300000900406008A0405008504050080040659
:10224000007A04050075040500700405006B0405A0
:102250000066040500610405005C040500570405E0
:1022600000520405004D0405004804050043040520
:10227000003E0404003A040500350405003004045F
:10228000002C04050027040400230405001E040498
:10229000001A04040016040500110404000D0404CF
:1022A00000090405000404040000040400FC030405
:1022B00000F8030400F4030400F0030400EC03043A
:1022C00000E8030400E4030400E0030400DC03046A
:1022D00000D8030400D4030400D0030400CC03049A
:1022E00000C8030300C50303005374617274206FB8
:1022F000662075626C2E6C696E655F746F5F6465D5
:102300007374696E6174696F6E5F63617274657313
:1023100069616E2829006F7574206F6620626F7581
:102320006E647320696E2075626C2E6C696E655FD9
:10233000746F5F64657374696E6174696F6E5F63F7
:10234000617274657369616E28290046494E414C7B
:102350005F4D4F564520696E2075626C2E6C696E1C
:10236000655F746F5F64657374696E6174696F6EC5
:102370005F63617274657369616E282900766572A6
:10238000746963616C206D6F766520646F6E652083
:10239000696E2075626C2E6C696E655F746F5F6428
:1023A000657374696E6174696F6E5F636172746581
:1023B0007369616E282900686F72697A6F6E746143
:1023C0006C206D6F766520646F6E6520696E207578
:1023D000626C2E6C696E655F746F5F64657374699F
:1023E0006E6174696F6E5F63617274657369616E4B
:1023F00028290067656E65726963206D6F766520B8
:10240000646F6E6520696E2075626C2E6C696E65F6
:102410005F746F5F64657374696E6174696F6E5F1A
:1024200063617274657369616E2829004D6F766906
:102430006E672E2E2E004D61696E004C69676874C0
:10244000204252494748544E455353004C696768EF
:1024500074204252494748544E455353004C6967D3
:102460006874204252494748544E455353004361D3
:102470007365206C69676874004F6E20004F666654
:102480000043617365206C6967687400326E642074
:102490006E6F7A7A6C65205800326E64206E6F7AA7
:1024A0007A6C65205900326E64206E6F7A7A6C65A2
:1024B000205A0043617365206C69676874005A2D67
:1024C0004F66667365743A20004175746F20686FBB
:1024D0006D6500473238004175746F74656D70002A
:1024E0005049442D49204531005049442D44204550
:1024F00031005049442D49204532005049442D4473
:1025000020453200416363656C00412D7265747231
:1025100061637400412D74726176656C004A756E5A
:102520006374696F6E2044657600587374657073C8
:102530002F6D6D005973746570732F6D6D005A7334
:10254000746570732F6D6D004573746570732F6DB6
:102550006D0046696C2E204469612E0046696C2E20
:10256000204469612E20310046696C2E2044696147
:102570002E2032005072696E742066726F6D205387
:1025800044005072696E742066726F6D205344006F
:102590004368616E67652066696C616D656E740085
:1025A000696E206D6F76655F746F2829206665659A
:1025B000645F76616C756520666F722058593A00C9
:1025C0004C656176696E67204732360047323620A7
:1025D00048656174696E67204E6F7A7A6C652E006B
:1025E0004732362048656174696E67204265642E03
:1025F00000446F6E65205072696D696E6700557397
:1026000065722D436F6E74726F6C6C6564205072CE
:10261000696D65004669786564204C656E6774680D
:10262000205072696D652E004D6573682056616C8F
:1026300069646174696F6E2053746F707065642E85
:10264000002C2065793D0029202D3E202865783D0D
:10265000002C2073793D0020436F6E6E65637469B2
:102660006E67207769746820766572746963616C3F
:10267000206C696E65202873783D002C2065793DBB
:102680000029202D3E202865783D002C2073793DBF
:102690000020436F6E6E656374696E67207769749E
:1026A0006820686F72697A6F6E74616C206C696EF5
:1026B00065202873783D004C656176696E67204718
:1026C0003236003F53706563696669656420582C33
:1026D0005920636F6F7264696E617465206F7574E1
:1026E000206F6620626F756E64732E0A003F285259
:1026F0002965706561742076616C7565206E6F74F4
:1027000020706C61757369626C653B206D757374C4
:10271000206265206174206C6561737420312E0A1B
:10272000003F537065636966696564206E6F7A7AED
:102730006C652074656D7065726174757265206E6C
:102740006F7420706C61757369626C652E0A003F4E
:102750005370656369666965642066696C616D655F
:102760006E742073697A65206E6F7420706C617569
:102770007369626C652E0A003F5370656369666910
:102780006564207072696D65206C656E6774682081
:102790006E6F7420706C61757369626C652E0A00CF
:1027A0003F537065636966696564206E6F7A7A6C01
:1027B000652073697A65206E6F7420706C61757323
:1027C00069626C652E0A003F5370656369666965CE
:1027D000642052657472616374696F6E204D756C0C
:1027E0007469706C696572206E6F7420706C6175AD
:1027F0007369626C652E0A003F526574726163747E
:10280000696F6E204D756C7469706C696572206DAE
:1028100075737420626520737065636966696564A9
:102820002E0A003F537065636966696564206C61B8
:1028300079657220686569676874206E6F742070AE
:102840006C61757369626C652E0A003F5370656335
:102850006966696564206265642074656D7065727F
:102860006174757265206E6F7420706C6175736928
:10287000626C65202834302D31343043292E0A0013
:1028800047323620636F6D6D616E642073746172C0
:102890007465642E2057616974696E6720666F7273
:1028A000206865617465722873292E0A0020746F90
:1028B0006F206C6F6E6720657874727573696F6EC8
:1028C0002070726576656E7465640A0020636F6CB3
:1028D0006420657874727573696F6E2070726576A6
:1028E000656E7465640A00436172642072656D6F81
:1028F000766564004361726420696E736572746505
:10290000640000060900FE0701920321207FFF07F3
:10291000FF07FF0000000600000107070602008015
:10292000808080800080030202060105A0A00507C8
:10293000070600005050F850F850500507070600F1
:10294000002078A07028F020050707060000C0C806
:1029500010204098180507070600006090A040A8C6
:102960009068020303060104C040800307070601C4
:10297000002040808080402003070706010080403F
:10298000202020408005050506000120A870A82011
:102990000505050600012020F82020020303060299
:1029A000FFC04080050101060003F8020202060292
:1029B00000C0C0050505060001081020408005077D
:1029C000070600007088888888887003070706015A
:1029D0000040C040404040E0050707060000708806
:1029E00008708080F8050707060000F8102010081E
:1029F00008F005070706000010305090F810100589
:102A00000707060000F880F0080888700507070629
:102A10000000708080F0888870050707060000F8C5
:102A20000810202020200507070600007088887005
:102A30008888700507070600007088887808087085
:102A4000020505060200C0C000C0C002060606025C
:102A5000FFC0C000C04080040707060000102040EF
:102A600080402010050303060002F800F804070761
:102A70000601008040201020408005070706000066
:102A800070880810200020050707060000708808DD
:102A900068A8A870050707060000708888F888886D
:102AA00088050707060000F08888F08888F0050789
:102AB0000706000070888080808870050707060080
:102AC00000F08888888888F0050707060000F880ED
:102AD00080F08080F8050707060000F88080F0800D
:102AE0008080050707060000708880B88888700518
:102AF0000707060000888888F88888880107070685
:102B000002008080808080808005070706000038F2
:102B10001010101090600507070600008890A0C0F4
:102B2000A09088050707060000808080808080F8DC
:102B300005070706000088D8A88888888805070741
:102B40000600008888C8A89888880507070600003E
:102B500070888888888870050707060000F08888D4
:102B6000F080808005070706000070888888A8909C
:102B700068050707060000F08888F0A09088050720
:102B800007060000788080700808F0050707060037
:102B900000F8202020202020050707060000888854
:102BA00088888888700507070600008888888888D4
:102BB00050200507070600008888888888A85005E7
:102BC00007070600008888502050888805070706F8
:102BD000000088888850202020050707060000F89C
:102BE0000810204080F8030707060100E08080807D
:102BF0008080E005050506000180402010080307DD
:102C000007060100E02020202020E0050303060045
:102C100004205088050101060000F80202020602A5
:102C200005804005050506000070087888780507CE
:102C3000070600008080B0C88888F00505050600FA
:102C400000708080887005070706000008086898F3
:102C50008888780505050600007088F880700507EB
:102C6000070600003048E0404040400506060600E8
:102C7000FF7088887808700507070600008080B01C
:102C8000C88888880107070602008000808080804D
:102C9000800308080601FF200020202020A0400417
:102CA0000707060000808090A0C0A09003070706D9
:102CB0000100C04040404040E0050505060000D04E
:102CC000A8A8A8A8050505060000B0C8888888053A
:102CD000050506000070888888700506060600FF56
:102CE000F08888F080800506060600FF78888878DE
:102CF0000808050505060000B0C8808080050505A8
:102D000006000070807008F00407070600004040CD
:102D1000E040404030050505060000888888986836
:102D20000505050600008888885020050505060071
:102D3000008888A8A8500505050600008850205086
:102D4000880506060600FF8888887808700505054E
:102D5000060000F8102040F8030707060100204095
:102D6000408040402001070706020080808080806C
:102D70008080030707060100804040204040800516
:102D8000020206000268900000000600004D657314
:102D900068204C6576656C696E67004564697420CF
:102DA0004D6573680056616C6964617465204D659A
:102DB0007368004D616E75616C6C79204275696C49
:102DC00064204D6573680047323920493939390A22
:102DD0004732392050322042205430004275696C0D
:102DE00064204D65736800556E69666965642042AC
:102DF0006564204C6576656C696E670037205361A9
:102E0000766520426564204D65736800362046690A
:102E10006E652054756E6520416C6C004732392018
:102E200050342052393939205400352056616C69AC
:102E300064617465204D65736800342046696E6571
:102E40002054756E6520416C6C0047323920503437
:102E50002052393939205400332056616C6964613D
:102E60007465204D657368003220536D6172742063
:102E700046696C6C2D696E004732392050332054FE
:102E8000300031204275696C6420436F6C64204DC2
:102E9000657368004732380A47323920503100558F
:102EA0006E696669656420426564204C6576656C70
:102EB000696E6700466164652048656967687400EB
:102EC00046616465204865696768740046616465A9
:102ED00020486569676874004F7574707574205573
:102EE000424C20496E666F004732392057005542E8
:102EF0004C20546F6F6C73004F7574707574204D57
:102F0000657368204D6170004D6573682053746F60
:102F100072616765004D657368204564697400538C
:102F20007465702D42792D537465702055424C00A4
:102F3000446561637469766174652055424C00474D
:102F400032392044004163746976617465205542CA
:102F50004C00473239204100507265706172650043
:102F60004D343238004D3238302050302053313615
:102F70003000424C546F7563682053656C662D5465
:102F8000657374004D323830205030205331323068
:102F9000005072656865617420414253005072654B
:102FA0006865617420504C4100436F6F6C646F77AB
:102FB0006E004368616E67652066696C616D656E61
:102FC000740044697361626C652073746570706528
:102FD0007273004D38340053657420686F6D65203E
:102FE0006F66667365747300526573657420424C36
:102FF000546F756368004C6576656C20636F726E04
:1030000065727300556E6966696564204265642067
:103010004C6576656C696E6700486F6D65205A0077
:10302000473238205A00486F6D65205900473238C2
:10303000205900486F6D65205800473238205800ED
:103040004175746F20686F6D6500473238004D6FB1
:1030500076652061786973004D61696E004D6F7609
:10306000652058004D6F76652059004D6F766520BC
:103070005A004578747275646572320045787472CE
:103080007564657231004D6F766520302E316D6D3F
:10309000004D6F766520316D6D004D6F7665203186
:1030A000306D6D004D6F76652061786973004578ED
:1030B000747275646572004D6F7665205A004D6FAD
:1030C00076652059004D6F76652058004368616E23
:1030D00067652066696C616D656E740050726F6221
:1030E00065205A204F666673657400466C6F7720C2
:1030F0003200466C6F77203200466C6F77203200CA
:10310000466C6F77203100466C6F77203100466C3B
:103110006F77203100466C6F7700466C6F77004602
:103120006C6F770046616E207370656564203200B5
:1031300046616E20737065656420320046616E20C2
:10314000737065656420320046616E20737065653A
:103150006420310046616E20737065656420310023
:1031600046616E20737065656420310042656400BD
:1031700042656400426564004E6F7A7A6C65203265
:10318000004E6F7A7A6C652032004E6F7A7A6C65E9
:103190002032004E6F7A7A6C652031004E6F7A7A59
:1031A0006C652031004E6F7A7A6C65203100466183
:1031B00064652048656967687400466164652048F5
:1031C0006569676874004661646520486569676879
:1031D00074005370656564005370656564005370D6
:1031E000656564004D61696E005072656865617463
:1031F00020504C4120416C6C0050726568656174D0
:1032000020504C4120456E64204532005072656864
:1032100065617420504C41203200507265686561D0
:103220007420504C4120456E642045310050726539
:103230006865617420504C4120426564005072659D
:103240006865617420504C41203100507265706196
:103250007265005072656865617420414253204177
:103260006C6C005072656865617420414253204562
:103270006E64204532005072656865617420414279
:1032800053203200507265686561742041425320BA
:10329000456E642045310050726568656174204157
:1032A0004253204265640050726568656174204134
:1032B0004253203100507265706172650042616353
:1032C0006B004E65787420636F726E6572004732D2
:1032D00039205031004D31303920532569004D31AE
:1032E00039302053256900473238004275696C64D3
:1032F00020437573746F6D204D657368004265647B
:103300002054656D70004265642054656D70004204
:1033100065642054656D7000486F74656E64205458
:10332000656D7000486F74656E642054656D700043
:10333000486F74656E642054656D70004275696CE9
:1033400064204D657368002E25690047323920508E
:10335000362043202D00496E666F207363726565C9
:103360006E0048656967687420416D6F756E740002
:1033700048656967687420416D6F756E74004865B3
:103380006967687420416D6F756E74004564697477
:10339000204D65736800496E666F207363726565C2
:1033A0006E0041646A757374204D657368204865CA
:1033B000696768740046696E652054756E652043C0
:1033C0006C6F736573740047323920503420540099
:1033D00046696E652054756E6520416C6C004732FD
:1033E00039205034205239393920540055424C206C
:1033F000546F6F6C730047323800473236204320D9
:1034000042256920482569205000496E666F207367
:10341000637265656E0056616C6964617465204312
:103420007573746F6D204D6573680056616C6964C7
:1034300061746520414253204D65736800473238FE
:103440000A47323620432042313130204832323070
:1034500020500056616C696461746520504C4120B5
:103460004D657368004732380A47323620432042A0
:103470003730204831393020500055424C20546FAD
:103480006F6C7300473239204A2569004C657665B8
:103490006C204D657368005369646520506F696ED8
:1034A0007473005369646520506F696E74730053C0
:1034B00069646520506F696E74730055424C2054E6
:1034C0006F6F6C7300496E666F2073637265656E13
:1034D0000047726964204D657368204C6576656CA1
:1034E000696E6700332D506F696E74204C65766588
:1034F0006C696E6700473239204A300055424C20D3
:10350000546F6F6C73004732392050332052204380
:103510002E256900496E666F2073637265656E00C3
:103520004D616E75616C2046696C6C2D696E00474B
:103530003239205032204220543000536D61727471
:103540002046696C6C2D696E00473239205033205B
:1035500054300046696C6C2D696E20416D6F756E3C
:10356000740046696C6C2D696E20416D6F756E74C8
:103570000046696C6C2D696E20416D6F756E74002C
:103580004275696C64204D657368004D65736820F1
:10359000696E76616C6964617465642E0A00496EB7
:1035A000666F2073637265656E00496E76616C6943
:1035B0006461746520436C6F7365737400473239BE
:1035C000204900496E76616C696461746520416CC4
:1035D0006C00436F6E74696E756520426564204DA2
:1035E0006573680047323920503120430046696CCA
:1035F0006C2D696E204D657368004275696C64209E
:10360000436F6C64204D657368004732380A473257
:1036100039205031004275696C6420437573746FB2
:103620006D204D657368004275696C64204142539A
:10363000204D657368004732380A4D3139302053C8
:103640003131300A4D31303920533232300A47326D
:10365000392050310A4D3130342053300A4D313445
:1036600030205330004275696C6420504C41204D2D
:10367000657368004732380A4D313930205337308E
:103680000A4D31303920533139300A473239205010
:10369000310A4D3130342053300A4D31343020530B
:1036A000300055424C20546F6F6C73004D313137F0
:1036B000204D657368202569207361766564004735
:1036C000323920532569004D313137204D657368FB
:1036D000202569206C6F6164656400473239204C95
:1036E0002569005361766520426564204D657368E5
:1036F000004C6F616420426564204D657368004D25
:10370000656D6F727920536C6F74004D656D6F72CB
:103710007920536C6F74004D656D6F727920536C16
:103720006F74004E6F2073746F7261676500556E21
:10373000696669656420426564204C6576656C69DC
:103740006E6700486F6D696E672058595A0047329E
:10375000392050342058257320592573205225696B
:1037600000202D2D2D2D2D000000A040B76D03420F
:103770006EDB72429224B1426EDBE842254910436F
:1037800092242C43000048436EDB6343DCB67F4346
:1037900025C98D43DCB69B4392A4A9434992B74304
:1037A0000080C543B76DD3430000A040B76D03420E
:1037B0006EDB72429224B1426EDBE842254910432F
:1037C00092242C43000048436EDB6343DCB67F4306
:1037D00025C98D43DCB69B4392A4A9434992B743C4
:1037E0000080C543B76DD343473238004F757470BE
:1037F0007574204D657368204D6170004F666620BA
:103800005072696E746572204261636B7570004717
:10381000323920532D31004F757470757420666FE6
:10382000722043535600473239205431004F75748B
:1038300070757420666F7220486F73740047323958
:1038400020543000556E69666965642042656420C5
:103850004C6576656C696E67000E00000F01000D07
:10386000000F01000F0E0000000F000D003A2000B5
:10387000454550524F4D2044756D703A0A00206600
:10388000726F6D2063757272656E74206D657368FA
:103890002E0A005375627472616374696E67206DDD
:1038A00065736820696E20736C6F7420003F5573D8
:1038B00065203020746F20003F496E76616C69642A
:1038C0002073746F7261676520736C6F742E0A00C9
:1038D0003F557365203020746F20003F53746F7222
:1038E00061676520736C6F74202320726571756940
:1038F0007265642E0A003F454550524F4D20737447
:103900006F72616765206E6F7420617661696C61AA
:10391000626C652E0A004D657368204564697469A0
:103920006E672053746F7070656400446F6E65201D
:1039300045646974696E67204D6573680A00446F59
:103940006E652045646974696E67204D6573680013
:1039500046696E652054756E696E67204D657368A3
:103960000028582C5929206F75747369646520707C
:1039700072696E7461626C65207261646975732E20
:103980000A004F6666736574206F7574206F662039
:10399000626F756E64732E20283020746F20313072
:1039A0006D6D290A0A00683863385E3859385D0A37
:1039B0000062656420706C616E65206E6F726D616F
:1039C0006C203D205B00436F756C64206E6F74202B
:1039D000636F6D706C657465204C53462100436FB6
:1039E000727265637465645F5A3D003F4572726F21
:1039F000722070726F62696E6720706F696E742ECC
:103A0000202041626F7274696E67206F7065726109
:103A100074696F6E2E0A00436F7272656374656419
:103A20005F5A3D00436F727265637465645F5A3D0F
:103A300000436F727265637465645F5A3D00505352
:103A4000553A2047656E657269630050726F746FF6
:103A5000636F6C3A20312E3000426175643A203237
:103A6000353030303000466F726D626F7400556EC5
:103A7000696669656420426564204C6576656C6999
:103A80006E67004578747275646572733A2032000F
:103A9000687474703A2F2F6D61726C696E66772E40
:103AA0006F726700466F726D626F7400323031382A
:103AB0002D30372D3331006275676669782D312ED0
:103AC000312E78004D61726C696E00546865726DBC
:103AD0006973746F727300426F61726420496E661D
:103AE0006F005072696E74657220496E666F004D8A
:103AF00061696E004D37303220542564004D3630F8
:103B00003020423020542564004D373032203B2590
:103B100064004D37303120542564004D363030205C
:103B20004230205431004368616E67652066696CDD
:103B3000616D656E74204532004D36303020423064
:103B4000205430004368616E67652066696C616D62
:103B5000656E742045310050726570617265005069
:103B600052494E542050415553454400554E4C4FF8
:103B700041442046494C414D454E54004C4F414430
:103B80002046494C414D454E5400507572676520A2
:103B90006D6F726500436F6E74696E756500524596
:103BA00053554D45204F5054494F4E533A00202015
:103BB0004E6F7A7A6C653A20006368616E676500C3
:103BC0006F66207468652066696C616D656E74004F
:103BD0005761697420666F7220737461727400207B
:103BE000204E6F7A7A6C653A2000200066696C611D
:103BF0006D656E7420756E6C6F61640057616974D9
:103C000020666F720020204E6F7A7A6C653A200031
:103C10002000506C6561736520776169742E2E2ECB
:103C20000048656174696E67206E6F7A7A6C650012
:103C300020204E6F7A7A6C653A200020006865611A
:103C400074206E6F7A7A6C652E00507265737320E3
:103C5000627574746F6E20746F0020204E6F7A7AD4
:103C60006C653A2000746F20636F6E74696E7565C1
:103C70002E2E2E00616E6420707265737320627543
:103C800074746F6E00496E736572742066696C613E
:103C90006D656E740020204E6F7A7A6C653A200054
:103CA000200066696C616D656E74206C6F616400E4
:103CB0005761697420666F720020204E6F7A7A6CAB
:103CC000653A2000200066696C616D656E74207035
:103CD00075726765005761697420666F7200746F52
:103CE00020726573756D65005761697420666F7227
:103CF000207072696E7400457874727564657232F2
:103D00000045787472756465723100457874727517
:103D10006465720053656C656374204532005431EC
:103D20000053656C656374204531005430004D6F5D
:103D30007665205A004D6F76652059004D6F766587
:103D40002058005072657061726500496E6974692F
:103D5000616C697A6520454550524F4D00436F6E46
:103D600074726F6C00526573746F7265206661695E
:103D70006C73616665004C6F61642073657474696F
:103D80006E677300496E697469616C697A65204574
:103D90004550524F4D0053746F72652073657474B3
:103DA000696E677300424C546F7563680046696CB6
:103DB000616D656E74004D6F74696F6E0054656D52
:103DC0007065726174757265004D61696E004D3386
:103DD0003033205531204525692053256900507224
:103DE00065686561742041425320636F6E660050C0
:103DF00072656865617420504C4120636F6E660087
:103E0000504944204175746F74756E6520453200C9
:103E1000504944204175746F74756E6520453200B9
:103E2000504944204175746F74756E6520453200A9
:103E30005049442D44204532005049442D442045EA
:103E400032005049442D49204532005049442D4903
:103E5000204532005049442D5020453200504944FD
:103E60002D50204532005049442D502045320050FD
:103E70004944204175746F74756E6520453100505A
:103E80004944204175746F74756E6520453100504A
:103E90004944204175746F74756E6520453100503A
:103EA00049442D44204531005049442D442045319A
:103EB000005049442D49204531005049442D4920A6
:103EC0004531005049442D50204531005049442D82
:103ED00050204531005049442D50204531002008E4
:103EE0002046616374002008204661637400200846
:103EF0002046616374002008204D6178002008206E
:103F00004D6178002008204D6178002008204D691F
:103F10006E002008204D696E002008204D696E005B
:103F20004F6666004F6E20004175746F74656D704A
:103F30000046616E20737065656420320046616ED4
:103F400020737065656420320046616E2073706571
:103F5000656420320046616E2073706565642031AF
:103F60000046616E20737065656420310046616EA5
:103F700020737065656420310042656400426564A9
:103F800000426564004E6F7A7A6C652032004E6F95
:103F90007A7A6C652032004E6F7A7A6C6520320036
:103FA0004E6F7A7A6C652031004E6F7A7A6C65209C
:103FB00031004E6F7A7A6C65203100436F6E7472F7
:103FC0006F6C0053544F505045442E20005072697E
:103FD0006E7465722073746F7070656420647565AB
:103FE00020746F206572726F72732E20466978207C
:103FF000746865206572726F7220616E64207573DB
:1040000065204D39393920746F207265737461727F
:10401000742E202854656D70657261747572652008
:1040200069732072657365742E20536574206974FA
:104030002061667465722072657374617274696E52
:1040400067290A004E6F20436865636B73756D20A6
:1040500077697468206C696E65206E756D62657233
:104060002C204C617374204C696E653A20004E6FB1
:1040700020436865636B73756D2077697468206C85
:10408000696E65206E756D6265722C204C6173746B
:10409000204C696E653A2000636865636B73756DCB
:1040A000206D69736D617463682C204C617374209A
:1040B0004C696E653A20004C696E65204E756D62E4
:1040C0006572206973206E6F74204C617374204C8C
:1040D000696E65204E756D6265722B312C204C61C6
:1040E0007374204C696E653A20004D313130004DBB
:1040F00033310053442072656164206572726F72BF
:104100000A00446F6E65207072696E74696E672074
:1041100066696C650A0020496E76616C6964206589
:10412000787472756465722000000028C200000077
:1041300000000000000000E1430000C8430000FA56
:1041400043486F6D6520257325732573206669725A
:104150007374002066697273740A005A005900581B
:1041600000486F6D65200053544F505045442E2039
:10417000005072696E7465722073746F707065643C
:104180002064756520746F206572726F72732E20C3
:1041900046697820746865206572726F7220616E5E
:1041A0006420757365204D39393920746F2072652C
:1041B00073746172742E202854656D706572617419
:1041C0007572652069732072657365742E2053655E
:1041D00074206974206166746572207265737461FD
:1041E0007274696E67290A0053544F502063616CE2
:1041F0006C65642062656361757365206F6620423B
:104200004C546F756368206572726F72202D207236
:104210006573746172742077697468204D39393917
:104220000A0024F4D43050C38E20C2A24017828BDF
:104230007011127A910D816CD90AA861E108C758F2
:104240006607615143061E4B5D05C145A7041A412F
:104250001104093D9803713931034036DB0265339F
:104260009102D4305402802E1D02632CEE01752A77
:10427000C501B028A001102781018F2564012B24DE
:104280004B01E0223401AC211F018D200D01801F64
:10429000FC00841EED00971DDF00B81CD200E61B59
:1042A000C600201BBC00641AB200B219A8000A198B
:1042B000A0006A189900D117910040178B00B5161D
:1042C000840031167E00B31579003A157300C714C7
:1042D0006F0058146A00EE136600881363002513FC
:1042E0005E00C7125B006C12570015125400C1111A
:1042F000510070114F0021114B00D61049008D1054
:1043000047004610440002104200C00F4000800FDA
:104310003E00420F3C00060F3B00CB0E3800930ED0
:1043200037005C0E3500270E3400F30D3200C10D4E
:104330003100900D3000600D2E00320D2D00050D66
:104340002C00D90C2B00AE0C2900850C29005C0C2C
:104350002700350C27000E0C2600E80B2400C40BA8
:104360002400A00B23007D0B23005A0B2100390BE6
:104370002100180B2000F80A1F00D90A1E00BB0AF2
:104380001E009D0A1D00800A1D00630A1C00470ACA
:104390001B002C0A1B00110A1A00F7091A00DD097C
:1043A0001900C4091900AB091900920917007B090B
:1043B0001800630917004C09160036091600200979
:1043C00016000A091500F5081500E0081400CC08CD
:1043D0001400B8081400A4081400900813007D0805
:1043E00012006B0813005808120046081200340827
:1043F0001100230811001208110001081100F00734
:104400001000E0071000D0071000C0071000B00730
:104410000F00A107100091070E0083070F0074071B
:104420000F0065070E0057070E0049070E003B07F7
:104430000D002E070E0020070D0013070D000607C4
:104440000D00F9060C00ED060D00E0060C00D40688
:104450000C00C8060C00BC060C00B0060C00A4063C
:104460000B0099060C008D060B0082060B007706E8
:104470000B006C060B0061060A0057060B004C0689
:104480000A0042060A0038060A002E060A00240620
:104490000A001A060A001006090007060A00FD05B0
:1044A0000900F4050900EB050900E2050900D9053A
:1044B0000900D0050900C7050900BE050900B505BA
:1044C0000800AD050800A50509009C050800940535
:1044D00008008C050800840508007C0508007405A8
:1044E00008006C050700650508005D050700560516
:1044F00008004E050700470507004005080038057D
:104500000700310507002A050700230507001C05E1
:104510000600160507000F0507000805060002053E
:104520000700FB040600F5040700EE040600E8049B
:104530000600E2040700DB040600D5040600CF04F1
:104540000600C9040600C3040600BD040600B70443
:104550000600B1040500AC040600A6040600A00491
:1045600005009B04060095040500900406008A04DB
:10457000050085040500800406007A040500750422
:104580000500700405006B04050066040500610465
:1045900005005C04050057040500520405004D04A5
:1045A000050048040500430405003E0404003A04E5
:1045B000050035040500300404002C040500270420
:1045C0000400230405001E0404001A040400160459
:1045D0000500110404000D0404000904050004048E
:1045E000040000040400FC030400F8030400F403C6
:1045F0000400F0030400EC030400E8030400E403F7
:104600000400E0030400DC030400D8030400D40326
:104610000400D0030400CC030400C8030300C50356
:10462000030024F404D9201BC40C5C0E9804C409B4
:104630005F0265077101F405F900FB04B30048044B
:104640008700C10369005803550003034500BE02FB
:104650003A008402310053022A0029022500040294
:104660002000E4011C00C8011900AF0117009801E7
:104670001400840113007101100061011000510148
:104680000E0043010D0036010B002B010B00200131
:104690000B00150109000C01090003010800FB00D3
:1046A0000800F3000800EB000700E4000600DE004D
:1046B0000600D8000600D2000600CC000500C700A6
:1046C0000500C2000500BD000400B9000400B500EB
:1046D0000400B1000400AD000400A9000400A5001E
:1046E0000300A20003009F0004009B000300980049
:1046F00003009500020093000300900003008D006A
:1047000002008B0003008800020086000200840083
:104710000300810002007F0002007D0002007B0098
:1047200002007900020077000100760002007400A8
:10473000020072000100710002006F0002006D00B3
:1047400001006C0002006A000100690002006700BD
:1047500001006600010065000100640002006200C3
:10476000010061000100600001005F0002005D00C7
:1047700001005C0001005B0001005A0001005900CB
:1047800001005800010057000100560001005500CB
:1047900001005400010053000000530001005200CA
:1047A000010051000100500001004F0001004E00C7
:1047B00000004E0001004D0001004C0001004B00C4
:1047C00000004B0001004A000100490001004800C0
:1047D00000004800010047000100460000004600BC
:1047E00001004500000045000100440001004300B5
:1047F00000004300010042000000420001004100AF
:10480000000041000100400001003F0000003F00A7
:1048100001003E0000003E0001003D0000003D00A0
:1048200001003C0000003C0000003C0001003B0097
:1048300000003B0001003A0000003A00010039008E
:104840000000390001003800000038000000380086
:10485000010037000000370001003600000036007C
:104860000000360001003500000035000000350072
:104870000100340000003400000034000100330067
:10488000000033000000330001003200000032005D
:104890000000320001003100000031000000310052
:1048A00001003000000030000000300001002F0047
:1048B00000002F0000002F0000002F0001002E003C
:1048C00000002E0000002E0001002D0000002D0031
:1048D00000002D0000002D0001002C0000002C0025
:1048E00000002C0000002C0001002B0000002B0019
:1048F00000002B0000002B0001002A0000002A000D
:1049000000002A0000002A00010029000000290000
:1049100000002900000029000000290001002800F3
:1049200000002800000028000000280000002800E7
:1049300001002700000027000000270000002700DA
:1049400000002700010026000000260000002600CD
:1049500000002600000026000100250000002500C0
:1049600000002500000025000000250000002500B3
:1049700001002400000024000000240000002400A6
:104980000000240001002300000023000000230099
:10499000000023000000230000002300000023008B
:1049A000010022000000220000002200000022007E
:1049B0000000220000002200010021000000210070
:1049C0000000210000002100000021000000210063
:1049D0000000210001002000000020000000200055
:1049E0000000200000002000000020000000200047
:1049F0000000200001001F0000001F0000001F0039
:104A000000001F0000001F0000001F0000001F002A
:104A100001001E0000001E0000001E0000001E001D
:104A20000000043700001E290000511B0000581030
:104A3000000010090000CC040000780200004101D1
:104A40000000466F726D626F742052656164792E4A
:104A5000005072696E74696E672E2E2E0050726956
:104A60006E74207061757365640053746F772042B3
:104A70004C546F756368004D3238302050302053ED
:104A80003930004465706C6F7920424C546F756307
:104A900068004D3238302050302053313000424CC5
:104AA000546F7563682053656C662D54657374008C
:104AB0004D3238302050302053313230005265733F
:104AC000657420424C546F756368004D3238302055
:104AD00050302053313630004D61696E004D353015
:104AE00032200A204D353030200A204D353031201B
:104AF0000A205430200A204D3139302053373520D8
:104B00000A204D3130362053313238200A204D31C1
:104B100030342053323235200A20473238200A20E0
:104B2000473239205031200A204732392053312072
:104B30000A204D3131372052756E20537465702034
:104B400032200A00473239205331200A20473239B7
:104B5000205330200A2047323920462031302E3071
:104B6000200A204732392041200A204D353030209C
:104B70000A20473238200A20473239204C31200A97
:104B8000205430200A204D31303620533132382025
:104B90000A204D3130392053323235200A20473136
:104BA0002058313530205920313530200A20473106
:104BB000205A30200A204D31313720536574205A55
:104BC000204F6666736574200A004D3139302037F6
:104BD00035200A205430200A204D31303620533100
:104BE0003238200A204D31303420323235200A202C
:104BF000473238200A20473239204C31200A2047DA
:104C0000312058313530205920313530200A2047A5
:104C100031205A30200A00473239205033200A20F0
:104C2000473239205033200A204732392050332070
:104C30000A204732392054200A00473236200A0021
:104C400046696C6C204D65736820506F696E747393
:104C5000005072657020666F72205A2041646A7538
:104C600073740055424C20436F6D6D697373696FA7
:104C70006E205374657020320052756E204D65733E
:104C8000682056616C69646174696F6E0055424CAE
:104C900020436F6D6D697373696F6E205374657017
:104CA0002031004D61696E004732380053617665EE
:104CB000204F666673657473004D35303000326E78
:104CC00064206E6F7A7A6C65205A00326E64206EB2
:104CD0006F7A7A6C65205A00326E64206E6F7A7A31
:104CE0006C65205900326E64206E6F7A7A6C652094
:104CF0005900326E64206E6F7A7A6C6520580032EB
:104D00006E64206E6F7A7A6C6520580046756C6C04
:104D100020636F6E74726F6C004D363035205330E7
:104D20000A4732382058004D6972726F72004D3652
:104D300030352053310A54300A4D36303520533245
:104D400020583230300A47323820580A473120582C
:104D50003130300A4D363035205333205832303020
:104D6000004D3630352053310A54300A4732380A64
:104D70004D36303520533220583230300A473238E1
:104D800020580A473120583130300A4D363035200E
:104D900053332058323030004475706C696361744D
:104DA000696F6E004D3630352053310A54300A4D4C
:104DB00036303520533220583230300A47323820CE
:104DC000580A47312058313030004D3630352053A5
:104DD000310A54300A4732380A4D363035205332C2
:104DE00020583230300A47323820580A473120588C
:104DF000313030004175746F2D5061726B004D364B
:104E000030352053310A47323820580A473120586C
:104E1000313030004D61696E004D313235004D3218
:104E200034005072696E742061626F727465640040
:104E300049444558204D6F6465004E6F205344200F
:104E400063617264005072696E742066726F6D20C7
:104E500053440053746F70207072696E7400526511
:104E600073756D65207072696E740041626F757440
:104E7000205072696E7465720050617573652070A0
:104E800072696E7400436F6E74726F6C005072655D
:104E9000706172650054756E65004F6666004F6EF6
:104EA000200043617365206C696768740043617317
:104EB00065206C6967687400437573746F6D204377
:104EC0006F6D6D616E647300496E666F20736372FF
:104ED00065656E000E000E000E000E000E000E0046
:104EE0000E000E007FC03F801F000E000400040073
:104EF0000E001F003F807FC00E000E000E000E004F
:104F00000E000E000E000E0003F8000FFE001E0F34
:104F100000380700380380700380700FE07007C00E
:104F20007003807001007000003800003807001E18
:104F30000F000FFE0003F80000FE0003FF80078350
:104F4000C00E01C00E00E01C00E07F00E03E00E06B
:104F50001C00E00800E00000E00001C00E01C00FEE
:104F6000078007FF0001FC00FFFFFF7F80FFC0FFFD
:104F7000C0FFC07F807F80FFC0FFC0FFC03F001E1A
:104F8000000C0050726F6265205A204F6666736590
:104F900074004D65736820456469746F7200205712
:104FA0003A0045256920436F6F6C696E672E2E2E7F
:104FB000004525692048656174696E672E2E2E00B4
:104FC00020573A0042656420636F6F6C696E672EEC
:104FD0002E2E004265642068656174696E672E2E0E
:104FE0002E00205A3A0020593A0020436F756E7403
:104FF00020583A0020453A00205A3A0020593A00F9
:10500000583A004469666665723A200046726F6DD0
:105010005374703A00537465707065723A0052614F
:10502000773A20202020000A4C6F676963616C3A50
:10503000002C20002C20003A004361703A00205AD6
:1050400000205900580020204D61783A2000205A55
:1050500000205900580020204D696E3A20004F6E04
:1050600020004F666600536F667420656E6473742B
:105070006F70733A2000486F74656E64206F6666C7
:10508000736574733A00496E76616C696420657863
:105090007472756465720A0020643A0020693A00EF
:1050A00020703A0020653A004B6420002364656656
:1050B000696E652044454641554C545F004B69205C
:1050C0000023646566696E652044454641554C542D
:1050D0005F004B70200023646566696E652044455F
:1050E0004641554C545F00504944204175746F74DB
:1050F000756E652066696E697368656421205075F8
:105100007420746865206C617374204B702C204B84
:105110006920616E64204B6420636F6E7374616EEE
:1051200074732066726F6D2062656C6F7720696E94
:10513000746F20436F6E66696775726174696F6E14
:105140002E680A00504944204175746F74756E656D
:10515000206661696C6564212074696D656F757482
:105160000A00453220544845524D414C2052554E7C
:105170004157415900453120544845524D414C203A
:1051800052554E41574159004245442054484552DA
:105190004D414C2052554E4157415900546865725B
:1051A0006D616C2052756E617761790045322048DF
:1051B000656174696E67206661696C65640045317C
:1051C0002048656174696E67206661696C6564007A
:1051D0004265642068656174696E67206661696C08
:1051E00065640048656174696E67206661696C6515
:1051F0006400504944204175746F74756E65206673
:1052000061696C6564212054656D706572617475A7
:10521000726520746F6F20686967680A00204B64AC
:105220003A2000204B693A2000204B703A20000AB7
:1052300020436C617373696320504944200A002045
:1052400054753A2000204B753A2000206D61783A61
:105250002000206D696E3A200020643A2000206210
:105260006961733A2000504944204175746F747528
:105270006E65206661696C6564212054656D70659A
:1052800072617475726520746F6F20686967680A4F
:1052900000504944204175746F74756E65207374B5
:1052A0006172740A00504944204175746F74756EC0
:1052B00065206661696C65642120426164206578BF
:1052C000747275646572206E756D6265720A002075
:1052D00000A401C1005E01CC005901D9005401E7CE
:1052E000004F01F5004A0106014501170140012A5E
:1052F000013B013E013601540131016C012C018654
:10530000012701A3012201C2011D01E401180109C5
:1053100002130131020E01670209018E020401C36A
:1053200002FF00FD02FA003C03F5008303F000D009
:1053300003EB002404E6008104E100E804DC0059EA
:1053400005D700D505D2005E06CD00F506C8009B46
:1053500007C3005208BE001B09B900F909B400EBED
:105360000AAF00F50BAA00180DA500550EA000AE5F
:105370000F9B0024119600B712910068148C00371F
:1053800016870022188200281A7D00461C780079B2
:105390001E7300BD206E000B2369005E256400AF04
:1053A000275F00F8295A00332C5500582E5000BAB8
:1053B000304B009932460016344100B8353C003479
:1053C00037370088383200B6392D00BE3A2800A49D
:1053D0003B2300693C1E00113D19009E3D14001640
:1053E0003E0F00763E0A00C63E0500083F00003C26
:1053F0003FFBFF663FF6FF873FF1FFA13FECFFB5A4
:105400003FE7FFC53FE2FFD03FDDFFD93FD8FFE0D8
:105410003FD3FFE43FCEFF202F002040002042403A
:105420003A0020403A00556E69666965642042651D
:1054300064204C6576656C696E6700205A00204ACE
:105440000020204D343231204900202047323920BD
:10545000493939390A006163746976652E0A006931
:105460006E002053797374656D2076312E303120B3
:10547000002020207C0A004E414E0020202E2020BB
:105480002000207C004C43443A0A004353563A0A19
:105490000020666F7220003A0A0A000A4265642002
:1054A000546F706F677261706879205265706F72A7
:1054B00074003F4D65736820746F6F2062696720C8
:1054C000666F7220454550524F4D2E0A00446F6E54
:1054D000652E0A003F557365203020746F20003F11
:1054E000496E76616C69642073746F7261676520C0
:1054F000736C6F742E0A003F454550524F4D207318
:10550000746F72616765206E6F7420617661696C7B
:1055100061626C652E0A00446F6E652E0A003F556D
:105520007365203020746F20003F496E76616C698E
:10553000642073746F7261676520736C6F742E0AD8
:10554000003F454550524F4D2073746F726167653F
:10555000206E6F7420617661696C61626C652E0AE1
:10556000004732392050322066696E69736865647D
:105570002E0A005859206F75747369646520707223
:10558000696E7461626C65207261646975732E0A5C
:10559000003F4572726F7220696E20427573696EAA
:1055A0006573732043617264206D65617375726504
:1055B0006D656E742E0A004D616E75616C6C79209C
:1055C00070726F62696E6720756E72656163686183
:1055D000626C65206D657368206C6F636174696FC0
:1055E0006E732E0A00292E0A0A0050726F62696ECD
:1055F00067204D65736820506F696E747320436C2B
:105600006F7365737420746F2028004D6573682074
:10561000696E76616C6964617465642E2050726F86
:1056200062696E67206D6573682E0A004D65736848
:10563000207A65726F65642E0A0044656661756C38
:10564000742073746F7261676520736C6F7420309F
:105650002073656C65637465642E0A004C6F616429
:10566000696E6720746573745F7061747465726EBF
:105670002076616C7565732E0A0A00496E76616C3E
:10568000696420746573745F7061747465726E20F0
:1056900076616C75652E20282D3120746F2032299B
:1056A0000A0A004C6F636174696F6E7320696E76CD
:1056B000616C6964617465642E0A0A00456E7469E0
:1056C0007265204D65736820696E76616C696461EE
:1056D0007465642E0A0A0057726974696E672074D3
:1056E0006F2066696C653A20006F70656E20666198
:1056F000696C65642C2046696C653A20006F7065A2
:105700006E206661696C65642C2046696C653A2080
:105710000046696C652073656C65637465640A0096
:105720002053697A653A200046696C65206F706580
:105730006E65643A20002066696C653A2000646FEB
:10574000696E67006672657368004E6F772000456A
:105750004E4420535542524F5554494E450A00225B
:1057600020706F73002220706172656E743A22009F
:10577000535542524F5554494E452043414C4C20BD
:105780007461726765743A22004B494C4C45442E53
:105790002000747279696E6720746F2063616C6C8D
:1057A000207375622D67636F64652066696C65732D
:1057B000207769746820746F6F206D616E79206C3A
:1057C0006576656C732E204D4158206C6576656C4E
:1057D0002069733A004572726F723A006F70656E9D
:1057E000206661696C65642C2046696C653A20000E
:1057F00043616E6E6F74206F70656E2073756264A6
:10580000697220006563686F3A00534420707269C2
:105810006E74696E67206279746520004E6F742023
:105820005344207072696E74696E670A004D657327
:105830006820736176656420696E20736C6F7420D4
:105840000020736C6F743D00206D65736865735F35
:10585000656E643D004532454E443D004D657368BC
:10586000206C6F616465642066726F6D20736C6F6D
:1058700074200048617264636F64656420446566E7
:1058800061756C742053657474696E6773204C6F16
:10589000616465640A00DC050000F4010000900109
:1058A0000000A00F0000000048430000C8420000B4
:1058B000A04000007A430000A0420000A042000087
:1058C00048440000BA4220204D36303320003A0AC6
:1058D0000020286D6D29002055005431204C0020F7
:1058E00055005430204C0046696C616D656E742023
:1058F0006C6F61642F756E6C6F6164206C656E6790
:105900007468733A0A0020204D383531205A005A05
:105910002D50726F6265204F666673657400204477
:105920000020490020204D33303420500020440016
:1059300020490020204D33303120500020440020E9
:10594000490020500020204D33303120450050497F
:10595000442073657474696E67733A0A00204600C8
:1059600020420020480020204D3134352053004D86
:105970006174657269616C2068656174757020700E
:105980006172616D65746572733A0A00206D6573AA
:105990006865732E0A0A00454550524F4D206361D9
:1059A0006E20686F6C6420000A416374697665201C
:1059B0004D65736820536C6F743A2000205A0020A4
:1059C000204D3432302053003A0A00205A0020592A
:1059D0000020580020204D323138205400486F7488
:1059E000656E64206F6666736574733A0A00205AA8
:1059F0000020590020204D323036205800486F6D6D
:105A000065206F66667365743A0A00204A00205468
:105A10000020530020204D323035205100204A3CD8
:105A20006A756E635F6465763E00416476616E639D
:105A300065643A20513C6D696E5F7365676D656E94
:105A4000745F74696D655F75733E20533C6D696E5C
:105A50005F66656564726174653E20543C6D696E75
:105A60005F74726176656C5F6665656472617465AA
:105A70003E0020540020520020204D32303420506F
:105A800000416363656C65726174696F6E2028758F
:105A90006E6974732F7332293A20503C7072696EAC
:105AA000745F616363656C3E20523C726574726121
:105AB00063745F616363656C3E20543C747261760D
:105AC000656C5F616363656C3E0A00204500205A87
:105AD0000020590020204D3230312058004D61788F
:105AE000696D756D20416363656C65726174696F82
:105AF0006E2028756E6974732F7332293A0A00205C
:105B00004500205A0020590020204D3230332058C3
:105B1000004D6178696D756D2066656564726174AC
:105B200065732028756E6974732F73293A0A0020F3
:105B30004500205A0020590020204D3932205800BD
:105B400053746570732070657220756E69743A0ABB
:105B50000020204D3230302044300A0020204D32C9
:105B6000303020543120440020204D323030204449
:105B7000002044697361626C65640A0046696C6167
:105B80006D656E742073657474696E67733A002076
:105B9000204D3134392043203B20556E69747320E9
:105BA000696E2043656C736975730A002020473263
:105BB00031202020203B00486F6D696E67206661B0
:105BC000696C656400545249474745524544006F2B
:105BD00070656E003A200066696C616D656E7400D8
:105BE0007A5F6D696E00795F6D617800785F6D61D5
:105BF0007800785F6D696E005265706F7274696EBF
:105C00006720656E6473746F70207374617475734C
:105C10000A0000091200FC0A01E803D720FFFD0E6C
:105C2000FD0BFD00000009000E010B0B09040080B4
:105C30008080808080800000808004040409030745
:105C400090909090080A0A090000242424FF24243C
:105C5000FF242424070B0B0901FF107C929050387D
:105C60001412927C10070A0A09010042A4A44810E9
:105C700010244A4A84070A0A090100609090906043
:105C80006294889462010404090407808080800380
:105C90000C0C0903FF2040408080808080804040C1
:105CA00020030C0C0903FF804040202020202020EE
:105CB000404080070707090103109254385492109E
:105CC000070707090101101010FE1010100204044C
:105CD0000904FEC0C04080070101090104FE020260
:105CE00002090400C0C0070A0A09010002040408EE
:105CF000101020404080070A0A09010038448282BF
:105D0000828282824438070A0A09010010305090CA
:105D10001010101010FE070A0A0901003844820210
:105D20000408102040FE070A0A090100FE020408C8
:105D3000180402028478070A0A090100040C1424DA
:105D40004484FE040404070A0A090100FE808080DE
:105D5000F80402028478070A0A0901003C408080A6
:105D6000B8C482824438070A0A090100FE0204040A
:105D7000080810101010070A0A090100384482446C
:105D8000384482824438070A0A0901003844828272
:105D9000463A02020478020707090400C0C0000066
:105DA00000C0C00209090904FEC0C0000000C0C054
:105DB0004080050909090200081020408040201099
:105DC00008070404090102FE0000FE050909090292
:105DD00000804020100810204080070A0A090100B6
:105DE00038448202040810100010070A0A09010052
:105DF00038449AAAAAAAAA9C403C070A0A090100A8
:105E000010282828447C44828282070A0A0901005B
:105E1000F8848284F884828284F8070A0A090100DF
:105E20003C42808080808080423C070A0A09010051
:105E3000F88482828282828284F8070A0A09010039
:105E4000FE808080F880808080FE070A0A090100B9
:105E5000FE808080F88080808080070A0A09010027
:105E600038448280808E82824438070A0A09010001
:105E700082828282FE8282828282050A0A0902006E
:105E8000F82020202020202020F8070A0A090100FD
:105E90003E080808080808888870070A0A090100EF
:105EA00082848890A0D088848282070A0A0901002F
:105EB000808080808080808080FE070A0A0901003F
:105EC0008282C6AA928282828282070A0A0901001D
:105ED0008282C2A2928A86828282070A0A0901000D
:105EE0007C82828282828282827C070A0A09010085
:105EF000F884828284F880808080080B0B0901FF7F
:105F0000384482828282828A443A01070A0A09015D
:105F100000F884828284F890888482070A0A090142
:105F2000007C8280807C020202827C070A0A0901CE
:105F300000FE101010101010101010070A0A0901AE
:105F40000082828282828282824438070A0A0901A0
:105F50000082828244444428282810070A0A090142
:105F6000008282828292929292AA44070A0A0901CE
:105F70000082824428101028448282070A0A0901FC
:105F80000082824428101010101010070A0A09011C
:105F900000FE0204081020408080FE040C0C09035F
:105FA000FFF080808080808080808080F0070A0AF7
:105FB00009010080404020101008040402040C0C69
:105FC0000902FFF010101010101010101010F00740
:105FD0000404090106102844820801010900FFFF9A
:105FE00003030309030A8040200707070901007C17
:105FF00002027E82867A070A0A090100808080BC3C
:10600000C2828282C2BC0707070901007C828080AD
:1060100080827C070A0A0901000202027A868282D3
:1060200082867A0707070901007C8282FE80827CD3
:10603000070A0A0901001C22222020F82020202023
:10604000070A0A0901FD7A84848478807C82827C34
:10605000070A0A090100808080BCC2828282828293
:10606000050A0A090200600000E02020202020F834
:10607000050D0D0902FD1800003808080808080879
:10608000888870070A0A090100808080848890B09F
:10609000C88482050A0A090200E02020202020206E
:1060A0002020F8070707090100EC92929292928251
:1060B000070707090100BCC28282828282070707A4
:1060C0000901007C82828282827C070A0A0901FD22
:1060D000B8C4828282C4B8808080070A0A0901FDA0
:1060E0003A46828282463A02020207070709010005
:1060F0009C6242404040400707070901007C8280C3
:106100007C02827C0709090901002020FC20202054
:1061100020221C0707070901008282828282867A78
:10612000070707090100828244442828100707074F
:106130000901008282929292AA440707070901008E
:1061400082442810284482070A0A0901FD42422499
:1061500024241818109060070707090100FE04089E
:10616000102040FE060B0B0902001C20202020C03E
:10617000202020201C010C0C0904FF8080808080DE
:1061800080808080808080060B0B090100E0101069
:1061900010100C10101010E00703030901076292A1
:1061A0008CFFFFFFFFFFFFFFFFFFFFFFFFFFFFFF72
:1061B000FFFFFFFFFFFFFFFFFFFFFFFFFFFFFFFFEF
:1061C000FFFF00000009000E010B0B090400808096
:1061D0000000808080808080800608080901000817
:1061E000789490A0A47840070A0A0901001C222094
:1061F00020F8202060A25C070606090103827C4487
:10620000447C82070A0A090100828244287C107CAF
:10621000101010010B0B0904FF808080808000802B
:1062200080808080040B0B0902FF6090806090905A
:10623000906010906003020209030BA0A0080909F6
:106240000900013C4299A5A1A599423C050707090F
:106250000103609070907800F807080809010112A6
:1062600024489090482412060404090102FC040406
:1062700004050101090204F80809090900013C426A
:10628000B9A5BDA9A5423C060101090109FC040408
:1062900004090306609090600709090901011010C4
:1062A00010FE10101000FE04060609010460901094
:1062B0006080F004060609010460902010906003DD
:1062C000030309030A2040800709090901FE8282AD
:1062D000828282C6BA8080070A0A0901007E8A8A01
:1062E0008A7A0A0A0A0A0A020202090404C0C004DD
:1062F00003030902FD20906003060609010440C063
:10630000404040E00506060901047088887000F8E6
:106310000708080901019048241212244890070A2E
:106320000A09010040C0404042E60A121A06070A64
:106330000A09010040C040404CF2020C101E070A3E
:106340000A0901006090201092660A121A06070AD4
:106350000A0901001000101020408082827C070E84
:106360000E0901002010080010282828447C4482CF
:106370008282070E0E09010008102000102828282C
:10638000447C44828282070E0E09010010284400DA
:1063900010282828447C44828282070D0D090100C0
:1063A00034580010282828447C44828282070D0D2E
:1063B00009010028280010282828447C4482828271
:1063C000070E0E0901001028281010282828447CE8
:1063D00044828282070A0A0901001E2828284E7872
:1063E0004888888E070D0D0901FD3C428080808021
:1063F0008080423C082418070E0E09010020100876
:1064000000FE808080F880808080FE070E0E0901EB
:106410000008102000FE808080F880808080FE07C9
:106420000E0E09010010284400FE808080F8808054
:106430008080FE070D0D090100282800FE80808065
:10644000F880808080FE050E0E09020040201000BA
:10645000F82020202020202020F8050E0E09020020
:1064600010204000F82020202020202020F8050EB9
:106470000E09020020508800F82020202020202033
:1064800020F8050D0D090200505000F820202020B2
:1064900020202020F8070A0A09010078444242F22D
:1064A0004242424478070D0D0901003458008282AF
:1064B000C2A2928A86828282070E0E0901002010F3
:1064C00008007C82828282828282827C070E0E0990
:1064D0000100081020007C82828282828282827C7B
:1064E000070E0E090100102844007C8282828282FD
:1064F0008282827C070D0D0901003458007C828263
:106500008282828282827C070D0D09010028280088
:106510007C82828282828282827C07070709010153
:1065200082442810284482070C0C0901FF027C8653
:106530008A8A9292A2A2C27C80070E0E09010020D4
:1065400010080082828282828282824438070E0E84
:1065500009010008102000828282828282828244A5
:1065600038070E0E090100102844008282828282C0
:106570008282824438070D0D09010028280082829A
:106580008282828282824438070E0E09010008103E
:10659000200082824428101010101010070A0A09E7
:1065A00001008080FC828282FC808080060A0A09C9
:1065B000010038444448D04844444458070B0B0970
:1065C0000100201008007C02027E82867A070B0BF5
:1065D000090100081020007C02027E82867A070BE7
:1065E0000B090100102844007C02027E82867A0793
:1065F0000A0A0901003458007C02027E82867A076A
:106600000A0A0901002828007C02027E82867A0795
:106610000C0C09010010282810007C02027E8286E2
:106620007A0707070901006C12127E90926C070A24
:106630000A0901FD7C82808080827C104830070B33
:106640000B090100201008007C8282FE80827C07FA
:106650000B0B090100081020007C8282FE80827CE6
:10666000070B0B090100102844007C8282FE808207
:106670007C070A0A0901002828007C8282FE8082A9
:106680007C050C0C0902008040200000E020202046
:106690002020F8050C0C0902001020400000E0202A
:1066A00020202020F8050C0C090200205088000052
:1066B000E02020202020F8050B0B0902005050009C
:1066C00000E02020202020F8070B0B0901004830B3
:1066D00050083C448282824438070A0A0901003487
:1066E0005800BCC28282828282070B0B0901002003
:1066F0001008007C82828282827C070B0B090100D9
:10670000081020007C82828282827C070B0B0901A8
:1067100000102844007C82828282827C070A0A0957
:1067200001003458007C82828282827C070A0A0936
:1067300001002828007C82828282827C0709090964
:10674000010010381000FE00103810070909090177
:10675000FF027C8A8A92A2A27C80070B0B090100AF
:10676000402010008282828282867A070B0B090108
:1067700000081020008282828282867A070B0B0931
:106780000100102844008282828282867A070A0AE7
:106790000901002828008282828282867A070E0EF2
:1067A0000901FD0408100042422424241818109006
:1067B00060070B0B0901FE8080B8C4828282C4B8D6
:1067C0008080070D0D0901FD242400424224242469
:1067D000181810906000060900FE0000000000017B
:1067E000090008FE000005080806000040F0C888FF
:1067F00088987810050808060000C0F888888888FE
:1068000088F80505050600012030F8302005080845
:106810000600002070F820202020E005090906006D
:10682000FF2070A8A8B8888870200509090600FF15
:10683000E080C0B0A8283028280509090600FFF824
:10684000A88888888888A8F8050A0A0600FE2050CB
:1068500050505088A8A8887003030306000340A086
:106860004025753A2530327500253032753A25308D
:1068700032750025756420253032753A2530327521
:1068800000202020202020005A0059002020202015
:10689000005800092000FFFFFF000000000000007A
:1068A0000000003FFFF88000010000000000000031
:1068B0000000003E80F88E00E100000000000000B3
:1068C0000000003980389F00F10000000000000047
:1068D0000000003781D893813900000000000000DB
:1068E00000000037C3D89F81F900000000000000BD
:1068F00000000027C7E89F81F900000000000000A9
:1069000000000023C7F89FB9F100001FE001FE005E
:1069100008208021FF888F28F100003EF003CF007F
:10692000041040206C0880380100003CF003B700E0
:10693000041040206C0880000100003AF003F700CA
:10694000082080206C089FFFF900001EE001EE0087
:1069500010410023FF0891749900001EE001DE0041
:106960002082003FC7889B06A900003EF003BF00BD
:106970002082002FC7C89B54A900003EF003870067
:106980001041003787D89B56A900003FF003FF0055
:106990000820803703D89B549900000FC000FC00EA
:1069A0000000003803389FFFF900000780007800DE
:1069B000FFFFC03E02F8FFFFFF00000300003000B1
:1069C000FFFFC03FFFF8FFFFFF00000000000000D6
:1069D0000000003FFFF88000010000000000000000
:1069E0000000003E00F88E00E10000000000000002
:1069F000000000380F389F00F10000000000000088
:106A0000000000341FD8938139000000000000000E
:106A1000000000361F989F81F90000000000000070
:106A20000000002F1F089F81F900000000000000F7
:106A30000000002F9E089FB9F100001FE001FE003A
:106A40000820802FFC088F28F100003EF003CF00C3
:106A50000410402FDC0880380100003CF003B70030
:106A600004104027EFC880000100003AF003F7004F
:106A70000820802077E89FFFF900001EE001EE006B
:106A8000104100207FE891749900001EE001DE00B3
:106A900020820020F3E89B06A900003EF003BF001F
:106AA00020820021F1E89B54A900003EF0038700FA
:106AB00010410033F0D89B56A900003FF003FF00BF
:106AC00008208037F0589B549900000FC000FC004C
:106AD00000000039E0389FFFF900000780007800CF
:106AE000FFFFC03E00F8FFFFFF0000030000300082
:106AF000FFFFC03FFFF8FFFFFF00000000000000A5
:106B00000000003FFFF880000100000000000000CE
:106B10000000003E00F88E00E100000000000000D0
:106B2000000000383F389F00F10000000000000026
:106B3000000000307E189381390000000000000042
:106B4000000000307C189F81F90000000000000068
:106B5000000000287C089F81F90000000000000070
:106B60000000002C38089FB9F100001FE001FE0072
:106B70000820802F39C88F28F100003EF003CF0095
:106B80000410402FFFE880380100003CF003B700FC
:106B90000410402FC7E880000100003AF003F7001E
:106BA0000820802FFFE89FFFF900001EE001EE00A3
:106BB0001041002739E891749900001EE001DE00C1
:106BC0002082002038689B06A900003EF003BF0029
:106BD000208200207C289B54A900003EF0038700FF
:106BE000104100307C189B56A900003FF003FF00C5
:106BF00008208030FC189B549900000FC000FC0056
:106C000000000039F8389FFFF90000078000780085
:106C1000FFFFC03E00F8FFFFFF0000030000300050
:106C2000FFFFC03FFFF84F66660A004661646520BB
:106C30004865696768742000426564204C65766524
:106C40006C696E6720004661696C656420746F2012
:106C5000656E61626C6520426564204C6576656C8A
:106C6000696E670A0076616C69640A53746F7261B9
:106C7000676520736C6F743A2000696E004D657310
:106C80006820697320003F557365203020746F20A1
:106C9000003F496E76616C69642073746F7261673E
:106CA0006520736C6F742E0A004D65736820706FD9
:106CB000696E742063616E6E6F7420626520726508
:106CC000736F6C7665640A004D34323120696E63EF
:106CD0006F727265637420706172616D6574657244
:106CE0002075736167650A004F666673657473206B
:106CF0006170706C696564004572723A20546F6F00
:106D0000206661722100546F6F2066617220667286
:106D10006F6D207265666572656E636520706F6960
:106D20006E740A00496E736572742066696C616DD9
:106D3000656E7420616E6420707265737320627575
:106D400074746F6E20286F72204D313038290A001C
:106D5000507265737320627574746F6E20286F7241
:106D6000204D3130382920746F2068656174206EA1
:106D70006F7A7A6C650A00496E7365727420666971
:106D80006C616D656E7420616E64207072657373E2
:106D900020627574746F6E20286F72204D31303808
:106DA000290A0046726F6D204D6F646520004D6F9B
:106DB0006465204368616E67652000496E76616C8A
:106DC00069642065787472756465720A0000002831
:106DD000C20000C84300000000416374697665206A
:106DE00045787472756465723A20004A756E6374F2
:106DF000696F6E20446576004A756E6374696F6EC4
:106E000020446576004D6F74696F6E00457374653C
:106E100070732F6D6D004573746570732F6D6D0009
:106E20005A73746570732F6D6D005A737465707347
:106E30002F6D6D005973746570732F6D6D005973EC
:106E4000746570732F6D6D005873746570732F6D5A
:106E50006D005873746570732F6D6D004D6F74699C
:106E60006F6E0053746570732F6D6D004A65726BA1
:106E700000416363656C65726174696F6E0056658D
:106E80006C6F636974790050726F6265205A204F8D
:106E9000666673657400436F6E74726F6C004C6F3E
:106EA0006164206D6D2032004C6F6164206D6D2037
:106EB00032004C6F6164206D6D2032004C6F616454
:106EC000206D6D2031004C6F6164206D6D203100AC
:106ED0004C6F6164206D6D2031004C6F6164206DDA
:106EE0006D004C6F6164206D6D004C6F6164206DAE
:106EF0006D00556E6C6F6164206D6D203200556EB3
:106F00006C6F6164206D6D203200556E6C6F616432
:106F1000206D6D203200556E6C6F6164206D6D20A8
:106F20003100556E6C6F6164206D6D203100556EBF
:106F30006C6F6164206D6D203100556E6C6F616403
:106F4000206D6D00556E6C6F6164206D6D00556E27
:106F50006C6F6164206D6D0046696C2E2044696120
:106F60002E20320046696C2E204469612E203200AA
:106F700046696C2E204469612E20310046696C2ED2
:106F8000204469612E20310046696C2E20446961DD
:106F90002E0046696C2E204469612E004F66660003
:106FA0004F6E20004520696E206D6D3300452069CD
:106FB0006E206D6D3300436F6E74726F6C004361B1
:106FC0006E6E6F7420656E7465722073756264698D
:106FD000723A2000022E2E004D61696E004D6178DC
:106FE0002054656D703A20313530004D696E205463
:106FF000656D703A203500544265643A312520624F
:107000006574612033393530004D61782054656DE9
:10701000703A20333530004D696E2054656D703AFA
:1070200020350054313A20466F726D626F74203300
:107030003530C2B043004D61782054656D703A2000
:10704000333530004D696E2054656D703A2035003F
:1070500054303A20466F726D626F7420333530C2FF
:10706000B04300FFFFFFFFFFFFFFFFFFFFFFFFFF3A
:10707000FFFFFFFFFFFFFFFFFFFFFFFFFFFFFFFF20
:10708000FFFFFFFFFFFFFFFFFFFFFFFFFFFFFFFF10
:10709000FFFFFFFFFFFFFFFFFFFFFFFFFFFFFFFF00
:1070A000FFFFFFFFFFFFFFFFFFFFFFFFFFFFFFFFF0
:1070B000FFFFFFFFFFFFFFFFFFFFFFFFFFFFFFFFE0
:1070C000FFFFFFFD55555555555FFFFFFFFFFFFFC4
:1070D000FFFFFFFE00000000003FFFFFFFFFFFFF7C
:1070E000FFFFFFFD000007FFFFFFFFFFFFFFFFFFA8
:1070F000FFFFFFFE07C00555555555555FFFFFFFC4
:10710000FFFFFFFC0A200600000000003FFFFFFF1A
:10711000FFFFFFFE141005000007FFFFFFFFFFFF4A
:10712000FFFFFFFC28080607C00555555555555F5C
:10713000FFFFFFFE5404040A200600000000003F89
:10714000FFFFFFFC600406141005000007FFFFFFAF
:10715000FFFFFFFE50040428080607C005555555DB
:1071600055555FFC6004065404040A200600000024
:1071700000003FFE54041C600406141005000000CB
:1071800000001FFC28082E50040428080607C00031
:1071900001F03FFE1410546004065404040A200059
:1071A00002081FFC0A206654041C60040614100028
:1071B00005043FFE07C05428082E50040428080088
:1071C0000A021FFC00002E14105460040654040030
:1071D00015013FFE00001C0A206654041C600400D8
:1071E00018011FFC00000607C05428082E50040098
:1071F00014013FFE00000400002E1410546004002F
:1072000018011FFCFFFFFE00001C0A206654041C2E
:1072100015013FFED5555400000607C05428082A22
:107220000A021FFC84104600000400002E141051B6
:1072300005043FFEC41044FFFFFE00001C0A20614D
:1072400002881FFC841046D5555400000607C05123
:1072500001F03FFE84104484104600000400002A20
:1072600000001FFCC41046C41044FFFFFE00001CB9
:1072700000003FFE841044841046D55554000000A1
:1072800000001FFCD55556841044841046000000B1
:1072900000003FFCFFFFFCC41046C41044FFFFFF8A
:1072A000FFFF9FFE000006841044841046D555550C
:1072B0005555BFFD555554D555568410448410413D
:1072C00004109FFFFFFFFCFFFFFCC41046C41041E9
:1072D0000411BFFFFFFFFE0000068410448410412C
:1072E00004109FFFFFFFFD555554D555568410419E
:1072F00004109FFFFFFFFFFFFFFCFFFFFCC41041D6
:107300000411BFFFFFFFFFFFFFFE000006841041D6
:1073100004109FFFFFFFFFFFFFFD555554D5555546
:107320005555BFFFFFFFFFFFFFFFFFFFFCFFFFFF04
:10733000FFFF9FFFFFFFFFFFFFFFFFFFFE000000BB
:1073400000003FFFFFFFFFFFFFFFFFFFFD5555550B
:1073500055555FFFFFFFFFFFFFFFFFFFFFFFFFFF31
:10736000FFFFFFFFFFFFFFFFFFFFFFFFFFFFFFFF2D
:10737000FFFFFFFFFFFFFFFFFFFFFFFFFFFFFFFF1D
:10738000FFFFFFFFFFFFFFFFFFFFFFFFFFFFFFFF0D
:10739000FFFFFFE02EFB7DFBFBCFC1DFBB3EC0E16B
:1073A000FE3C1FFDEE7B39F9F3CF9EDFBB3EDFDEF7
:1073B000FCDDE7FDEE3BBBF9EBD7BF5FBB5EDFDE7D
:1073C000FDEDF7FDEEBBD3FAEBB73FDFBB4EDFDFE2
:1073D000FFCDF3FDEEDBC7FAEBBB7FC03B6EC0E336
:1073E000FF1DF3FDEECBEFFADBBB7FDFBB66DFF803
:1073F000FFCDF3FDEEEBEFFB5B033F5FBB76DFFE04
:107400007FEDF3FDEEF3EFFB5B79BEDFBB7ADFDEF2
:107410007DEDF7FDEEF3EFFBBAFD9EDFBB7CDFDE1B
:10742000FDCDE7FDEEFBEFFBBAFDC1DFBB7EC0E0AB
:10743000FE1C1FFFFFFFFFFFFFFFFFFFFFFFFFFF20
:10744000FFFFFFFFFFFFFFFFFFFFFFFFFFFFFFFF4C
:10745000FFFFFFFFFFFFFFFFFFFFFFFFFFFFFFFF3C
:10746000FFFFFF1FFFFFFFFFFFFF600000000001A5
:10747000FF400000000000FF8000000000007F834C
:10748000CF00000C303F87FF80000C301F867980D2
:10749000000C000F8C30C7838C30E78C30CFC7CC0A
:1074A00031F38C30DCECEC33B98C30D86C6C3319A4
:1074B0008C30D06C0C33198C30D86C0C33198C3068
:1074C000DC6C0E3B198C30CF7C079F198C30C77C4D
:1074D000038F19400000000000026000000000005F
:1074E000061FFFFFFFFFFFF82020506C616E6E65E6
:1074F0007242756666657242797465733A2000203F
:1075000046726565204D656D6F72793A2000436F54
:107510006D70696C65643A204A756E20203920329E
:107520003031390A00207C20417574686F723A202E
:1075300054696E794D616368696E657333440A00FE
:10754000323031382D30372D333100204C61737497
:1075500020557064617465643A20006275676669DD
:10756000782D312E312E780A004D61726C696E00D3
:1075700020536F6674776172652052657365740A73
:1075800000205761746368646F6720526573657487
:107590000A002042726F776E206F757420526573F7
:1075A00065740A002045787465726E616C205265BE
:1075B0007365740A00506F77657255700A007374B2
:1075C0006172740A006175746F25692E67006572B7
:1075D000726F722077726974696E6720746F2066AB
:1075E000696C650A00456E6473746F70732025635F
:1075F00020256320256320256300205A3A00205966
:107600003A0020583A00656E6473746F7073206896
:1076100069743A2000446F6E6520736176696E6705
:107620002066696C652E0A004D323900496E73750B
:107630006666696369656E7420646174610A0064DA
:107640006F6E650A004578747261706F6C61746961
:107650006E67206D6573682E2E2E005374616E6404
:1076600061726420446576696174696F6E3A2000C6
:107670004D65616E204D6573682048656967687463
:107680003A200023206F662073616D706C65733A39
:1076900020000A4D657368206F6E6C7920706172EE
:1076A0007469616C6C7920706F70756C617465645D
:1076B0002E0A0A0020616E642074616B65206120CF
:1076C0006D6561737572656D656E742E0A006D6D02
:1076D00020746869636B2E0A00427573696E657366
:1076E000732043617264206973200052656D6F7668
:1076F000652026206D656173757265206265640082
:1077000052656D6F7665207368696D00506C6163BA
:1077100065207368696D2026206D656173757265DB
:1077200000506C616365207368696D20756E6465D7
:1077300072206E6F7A7A6C65004D65736820506FA9
:10774000696E74204D656173757265642061743A69
:1077500020000A4D657368206F6E6C79207061722D
:107760007469616C6C7920706F70756C617465649C
:107770002E0A004D65617375726500506C6163651A
:10778000207368696D2026206D65617375726500D0
:107790004D6F76696E6720746F206E65787400494E
:1077A0006E76616C6964206D617020747970652EED
:1077B0000A0A003F28462961646520686569676890
:1077C0007420666F7220426564204C6576656C207B
:1077D000436F7272656374696F6E206E6F74207090
:1077E0006C61757369626C652E0A0A003F43616EB5
:1077F000277420616374697661746520616E64200A
:10780000646561637469766174652061742074686D
:10781000652073616D652074696D652E0A0A0042EA
:107820006F7468205820262059206C6F636174693A
:107830006F6E73206D75737420626520737065635D
:1078400069666965642E0A0A003F496E76616C6953
:107850006420677269642073697A6520284A292048
:107860007370656369666965642028322D39292E35
:107870000A0A003F285029686173652076616C759B
:107880006520696E76616C69642028302D36292E5A
:107890000A0A003F2856296572626F7365206C657D
:1078A00076656C20697320696D706C6175736962AF
:1078B0006C652028302D34292E0A0A003F285229D1
:1078C000657065746974696F6E20636F756E74207E
:1078D000696E76616C69642028312B292E0A0A00B2
:1078E000446F696E6720473239002073616E697496
:1078F0007920636865636B73207061737365642EB0
:107900000A00202073746174653A004B696C6C2026
:1079100070696E206F6E203A00202000592D41784A
:107920006973204D65736820506F696E74732061B0
:10793000743A2000202000582D41786973204D654D
:10794000736820506F696E74732061743A20004D23
:107950004553485F595F444953542020004D4553D7
:10796000485F585F44495354202000475249445FC0
:107970004D41585F504F494E54535F5920200047A6
:107980005249445F4D41585F504F494E54535F58E0
:107990002020004D4553485F4D41585F5920202815
:1079A000282828282834303029202F203229202B3D
:1079B000202834303029202F203229202D2028352E
:1079C00029293C28343030293F28282828343030D1
:1079D00029202F203229202B202834303029202F15
:1079E000203229202D20283529293A2834303029E1
:1079F00029293D004D4553485F4D41585F5820208F
:107A000028282828282834303029202F20322920DF
:107A10002B202834303029202F203229202D2028D7
:107A20003529293C28343530293F28282828343066
:107A30003029202F203229202B20283430302920B3
:107A40002F203229202D20283529293A2834353075
:107A50002929293D004D4553485F4D494E5F592026
:107A60002028282828282834303029202F2032297F
:107A7000202D202834303029202F203229202B207F
:107A800035293E2830293F2828282834303029201D
:107A90002F203229202D202834303029202F203249
:107AA00029202B2035293A28302929293D004D4508
:107AB00053485F4D494E5F58202028282828282801
:107AC00034303029202F203229202D202834303006
:107AD00029202F203229202B2035293E282D3432F1
:107AE000293F2828282834303029202F20322920E7
:107AF0002D202834303029202F203229202B2035EA
:107B0000293A282D34322929293D007A70726F6272
:107B1000655F7A6F66667365743A2000706C616E9B
:107B20006E65722E7A5F666164655F686569676815
:107B300074203A200055424C206F626A65637420BD
:107B4000636F756E743A2000204C6F616465642E1B
:107B5000004D65736820004E6F204D657368204CA2
:107B60006F616465642E004D3234004D3233202540
:107B70007300556E6B6E6F776E20636F6D6D616E07
:107B8000643A202200496E736572742066696C61E4
:107B90006D656E7420616E6420707265737320620F
:107BA0007574746F6E20286F72204D313038290A39
:107BB000002F2F616374696F6E3A726573756D651E
:107BC0000A00486F74656E6420746F6F20636F6C79
:107BD000640A00206D65736820736C6F7473206194
:107BE0007661696C61626C652E0A003F496E766150
:107BF0006C696420736C6F742E0A005344206361B7
:107C00007264206F6B0A006F70656E526F6F742024
:107C10006661696C65640A00766F6C756D652E69C6
:107C20006E6974206661696C65640A00534420695A
:107C30006E6974206661696C0A00062DFFFFFFFF04
:107C40000001020202026265640A002C207379734B
:107C500074656D2073746F70706564212048656170
:107C60007465725F49443A2000426564206865612A
:107C700074696E67206661696C656400486561744B
:107C8000696E67206661696C6564004531204865EE
:107C90006174696E67206661696C656400453220B5
:107CA00048656174696E67206661696C6564004847
:107CB000656174696E67206661696C6564004B4933
:107CC0004C4C45442E20001000AA03F0013A0190CC
:107CD00002220130031001D00302017004F70010EA
:107CE00005ED00B005E5005006DD00F006D7009078
:107CF00007D1003008CC00D008C7007009C30010BD
:107D00000ABE00B00ABB00500BB700F00BB30090E6
:107D10000CB000D00DAA00100FA5005010A00090CC
:107D2000119B00D0129600B014900090168B00703A
:107D3000188500501A8000301C7B00B01E75003082
:107D4000216F00B02369003026640010285F009086
:107D50002A5A00702C5500F02E4F0070314800B0A8
:107D6000324500F03341007036390010373700508B
:107D700038330090392D00D03A2700B03C1C005019
:107D80003D1700F03D1100903E0900D03FE5FF4552
:107D90003220544845524D414C2052554E41574196
:107DA0005900453120544845524D414C2052554EC2
:107DB000415741590042454420544845524D414C99
:107DC0002052554E4157415900546865726D616C9F
:107DD0002052756E61776179004532204572723AA2
:107DE000204D415854454D50004531204572723A5E
:107DF000204D415854454D50004572723A204D4136
:107E00005854454D5020424544004D415854454D2D
:107E10005020747269676765726564004532204559
:107E200072723A204D494E54454D5000453120451F
:107E300072723A204D494E54454D50004572723A87
:107E4000204D494E54454D5020424544004D494E29
:107E500054454D5020747269676765726564004DC2
:107E6000383420582059205A204500000021002491
:107E70000027002A002D003000330001010000041B
:107E80000107010A0100002200250028002B002E16
:107E9000003100340002010000050108010B01005F
:107EA0000020002300260029002C002F00320000B3
:107EB0000100000301060109010505050507050884
:107EC000080808020202020A0A080804040404015D
:107ED000010101010101010303030303030303047F
:107EE0000707070C0C0C0C0C0C0C0C02020202060F
:107EF000060606060606060B0B0B0B0B0B0B0B01FF
:107F000002102020080810204010204080020102AA
:107F10000108040201010204081020408080402072
:107F200010080402018004020180402010080402AD
:107F3000010804020101020408102040800102042B
:107F4000081020408000000A0B02090C0D0E0807E3
:107F50000304010000000000000000000000000019
:107F60000000000000000000000000000000000011
:107F700000121110000000000000000000000000CE
:107F800000000000000000000000004368616E6710
:107F9000652066696C616D656E7400556E6C6F610D
:107FA000642066696C616D656E74004C6F6164205D
:107FB00066696C616D656E740050726568656174A8
:107FC00020414253005072656865617420504C41F5
:107FD000004368616E67652066696C616D656E74EB
:107FE0000053746F72652073657474696E677300F3
:107FF0004265640042656400426564004E6F7A7AAF
:108000006C65004E6F7A7A6C65004E6F7A7A6C659B
:108010000046616E2073706565640046616E207372
:10802000706565640046616E207370656564005418
:10803000656D706572617475726500565472617613
:10804000206D696E005654726176206D696E00561F
:1080500054726176206D696E00566D696E00566DC2
:10806000696E00566D696E00566D61782045005648
:108070006D6178204500566D6178204500566D6130
:1080800078205A00566D6178205A00566D6178202C
:108090005A00566D6178205900566D61782059005C
:1080A000566D6178205900566D6178205800566DE4
:1080B0006178205800566D61782058004D6F7469C2
:1080C0006F6E00416D6178204500416D61782045FB
:1080D00000416D6178204500416D6178205A004172
:1080E0006D6178205A00416D6178205A00416D61C0
:1080F00078205900416D6178205900416D617820E8
:108100005900416D6178205800416D617820580018
:10811000416D6178205800412D74726176656C0064
:10812000412D74726176656C00412D7265747261C7
:10813000637400412D7265747261637400416363FE
:10814000656C00416363656C004D6F74696F6E0010
:10815000526573656E643A20002042002050006F23
:108160006B000E02860111241FBECFEFD1E2DEBFED
:10817000CDBF00E00CBF14E0A0E0B2E0ECE9F8EA0B
:1081800003E00BBF02C007900D92A438B107D9F7E6
:108190002AE1A4E8B4E001C01D92AF3FB207E1F7C5
:1081A00010E4C2EBD0E400E006C021970109802F63
:1081B000FE010F9443CFC13BD10780E00807A9F728
:1081C0000F9446BB0D943CD40C9400002F923F9228
:1081D0004F925F926F927F928F929F92AF92BF92D7
:1081E000CF92DF92EF92FF920F931F93CF93DF9383
:1081F000CDB7DEB7C354D1090FB6F894DEBF0FBEBA
:10820000CDBF21E0209326188091F81A8D3409F40F
:10821000B4C4843511F40C948055873411F00C9457
:10822000AC558091F61A9091F71A8B31910509F4AB
:108230000CC2A4F48430910534F482309105A4F585
:1082400097FF2BC096C48430910509F4BFC14A97AB
:1082500009F08FC40E94DC990C94AE558A329105C6
:1082600009F405C354F48D31910509F426C20CF4C8
:108270001FC24E9709F425C27CC48B35910509F4C1
:10828000F6C38C35910509F4F6C38A35910509F0DA
:1082900070C4109296040C94AE55809180028111A6
:1082A0000C94B3550C94AE5520918002222311F406
:1082B0000C94AE5511E0029709F010E00E94ED78A1
:1082C00019821A821B821C821D821E821F821886BE
:1082D00082E50E945998882309F428C10E94D99701
:1082E0004B015C0120E030E0A9010F9446C88823CF
:1082F00009F432C18091BC189091BD18A091BE18AC
:10830000B091BF1888A799A7AAA7BBA78091C0184A
:108310009091C118A091C218B091C3188CA79DA7C5
:10832000AEA7BFA78091D0189091D118A091D21874
:10833000B091D31888AB99ABAAABBBAB8091D418E2
:108340009091D518A091D618B091D7188CAB9DAB51
:10835000AEABBFAB28A939A94AA95BA968A579A585
:108360008AA59BA50F9446C881110DC02CA93DA9D3
:108370004EA95FA96CA57DA58EA59FA50F9446C8A3
:10838000882309F4E9C020E030E0A901C501B40167
:108390000F9446C8881F8827881F181729F080E087
:1083A00090E0A0E8BFEB04C080E090E0A0E8BFE36D
:1083B0008CAF9DAFAEAFBFAF28A539A54AA55BA5D1
:1083C00068A979A98AA99BA90F944BCF68AF79AF07
:1083D0008AAF9BAF2CA53DA54EA55FA56CA97DA935
:1083E0008EA99FA90F944BCF6B017C0128AD39ADAD
:1083F0004AAD5BADCA01B9010F94ACC82B013C0179
:10840000A7019601C701B6010F94ACC89B01AC014E
:10841000C301B2010F944CCF0F944AD22B013C01FF
:1084200020E030E040E05FE30F94ACC824966CAFEE
:108430007DAF8EAF9FAF2497A5019401C501B40114
:108440000F94ACC84B015C0124962CAD3DAD4EADF4
:108450005FAD2497CA01B9010F94ACC89B01AC0170
:10846000C501B4010F944BCF0F944AD22CAD3DAD52
:108470004EAD5FAD0F94ACC84B015C01C701B601B6
:108480009058A30192010F9446D0A50194010F9436
:10849000ACC86B017C0128A939A94AA95BA968A5C8
:1084A00079A58AA59BA50F944CCF20E030E040E051
:1084B0005FE30F94ACC89B01AC01C701B6010F94F8
:1084C0004CCF28A539A54AA55BA50F944BCF69834E
:1084D0007A838B839C832CA93DA94EA95FA96CA5A7
:1084E0007DA58EA59FA50F944CCF20E030E040E005
:1084F0005FE30F94ACC86B017C01A301920168ADEE
:1085000079AD8AAD9BAD0F9446D0A50194010F942F
:10851000ACC89B01AC01C701B6010F944CCF2CA590
:108520003DA54EA55FA50F944BCF12C089E40E94D4
:108530005998882331F00E94D99769837A838B8375
:108540009C838AE40E945998882331F00E94D9972D
:108550006D837E838F83988720E030E0A901698155
:108560007A818B819C810F9446C881110EC020E0D6
:1085700030E0A9016D817E818F8198850F9446C876
:10858000811103C0E5EDF7E50DC0412FBE016F5F1E
:108590007F4F80ED98E10E94A6730C94AE550F9426
:1085A0001E14F80184918F010F5F1F4F8111F7CFC7
:1085B000EBE0F7E084918F010F5F1F4F882311F4E8
:1085C0000C94AE550F941E14F801F4CF80E50E9470
:1085D0005998882329F00F94FD136B017C0103C087
:1085E000C12CD12C760183E50E945998882361F033
:1085F0000E94D99720E030E04AE754E40F94ACC8D9
:108600000F94BFD06B017C010E94ECB680914F1893
:10861000811105C060E081E297E00E9466C40F947A
:10862000257DC60ED71EE81EF91E0F94257DDC01A0
:10863000CB018C199D09AE09BF09B7FD02C00C948E
:10864000AE5580E00E94906FF0CF41E061E081E0A4
:108650000F949F1481110C94AE5580E090E0A6E138
:10866000B3E489839A83AB83BC8380E090E0A0E28B
:10867000B1E48D839E83AF83B88780E090E0A0EA69
:10868000B1E489879A87AB87BC8780E50E945998B7
:10869000882319F00E94A59701C060E068A3BE017D
:1086A0006F5F7F4FCE0180960E9412B80C94AE553A
:1086B00080E00E94577A0C94AE550F9460440C945D
:1086C000AE55C090BC18D090BD18E090BE18F09088
:1086D000BF1888E50E945998811109C020E030E058
:1086E00040E450E4C701B6010F944BCF02C00E9492
:1086F000D99768A379A38AA39BA3C090C018D090F0
:10870000C118E090C218F090C31889E50E945998EA
:10871000811109C020E030E048EF51E4C701B60103
:108720000F944CCF02C00E94D9979B01AC01698382
:108730007A838B839C8368A179A18AA19BA10F94E2
:108740004682882311F40C94AE5580E00E94117A81
:108750000F94A30D85E40E945998882321F00E946C
:10876000C997182F04C085E40E94109811E086E58F
:108770000E945998882321F00E94A597262F01C0B6
:1087800021E001E0412FBE016F5F7F4FCE01809657
:108790000E94857D6B017C019B01AC010F9499D2F5
:1087A00081115FC088A099A0AAA0BBA020E030E002
:1087B000A901C501B4010F9446C887FF05C027E190
:1087C00037EB41E558EB04C027E137EB41E558E3CF
:1087D000C501B4010F944CCFAB01BC0184E397E019
:1087E0000F94592389809A80AB80BC8020E030E0D0
:1087F000A901C501B4010F9446C887FF05C027E150
:1088000037EB41E558EB04C027E137EB41E558E38E
:10881000C501B4010F944CCFAB01BC018FE297E0CE
:108820000F94592320E030E0A901C701B6010F944D
:1088300046C887FF05C027E137EB41E558EB04C088
:1088400027E137EB41E558E3C701B6010F944CCF60
:10885000AB01BC018AE297E00F9459238AE00F94A0
:108860001E140F948A0D0F9476360C94AE55809199
:108870008002882311F40C94AE5589E40E94599823
:10888000082F882321F00E94A597E62E01C0E12C35
:108890008AE40E945998182F882321F00E94A597F6
:1088A000F62E01C0F12C002319F09EE09E1528F051
:1088B000112389F0AEE0AF1570F4ECE3F7E084919A
:1088C0008F010F5F1F4F882311F40C94AE550F9446
:1088D0001E14F801F4CF0E948B98002391F1EE2D25
:1088E000F0E0BEE0BE1570F0EE0FFF1FEE0FFF1FB1
:1088F000E855F84C4591559165917491342F252F89
:10890000CB0114C0BF01FF0F880B990B0F944DC80A
:108910002EE63BED4EED51E40F94ACC820E030E084
:1089200040EA50E40F944CCF362F272F432F522F7D
:10893000BC014093D0185093D1186093D218709313
:10894000D318112391F1EF2DF0E02EE02F1570F0E8
:10895000EE0FFF1FEE0FFF1FE859F84C45915591A0
:1089600065917491342F252FCB0114C0BF01FF0FE7
:10897000880B990B0F944DC82EE63BED4EED51E45C
:108980000F94ACC820E030E040EA50E40F944CCFA4
:10899000362F272F432F522FBC014093D4185093CA
:1089A000D5186093D6187093D71880E50E9459980F
:1089B0008823E9F00E94C9978823A9F10023D9F000
:1089C00020E030E040E450E46091D0187091D1187C
:1089D0008091D2189091D3180F944CCF6093D018F7
:1089E0007093D1188093D2189093D31804C080E567
:1089F0000E941098E1CF1123B1F020E030E048EF61
:108A000051E46091D4187091D5188091D618909146
:108A1000D7180F944BCF6093D4187093D5188093C8
:108A2000D6189093D71886E40E9459988823D9F0D5
:108A30000E94D9976B017C0120E030E0A9010F94DE
:108A4000ACD1181684F420E030E040E752E4C701CE
:108A5000B6010F9446D06093090270930A02809386
:108A60000B0290930C020E943A640C94AE55209332
:108A700096040C94AE55E1E62E2EE3E03E2EF4E88B
:108A8000EF2EF4E0FF2E8CEB98E199A788A7ABE9D5
:108A9000CA2EA5E0DA2E00E010E0D1018D911D0173
:108AA0000E945998882309F44BC00E94D9972B0142
:108AB0003C01133049F0F60120813181428153811C
:108AC0000F944BCF2B013C01A8A5B9A52D913D9149
:108AD0004D915C91C301B2010F944BCF4B015C01EE
:108AE0002DEB37E346E855EB0F94ACD187FD0AC078
:108AF0002DEB37E346E855E3C501B4010F9446C8B2
:108B00001816F4F4133051F44092C8185092C91852
:108B10006092CA187092CB1801E012C0A5019401AE
:108B2000F70160817181828193810F944CCFD701CD
:108B30006D937D938D939C931397812F0F94950F35
:108B40001F5FB4E0EB0EF11CE8A5F9A53496F9A778
:108B5000E8A7F4E0CF0ED11C143009F09ECF00231B
:108B600021F088EC98E10F9476980F9476360C9467
:108B7000AE550F94E89C0C94AE558091F61A9091E6
:108B8000F71A8737910511F40C94644F0CF003C168
:108B90008B34910509F4F4C50CF081C08A3191053C
:108BA00009F444C3F4F58431910509F43AC284F41C
:108BB0008131910509F4B0C22CF4029708F434C253
:108BC0000C947D55429711F40C94EA4D0C947D550C
:108BD0008731910509F4EAC274F48531910509F4ED
:108BE000E1C2469711F00C947D5510922C1310920F
:108BF0002D130C94AE558831910509F4EDC24997B7
:108C000011F00C947D5510922C130F94F7A087E966
:108C100097E090930D1880930C180F94EE100C941D
:108C2000AE558032910509F438C40CF58D319105AB
:108C300011F40C94AE5594F48B31910509F404C3EE
:108C40004C9711F00C947D5540E060E08091F41A4F
:108C50009091F51A0F9433560C94AE558E319105C0
:108C600009F489C34F9709F468C40C947D55803387
:108C7000910509F44DC54CF48132910509F44CC4B9
:108C80008A9709F410C50C947D558133910509F438
:108C900043C58934910509F466C50C947D558A361F
:108CA000910509F4AEC694F58335910509F48EC794
:108CB0009CF48D34910509F46BC50CF465C58135C0
:108CC000910509F46AC78235910511F00C947D5520
:108CD000109295040C94AE558C35910511F40C94BA
:108CE000404E54F48435910509F474C785359105D7
:108CF00009F4ADC70C947D558836910509F44CC52F
:108D00008936910509F421C60C947D55803791056B
:108D100011F40C94AE55D4F48D36910509F457C670
:108D20005CF48B36910509F493C68C36910511F4E9
:108D30000C94AE550C947D558E36910509F472C590
:108D40008F36910509F481C50C947D5583379105C3
:108D500009F464C16CF48137910509F4C9C58237FF
:108D6000910511F00C947D550F9440370C94AE553D
:108D70008537910511F40C940F4F8637910511F04A
:108D80000C947D550091F41A1091F51A83E0D12CC2
:108D900040E00C94244F8E3221E0920711F40C94A1
:108DA00014530CF097C08C3C910511F40C948D5029
:108DB0000CF041C08139910511F40C94724F94F478
:108DC0008937910511F40C946D4F14F40C94674F8E
:108DD0008D37910509F454C68C38910509F4FBC50B
:108DE0000C947D55883C910511F40C94EA4F6CF479
:108DF0008B39910509F4C4C58E3B910511F00C9493
:108E00007D550F94DE380C94AE55893C910511F4D4
:108E10000C9456508B3C910511F00C947D5561E6F5
:108E2000E62E63E0F62E0EEA1AE17EEBC72E7AE11B
:108E3000D72E0C947E508D3D910511F40C949D51CC
:108E40003CF5833D910511F40C948A51ACF48D3CB2
:108E5000910511F40C9402518E3C910511F00C9483
:108E60007D5541E6C42E43E0D42E57E5E52E56E16C
:108E7000F52E10E00C9475518A3D910511F40C9477
:108E80008D518C3D910511F40C9490510C947D55AD
:108E90008232A1E09A0711F40C94E05264F4823E0D
:108EA000910511F40C940C528831914011F40C94FA
:108EB00035520C947D558C32F1E09F0711F40C94DF
:108EC000EB528D32914011F00C947D550F940C347F
:108ED0000C94AE55853F31E0930711F40C9438544F
:108EE0000CF052C08239B1E09B0711F40C942F545E
:108EF00034F58336F1E09F0711F40C94E8536CF4D9
:108F00008F3231E0930711F40C9468538033914011
:108F100011F40C946B530C947D558039B1E09B0790
:108F200011F40C942C548139914011F00C947D551E
:108F300081E00F94F60E0F9476360C94AE55853A78
:108F4000F1E09F0711F40C9435547CF48A3931E038
:108F5000930711F40C94AE55843A914011F00C949F
:108F60007D550F942E720C94AE558C3AB1E09B0750
:108F700011F40C948751843F914011F00C947D556D
:108F80000E94E5860C94AE558B35F2E09F0711F4F4
:108F90000C9477541CF5883F31E0930711F40C943E
:108FA0004A546CF4863FB1E09B0711F40C943B5497
:108FB000873F914011F40C943E540C947D558C30B5
:108FC000F2E09F0711F40C946E548835924011F032
:108FD0000C947D550F94026E0C94AE558B3833E093
:108FE000930711F40C94AE556CF48D35B2E09B07E9
:108FF00011F40C9400558335934011F40C940355EF
:109000000C947D55803AF3E09F0709F489C2873EAE
:10901000934011F40C9468550C947D55E5E4F9E007
:10902000A3C6E6E8F7E08DC0A090F41AB090F51A58
:1090300080E50E945998882359F00F94FD136B0125
:109040007C0111E0672B682B692B31F410E004C020
:1090500010E0C12CD12C760183E50E945998882319
:1090600011F40C94B8550E94D99720E030E04AE7FB
:1090700054E40F94ACC80F94BFD06B017C01111164
:109080000BC0672B682B692B39F4A114B10421F0B4
:10909000D5018C91811102C010E001C011E00E9445
:1090A000ECB6112329F061E0C5010E94A2C405C0FD
:1090B00060E08BE597E00E9466C483E08093261809
:1090C00081E080932518C114D104E104F104B1F0CA
:1090D0000F94257DC60ED71EE81EF91E0F94257D20
:1090E000DC01CB018C199D09AE09BF09B7FF0EC089
:1090F0008091251881110C94BD5508C080912518C8
:10910000882321F080E00E94906FF8CF0F94FD2B10
:10911000109225180C94AE5560E08EE697E00E9400
:1091200066C45F9880910B018072809309018A98D0
:1091300080910801817080930601129847980C94E1
:10914000AE5584918F010F5F1F4F882321F00F943C
:109150001E14F801F6CF1092D11584E893E10E9415
:109160006E5960E873E1CE0101960F94E05140E042
:1091700050E0BE016F5F7F4F80E090E00F9490530E
:10918000CE0101960E94AC63E7E7F7E084918F017E
:109190000F5F1F4F882311F40C94AE550F941E14CB
:1091A000F801F4CF0F943A950C94AE55E091F41A6F
:1091B000F091F51A8081882329F0803209F4108219
:1091C0003196F8CF40E061E08091F41A9091F51A61
:1091D0000F9433560C94AE5580E090E0A0EAB1E4D1
:1091E00089839A83AB83BC8318A219A21AA21BA2FB
:1091F0001CA21DA21EA21FA280913112882359F029
:1092000020E0AE014F5F5F4FBE01605E7F4FCE0139
:1092100084960F94349B80912D13882319F081E05C
:1092200080932C130F94D3A00C94AE5580912D13E2
:10923000882311F40C94AE5583E50E94599881114E
:109240000C94C2550C94AE5583E40E941098882368
:1092500009F468C0E6EAF7E084918F010F5F1F4FC1
:10926000882321F00F941E14F801F6CF80911F156A
:10927000811103C0ECE9F7E02AC0BE016F5F7F4FA8
:109280008CE195E10E943A598E010F5F1F4FF80162
:1092900081918F01882319F00F941E14F8CFBE011D
:1092A0006F5F7F4F80E090E00F94425580913D13B7
:1092B000882399F180E20F941E140DE313E1D80185
:1092C0008D918D01882349F10F941E14F8CF84915C
:1092D0008F010F5F1F4F882301F10F941E14F801B7
:1092E000F6CF6AE3C62E68E0D62EE12CF12C20E002
:1092F0008091491890E00E2C02C0959587950A94AC
:10930000E2F780FDD2C23FEFE31AF30A82E0C80E13
:10931000D11C95E0E916F10459F78AE00F941E1468
:109320000C94AE5583E50E945998882301F10E9460
:10933000B597182F8D3308F01CE31093B9040F94E0
:10934000257D6B017C01212F30E0A8EEB3E00F9466
:1093500000CFC60ED71EE81EF91EC092B504D092EB
:10936000B604E092B704F092B8040C94AE550F9492
:109370000B510C94AE5580912D13882311F40C944D
:10938000AE558CE195E10E94FE588CE195E10E947A
:10939000315910922B1310922A1380912D13882388
:1093A00011F40C94AE550091F41A1091F51A0F9423
:1093B000F451B801CE0180960F9477558C01892B1A
:1093C00011F40C94AE5568A179A16115710511F0E5
:1093D0006C5F7F4F19821C8222E0A801CE010196AA
:1093E0000E94BB62811102C0F12C14C0CE01019613
:1093F0000F944E518823C1F361E0CE0101960E9483
:10940000E258009789F325EEFC0120831C820E941C
:10941000F292F82ECE0101960F940D14F11003C0B4
:10942000E3ECF7E022C0E5EBF7E084917F012FEF5A
:10943000E21AF20A882321F00F941E14F701F5CFE7
:10944000D8018D918D01882319F00F941E14F8CF47
:109450008AE00F941E141092CD151092CE15109222
:10946000CF151092D0150C94AE5584917F01BFEFAB
:10947000EB1AFB0A882321F00F941E14F701F5CF95
:10948000F80181918F01882319F00F941E14F8CFF1
:109490008EE20F941E140C94AE5580912C13811102
:1094A0000E94ECB680912D13882311F40C94AE55D4
:1094B00080E50E945998882319F00E94C99703C03B
:1094C00080E50E941098182F482F61E08091F41ACF
:1094D0009091F51A0F94335683E50E94599888238A
:1094E00081F00E94A597AB01BC014093CD1550932C
:1094F000CE156093CF157093D0158CE195E10E9445
:10950000F85780912D13882319F081E080932C1354
:1095100011110C94AE5586CE0E94F6840C94AE5573
:109520008091F41A9091F51A21E020932B1340E0DA
:1095300060E00F9433560C94AE550F9484A07B01D9
:109540008C0120E831E541E050E00F94ACCEC90138
:109550006DE671E00F941BCF4B015C01C801B701B0
:1095600020E13EE040E050E00F94ACCECA01B901EA
:1095700028E130E040E050E00F94ACCE762E672E2C
:10958000C62ED72E7CE3272E312C412C512CC8011E
:10959000B701A20191010F94ACCEF62EE72ECA01BD
:1095A000B901A20191010F94ACCECB018E010F5FE6
:1095B0001F4F8114910499F0EF92FF927F936F9364
:1095C0006F927F92BF92AF929F928F9283E098E0CA
:1095D0009F938F931F930F930F94DEC713C0A11413
:1095E000B104B1F0EF92FF927F936F936F927F92ED
:1095F000BF92AF9283EF97E09F938F931F930F9348
:109600000F94DEC70FB6F894DEBF0FBECDBF30C0DB
:10961000CD2879F0EF92FF927F936F936F927F92B4
:1096200087EE97E09F938F931F930F930F94DEC75E
:10963000E9CF892B69F0EF92FF927F936F938FEDC3
:1096400097E09F938F931F930F930F94DEC7DACF0A
:10965000EF92FF928BED97E09F938F931F930F9361
:109660000F94DEC70F900F900F900F900F900F90F8
:1096700060E0C8010E94A2C4E4E0F8E584917F01A3
:109680002FEFE21AF20A882321F00F941E14F7013B
:10969000F5CFB80187E198E00F948E238AE00F940C
:1096A0001E140C94AE5583E50E945998882311F43A
:1096B0000C94AE550E94B597E82E80E50E9459980B
:1096C000882339F00E94B597182F87FF03C00C94A8
:1096D000AE551DE089E40E945998882351F00E94FC
:1096E000C99781110C94BD56E2E7FAE08CEA9AE042
:1096F0000AC089E40E941098F4CF31968E179F0714
:1097000011F40C94BD5624911213F7CF0C941756F4
:109710000E948A7F0C94AE559091A80481E089271D
:109720008093A804EFE2F8E084918F010F5F1F4F50
:10973000882321F00F941E14F801F6CF8091A8041D
:10974000882319F0E4E2F8E002C0E9E2F8E084914D
:109750008F010F5F1F4F882311F40C94AE550F94A7
:109760001E14F801F4CF80912C1381110C94AE5586
:1097700080E50E94109881110C94D3550C94AE553D
:109780000F94D3A00C94AE550F94F7A00C94AE5543
:109790000F940CA10C94AE5588E690E00F944818F5
:1097A00081110C94AE558091491883FF02C00C942E
:1097B000AE5583E50E945998882381F10E94D9977C
:1097C0000F94B8D06B017C0160911210C6010E9409
:1097D000749880910802823099F48091121081115E
:1097E0000FC0C114D10439F080919004909191047C
:1097F0008C0D9D1D02C080E090E061E00E94749895
:109800000E94D99720E030E04AEA52E40F9446C81B
:10981000181624F00F940CA10F94FD2B0F94E7233E
:109820000C94AE558EE40E945998882311F40C9440
:10983000AE550E94A59760932D1270932E128093BF
:109840002F12909330120C94AE5583E50E9410981D
:10985000882359F083E50E945998882319F00E94C3
:10986000B59701C080E080934918E4E0F8E5849161
:109870008F010F5F1F4F811103C0E8E4F8E004C0BF
:109880000F941E14F801F3CF84918F010F5F1F4FC7
:10989000882321F00F941E14F801F6CF8091491807
:1098A00081111FCDE4E4F8E018C0BB24B394B20EDC
:1098B000222319F08CE20F941E14F60185919491E5
:1098C000FC0184918F010F5F1F4F882321F00F94BB
:1098D0001E14F801F6CF2B2D16CD84918F010F5F4A
:1098E0001F4F882309F419CD0F941E14F801F5CFEA
:1098F00083E50E945998811103C0E4E0F8E50DC0AA
:109900000E94B5978D3320F480930D020C94AE55D0
:109910008CE380930D020C94AE5584918F010F5F00
:109920001F4F882321F00F941E14F801F6CF4091A9
:109930000D0250E060E070E08FE498E00F943C236B
:109940008AE00F941E140C94AE5589E690E00F94B3
:109950004818811111C0E6E5F8E084918F010F5F8E
:109960001F4F882321F00F941E14F801F6CF0F9497
:109970007E438AE00F941E14109226180C94D95638
:1099800083E50E945998882311F40C94AE550E94E7
:10999000B597182F8D3308F01CE31093BE040F9475
:1099A000257D6B017C01212F30E0A8EEB3E00F9400
:1099B00000CFC60ED71EE81EF91EC092BA04D09280
:1099C000BB04E092BC04F092BD040C94AE550F941D
:1099D000A63A0C94AE558091491883FF02C00C94AE
:1099E000AE5583E50E945998882311F40C94AE5526
:1099F0000E94D9970F94B8D0CB010E9466980C941E
:109A0000AE5580E50E945998882341F00E94B59791
:109A1000182F823010F00C94AE5501C010E083E591
:109A20000E945998882319F00E94A59702C06FEFF1
:109A300070E0E12FF0E06F3F710510F06FEF70E024
:109A4000EE0FFF1FE551F84E718360830C94AE5505
:109A500080E50E945998882341F00E94A5976230C2
:109A6000710510F00C94AE5502C060E070E0660F16
:109A7000771FFB01E551F84E118210820C94AE5510
:109A80008CE40E941098882381F00E94D9976B0182
:109A90007C0120E030E0A9010F94ACD187FF0BC01E
:109AA000F7FAF094F7F8F09406C0C12CD12C30E806
:109AB000E32E30E4F32EF7FAF094F7F8F094CCA20A
:109AC000DDA2EEA2FFA280E090E0A6E1B3E48983EC
:109AD0009A83AB83BC8380E090E0A0E2B1E48D8305
:109AE0009E83AF83B88780E090E0A0EAB1E48987E5
:109AF0009A87AB87BC8788E50E945998882379F0BC
:109B000088E50E945998882319F00E94D99703C0CC
:109B100060E070E0CB0169837A838B839C8389E565
:109B20000E945998882379F089E50E9459988823E2
:109B300019F00E94D99703C060E070E0CB016D83FB
:109B40007E838F8398878AE50E945998882379F0CD
:109B50008AE50E945998882319F00E94D99703C07A
:109B600060E070E0CB0169877A878B879C8718A2B9
:109B700019A21AA21BA28091311281110C94AE5528
:109B800020E0AE01405E5F4FBE016F5F7F4FCE01B0
:109B900084960E94635F0C94AE550F9421A10E949D
:109BA00013B71092EC171092EB171092EE17109259
:109BB000ED1768EE73E080E090E00E944FC360E034
:109BC00089E598E00E9466C40C94AE5520939504F4
:109BD0000C94AE5583E50E9459988823A1F00E9409
:109BE000D99720E030E04AE754E40F94ACC80F94D2
:109BF000BFD060930E0270930F0280931002909377
:109C000011020C94AE5588E50E94109881110C94B5
:109C1000DE5589E50E94109881110C94DE558AE585
:109C20000E94109881110C94DE5585E40E941098D2
:109C300081110C94DE550E9413B78091C9058823C9
:109C400009F48CC710924A181092C90587C783E59A
:109C50000E941098882309F481C70E94D99720E0B8
:109C600030E04AE754E40F94ACC80F94BFD060933F
:109C7000B1047093B2048093B3049093B4046EC79C
:109C800091E6C92E93E0D92E24EAE22E28E1F22EA5
:109C900010E0D6018D916D010E941098882309F47F
:109CA00059C0133009F04FC00E94D9974B015C0195
:109CB00020E030E040EA51E40F9446C887FF3AC004
:109CC000A50194016091B0187091B1188091B218FB
:109CD0009091B3180F9446D02B013C019B01AC012D
:109CE0006091BA1A7091BB1A8091BC1A9091BD1AFA
:109CF0000F94ACC86093BA1A7093BB1A8093BC1AC5
:109D00009093BD1A6091940A7091950A8091960A79
:109D10009091970A0F944BC8A30192010F94ACC87D
:109D20000F94BFD06093940A7093950A8093960A1B
:109D30009093970A8092B0189092B118A092B2189E
:109D4000B092B31807C00E94D997F701608371835E
:109D5000828393831F5FF4E0EF0EF11C143009F04F
:109D600098CF0F947225FAC684918F010F5F1F4F11
:109D7000882321F00F941E14F801F6CF60E085E3EC
:109D800099E00F943F3661E08EE299E00F943F3600
:109D900061E083E299E00F943F3661E083E199E06E
:109DA0000F943F3660E08AE099E00F943F3661E01F
:109DB00080E099E00F943F3661E086EF98E00F94E1
:109DC0003F3661E08EEE98E00F943F3661E080EE22
:109DD00098E00F943F3661E082ED98E00F943F36B3
:109DE00060E083EC98E00F943F3661E085EB98E00B
:109DF0000F943F3660E08FE998E00F943F3661E0C2
:109E00008EE898E00F943F3661E089E798E00F9480
:109E10003F3661E086E698E00F943F369FC680911A
:109E2000F41A9091F51ADC012C91222321F060E0C4
:109E30000E94A2C493C60F94FD2B90C6F801908196
:109E4000292F2B7F213419F08150C1F716C02181B1
:109E50002133D1F7913421F0953421F441E002C04F
:109E6000DD24D39498012E5F3F4F89012F5F3F4F30
:109E7000D8019C919032C9F3E7CF442369F0E4E024
:109E8000F8E584917F01BFEFEB1AFB0A882321F0EC
:109E90000F941E14F701F5CFDD2069F0EFE0FAE032
:109EA00084917F012FEFE21AF20A882321F00F94A8
:109EB0001E14F701F5CFD8018D918D01882309F487
:109EC0002CCA0F941E14F7CF0F94A75847C681E0F1
:109ED000809352168093511641C6109252161092DA
:109EE00051163CC683E50E945998882319F00E94B8
:109EF000A59702C060E070E08B01112702301105C8
:109F0000D4F0E5EDF7E584918F010F5F1F4F8111CC
:109F100003C0E3E1FAE004C00F941E14F801F3CF8C
:109F200084918F010F5F1F4F882309F417C60F9488
:109F30001E14F801F5CF88E40E9459988823A9F0EF
:109F40000E94A5976A3A71053CF06035B1E07B0745
:109F50002CF06FE471E002C06AEA70E0F801EE0FE5
:109F6000FF1FE256F54E7183608386E40E94599884
:109F70008823A9F00E94A597F801EE0FFF1FEE5568
:109F8000F54E718360836F3F710519F014F06FEF28
:109F900070E077FF02C060E070E07183608382E46C
:109FA0000E945998882309F4D9C50E94A597653065
:109FB000710534F0683871052CF067E870E002C074
:109FC00065E070E0000F111FF801E656F54E718351
:109FD0006083C4C588EC90E00F9448188111BEC519
:109FE00084E40E941098882309F45DC00E94D997E8
:109FF0006B017C0111E020E030E0A9010F9446C81C
:10A00000811101C010E01093451620E030E0A90155
:10A01000C701B6010F9446C8882309F444C00E94C2
:10A02000D997E091121024E0E29FF0011124E35C43
:10A03000F94E608371838283938320E030E0A9012D
:10A0400060913D1670913E1680913F16909140169A
:10A050000F9446C881110CC080E090E0A0EEBFE3F1
:10A0600080933D1690933E16A0933F16B0934016F2
:10A0700020E030E0A9016091411670914216809174
:10A080004316909144160F9446C881110CC080E08D
:10A0900090E0A0EEBFE38093411690934216A09308
:10A0A0004316B09344160E943BA558C5E1E6EE2E38
:10A0B000E3E0FE2E0EEB1AE1FEECCF2EFAE1DF2EEE
:10A0C000D7018D917D010E941098882349F00E944C
:10A0D000D9970F94BFD0F8016083718382839383F3
:10A0E0000C5F1F4FC016D10659F70F94172436C5C1
:10A0F0000C5F1F4FC016D10609F430C5D7018D91F2
:10A100007D010E941098882399F30E94D997F80145
:10A110006083718382839383EBCF83E50E94599898
:10A120008823A1F00E94D9976093D21A7093D31A12
:10A130008093D41A9093D51A6093CE1A7093CF1A45
:10A140008093D01A9093D11A10E001C011E080E5FD
:10A150000E945998882359F00E94D9976093D21A87
:10A160007093D31A8093D41A9093D51A10E082E595
:10A170000E945998882359F00E94D997609321181A
:10A1800070932218809323189093241810E084E58C
:10A190000E945998882359F00E94D9976093CE1A4B
:10A1A0007093CF1A8093D01A9093D11AD7C41123E9
:10A1B00009F4D4C44091D21A5091D31A6091D41AA0
:10A1C0007091D51A8BE39AE00F945923409121188E
:10A1D00050912218609123187091241888E39AE016
:10A1E0000F9459234091CE1A5091CF1A6091D01AF2
:10A1F0007091D11A85E39AE00F9459238AE00F9465
:10A200001E14ACC481E50E941098882351F00F946D
:10A21000FD136093520570935305809354059093FA
:10A22000550583E50E941098882351F00E94D99724
:10A230006093AA1A7093AB1A8093AC1A9093AD1ADC
:10A2400084E50E941098882351F00E94D99760936A
:10A25000A61A7093A71A8093A81A9093A91A8AE451
:10A260000E941098882309F479C40E94D9976B0141
:10A270007C012AE037ED43E25CE30F94ACD187FD2B
:10A280000AC02AE939E949E95EE3C701B6010F943A
:10A2900046C818161CF4E5EDF7E50CC0C092291667
:10A2A000D0922A16E0922B16F0922C1657C40F94D7
:10A2B0001E14F80184918F010F5F1F4F8111F7CF9A
:10A2C000EBE4FAE084918F010F5F1F4F882309F4BC
:10A2D00045C40F941E14F801F5CF1F5FF4E0EF0E94
:10A2E000F11C133011F40C94B545D6018D916D011C
:10A2F0000E941098882389F30E94D997F701608300
:10A30000718382839383812F0F94950FE6CF0F94EF
:10A31000437024C40F94613521C40F94C6341EC405
:10A3200083E50E945998882309F418C40E94A597D0
:10A3300070933B0260933A0211C48DED90E00F944C
:10A34000481881110BC483E50E945998811103C0FC
:10A35000E4E0F8E53BC00091121010E00E94A597E0
:10A36000000F111FF801EA5CFD4F7183608380913B
:10A37000121090E08C01000F111F000F111F9801A7
:10A38000225D3D4F7901880F991FFC01EA5CFD4F6A
:10A3900060817181072E000C880B990B0F944DC8BA
:10A3A0002AE037ED43E25CE30F94ACC8F801EF53C9
:10A3B000FA4F20813181428153810F94ACC8D7017B
:10A3C0006D937D938D939C931397C8C384918F0154
:10A3D0000F5F1F4F882321F00F941E14F801F6CF52
:10A3E00085E40F941E1480911210805D0F941E144A
:10A3F000E0911210F0E0EE0FFF1FEA5CFD4F60816C
:10A4000071818AE69AE00F94762385E20F941E14F8
:10A410008AE00F941E14A2C380E50E94109888233E
:10A4200009F49CC30E94A5976B017C0183E50E94FF
:10A430005998882321F00E94A5978B0102C00FEF45
:10A440001FEFC8010196039708F088C3D7FC86C3A5
:10A450008C2DE2E7FAE09491891709F4E8C331966C
:10A46000BAE0EC3AFB07B9F7E5C380E50E94109823
:10A47000882309F473C30E94A5976B017C018B01AB
:10A48000672B19F0E5EDF7E57FC083E50E94109892
:10A49000811103C0E4E0F8E507C00E94A59789E0B8
:10A4A00093E10F94F9215AC384917F012FEFE21AAF
:10A4B000F20A882321F00F941E14F701F5CF60E013
:10A4C00070E085EC9AE00F94762380910B1328E5D9
:10A4D00032E06901C81AD10887FDD394CC0CDD1C89
:10A4E000CC0CDD1C0D2C000CEE08FF0880910A132B
:10A4F00028E830E04901881A910887FD9394880C78
:10A50000991C880C991C092C000CAA08BB08809186
:10A5100009138F3FB9F090E0FC01EE0FFF1F8E0F83
:10A520009F1FFC01E456FD4E0181128153E0000F94
:10A53000111F5A95E1F764E0169507956A95E1F7C2
:10A540000E5F1F4F98012F5F3F4FC901330FAA0BBA
:10A55000BB0B9C01AD01281939094A095B09A4EB21
:10A56000B0E00F94EDCEA7019601281939094A09E8
:10A570005B090F94CECEB90182EC9AE00F9476235A
:10A580008AE00F941E14EAC284918F010F5F1F4F5F
:10A59000882321F00F941E14F801F6CFB6018BEB3F
:10A5A0009AE00F947623ECEAFAE084918F010F5F32
:10A5B0001F4F882309F4D2C20F941E14F801F5CF5F
:10A5C0008AE50E94599881115EC383E50E945998DB
:10A5D000811159C3C3C283E50E945998882319F099
:10A5E0000E94A59702C064E071E079A368A380E5AA
:10A5F0000E945998882339F00E94A597693833E161
:10A60000730730F402C068EE73E07A83698304C094
:10A6100088E893E19A838983BE01605E7F4FCE0113
:10A6200001960F94D7509AC283E50E941098182F74
:10A63000882371F00E94D9970F94B8D070937A0252
:10A640006093790221E0672B09F020E02093431802
:10A6500080E50E941098882359F02091790230916A
:10A660007A02232B11F00E94C9978093431876C277
:10A67000111174C2E4E0F8E584918F010F5F1F4F60
:10A68000882321F00F941E14F801F6CF809143180F
:10A69000882319F061E773E002C064E773E083EF99
:10A6A0009AE00F948E236091790270917A0282EE83
:10A6B0009AE00F947623EEEDFAE084918F010F5F1C
:10A6C0001F4F882309F44AC20F941E14F801F5CFD6
:10A6D0000F94812E43C280E50E941098882351F088
:10A6E0000E94D9976093F8187093F9188093FA181C
:10A6F0009093FB1889E40E941098882381F00E94AF
:10A70000D9972CEA35EC47E25EE30F94ACC860932E
:10A71000F4187093F5188093F6189093F71884E462
:10A720000E941098882381F00E94D9972CEA35EC7A
:10A7300047E25EE30F9446D06093F0187093F118EF
:10A740008093F2189093F318E4E0F8E584918F0178
:10A750000F5F1F4F882321F00F941E14F801F6CFCE
:10A760004091F8185091F9186091FA187091FB18FF
:10A770008EE09BE00F9459232CEA35EC47E25EE330
:10A780006091F4187091F5188091F6189091F7186F
:10A790000F9446D0AB01BC018AE09BE00F94592393
:10A7A0002CEA35EC47E25EE36091F0187091F11805
:10A7B0008091F2189091F3180F94ACC8AB01BC01D2
:10A7C00086E09BE00F9459238AE00F941E14C6C1C3
:10A7D00080E50E945998882331F00E94B5978093B4
:10A7E000551611E001C010E083E50E9459988823B6
:10A7F00029F00E94C9978093561601C011110F9439
:10A80000C76CE4E0F8E584918F010F5F1F4F882348
:10A8100021F00F941E14F801F6CF8091561688236C
:10A8200019F0E3E2FBE00DC0E2E1FBE084918F016F
:10A830000F5F1F4F882309F491C10F941E14F80174
:10A84000F5CF84918F010F5F1F4F882309F486C1D4
:10A850000F941E14F801F5CF0E94ECB67FC180E082
:10A860000F94F60E0F94763679C10F944C7176C121
:10A870000F94296173C10F94D05E70C183E50E946B
:10A880001098882321F00E94C99791E089270F949E
:10A89000225964C181E08093DA150E94438C1092A2
:10A8A000DA15882309F45AC1E4E0F8E584918F01B0
:10A8B0000F5F1F4F811103C0E3E3FBE004C00F945F
:10A8C0001E14F801F3CF84918F010F5F1F4F88236F
:10A8D00009F444C10F941E14F801F5CF80912C1394
:10A8E000882309F43BC181E080932F1337C18BE5A6
:10A8F00092E00F944818811131C185E50E941098AB
:10A900008823D9F10091121010E00E94D9976B01B1
:10A910007C0120E030E0A9010F94ACD187FF04C096
:10A92000F7FAF094F7F8F094000F111F000F111FC1
:10A93000F801EB5CF94EC082D182E282F382009191
:10A94000121084E0089F800111240B5C194E20E056
:10A9500030E048E453E4D8016D917D918D919C9154
:10A960000F94ACD118164CF480E090E0A8E4B3E466
:10A97000F80180839183A283B3838CE40E941098B2
:10A98000882309F4EBC00091121010E00E94D997BF
:10A990006B017C0120E030E0A9010F94ACD187FF6E
:10A9A00004C0F7FAF094F7F8F094000F111F000FAD
:10A9B000111FF801E35DF94EC082D182E282F38279
:10A9C00000911210F4E00F9F80011124035D194ED5
:10A9D00020E030E048E453E4D8016D917D918D9101
:10A9E0009C910F94ACD118160CF0B8C080E090E0A8
:10A9F000A8E4B3E4F80180839183A283B383AEC05B
:10AA00000F94D06CABC08AE50E945998811103C0A5
:10AA1000E4E0F8E53BC00E94D9976B017C0120E09F
:10AA200030E040EA51EC0F94ACD187FD0AC020E041
:10AA300030E040EA51E4C701B6010F9446C8181649
:10AA40001CF4E5EDF7E50CC0C092F40FD092F50FC1
:10AA5000E092F60FF092F70F81C00F941E14F801E8
:10AA600084918F010F5F1F4F8111F7CFEEE3FBE061
:10AA700084918F010F5F1F4F882309F46FC00F94DB
:10AA80001E14F801F5CF0F941E14F80184918F0164
:10AA90000F5F1F4F8111F7CFEEE5FBE084918F012F
:10AAA0000F5F1F4F882321F00F941E14F801F6CF7B
:10AAB0004091F40F5091F50F6091F60F7091F70FE0
:10AAC0008BE59BE00F9459238AE00F941E1446C037
:10AAD00081E0809380021092921883E50E94599839
:10AAE000882339F00E94C997811138C00F9465B549
:10AAF00035C083E50E941098F7CF0F94E89C2EC0D4
:10AB00000091F61A80914818081769F083E50E94B1
:10AB10005998882319F00E94C99703C083E50E94C1
:10AB20001098182F01C011E086E40E9459988823DC
:10AB300019F00E94D99703C060E070E0CB0120E0DB
:10AB400030E040E752E40F9446D0AB01BC01212F26
:10AB5000802F0F94A66902C00F94E89C10922618CB
:10AB60000F94F9B426C10E94ED780E943A64F6CFA2
:10AB700011110C944C480C94454880E00E94906F51
:10AB80000C946E480E94A597AB01BC014093CD1573
:10AB90005093CE156093CF157093D0158CE195E14D
:10ABA0000E94F857DBCF0E94B597853620F084E6E7
:10ABB0008093E915D3CF8093E915D0CF0E94ECB6EE
:10ABC00088E50E941098882361F05F9A80910B01BC
:10ABD0008095807280930901809153168E7F8093B7
:10ABE000531689E50E941098882331F08A9A809143
:10ABF00053168D7F809353168AE50E941098882300
:10AC000059F08091080180958170809306018091B0
:10AC100053168B7F8093531685E40E9410988823E7
:10AC200011F40C941D4E0E94B4630C941D4E0F94AD
:10AC300030B794CF0E94ECB6BC2C60E08C2D0F9402
:10AC4000B6AC0F3FFFEF1F0759F48C2D0F945EAC8D
:10AC500031E020E0892B09F030E0032F122F05C0EE
:10AC60000130110569F401E010E08B2D0F945EAC0A
:10AC70008017910709F472CF80E00E94906FF5CFA2
:10AC800000E010E0F2CF0E94D99720E030E040E0F1
:10AC900050EC0F9446C887FD15C00E94D99720E05C
:10ACA00030E040E050E40F94ACD118162CF00E9434
:10ACB000D9976B017C010BC0C12CD12CE12C30E465
:10ACC000F32E05C0C12CD12CE12C20ECF22E80916A
:10ACD000531682FF18C00091F20F1091F30F2091CC
:10ACE000AC183091AD184091AE185091AF18C70113
:10ACF000B6010F94ACC80F94B8D0600F711F709359
:10AD0000F30F6093F20F80E50E941098882329F0DA
:10AD10000E94C997882309F421CFA7019601609169
:10AD2000F40F7091F50F8091F60F9091F70F0F943B
:10AD30004CCF6093F40F7093F50F8093F60F9093C0
:10AD4000F70FE4E0F8E584918F010F5F1F4F882330
:10AD500021F00F941E14F801F6CF4091F40F50919A
:10AD6000F50F6091F60F7091F70F8DEC9AE00F944C
:10AD700059238AE00F941E14F1CE61E0812F0F94C5
:10AD8000B6AC6E2D812F0F9487ACF12CB701812FBB
:10AD90000F94F2AC193029F4F092EC17E092EB1713
:10ADA000DDCE1C3009F0DACEF092EE17E092ED170E
:10ADB000D5CECD5BDF4F0FB6F894DEBF0FBECDBF53
:10ADC000DF91CF911F910F91FF90EF90DF90CF9087
:10ADD000BF90AF909F908F907F906F905F904F90BB
:10ADE0003F902F9008953F924F925F926F927F9283
:10ADF0008F929F92AF92BF92CF92DF92EF92FF928B
:10AE00000F931F93CF93DF93CDB7DEB72C970FB679
:10AE1000F894DEBF0FBECDBF5C01DC0159968D906A
:10AE20009C905A97F40181859285A385B4859C01F5
:10AE3000AD012F5F3F4F4F4F5F4F29873A874B87B9
:10AE40005C87D5011496CD90DD90ED90FC9017971E
:10AE5000C114D104E104F10439F0BFEFCB1ADB0ACD
:10AE6000EB0AFB0A312C07C0F401C080D180E280DC
:10AE7000F38033243394260137011D821E821F8202
:10AE80001886F40181859285A385B4852D813E8144
:10AE90004F815885281739074A075B0708F064C0B7
:10AEA00089859A85AB85BC858C159D05AE05BF054A
:10AEB00050F482E0C82ED12CE12CF12C92E0492EE6
:10AEC000512C612C712C9E012F5F3F4FB701A601C1
:10AED000C4010E94FD93882309F446C089819A81A8
:10AEE000AB81BC81892B8A2B8B2B41F0260137014A
:10AEF0009FEF491A590A690A790A05C0C414D50492
:10AF0000E604F70491F02D813E814F8158852F5F33
:10AF10003F4F4F4F5F4F2D833E834F8358873FEF07
:10AF2000C31AD30AE30AF30AACCF0FEF1FEF2FEFD8
:10AF30003FE0B301A201C4010E946B93F82E882365
:10AF400099F0D50114964D915D916D917C91179773
:10AF5000411551056105710549F093018201C40154
:10AF60000E946B93811102C0F12C29C0D501149667
:10AF70004D925D926D927C921797332051F0D301E0
:10AF8000C2010196A11DB11DF40180839183A283AA
:10AF9000B383F50185899689A789B08D892B8A2B82
:10AFA0008B2B69F4D50155964D925D926D927C92F2
:10AFB000589711968C911197806811968C938F2DCC
:10AFC0002C960FB6F894DEBF0FBECDBFDF91CF91A8
:10AFD0001F910F91FF90EF90DF90CF90BF90AF90B7
:10AFE0009F908F907F906F905F904F903F900895CB
:10AFF0008F929F92AF92BF92CF92DF92EF92FF9289
:10B000000F931F93CF93DF93EC018B81811102C0CB
:10B0100080E078C009891A892B893C8904171507B3
:10B0200026073707A8F36A017B01823029F4C88616
:10B03000D986EA86FB860DC0C114D104E104F1046F
:10B0400051F4188619861A861B861C821D821E8260
:10B050001F8281E057C088849984AA84BB84E98DCB
:10B06000FA8D258530E0275F3F4FB501A40141509F
:10B07000510961097109022E04C0769567955795AB
:10B0800047950A94D2F7D701C6010197A109B109E2
:10B0900004C0B695A795979587952A95D2F78417FA
:10B0A0009507A607B70720F089288A288B2871F40E
:10B0B0004D895E896F89788D4C835D836E837F8334
:10B0C0004C015D018E010C5F1F4F16C0841B950B58
:10B0D000A60BB70BF5CF4C815D816E817F81980106
:10B0E000898D9A8D0E94FD9391E0891A9108A1089B
:10B0F000B108882309F48CCF81149104A104B10410
:10B1000051F795CFDF91CF911F910F91FF90EF9065
:10B11000DF90CF90BF90AF909F908F9008950F9346
:10B120001F93CF93DF93FC012381222311F080E052
:10B1300044C08B01EC01FB018789803139F18032F9
:10B14000B1F783E08B83F801428D538D648D758D4B
:10B150004D8B5E8B6F8B788F9E012F5E3F4FC801AA
:10B160000E947E94882319F31A8F098F81E08983C6
:10B17000188619861A861B861C821D821E821F82D3
:10B18000188A1C861D861E861F8617C082E08B8348
:10B190001D8A1E8A1F8A188EFB01808D918DA0E06A
:10B1A000B0E025E0880F991FAA1FBB1F2A95D1F791
:10B1B000898B9A8BAB8BBC8BD7CFDF91CF911F91B3
:10B1C0000F910895CF93DF93EC0141E0611101C02D
:10B1D00040E06C857D858E859F850E943293882313
:10B1E00041F0888920E2829FC0011124805E9F4E39
:10B1F00002C080E090E0DF91CF910895CF93DF937C
:10B20000EC018B81882339F1898187FF20C061E0BF
:10B21000CE010E94E258FC01892BE9F08081853E35
:10B22000D1F08B81823040F489899A89AB89BC89BD
:10B23000848F958FA68FB78F8D899E89AF89B88DA2
:10B24000938F828FB58BA48B89818F778983DF91D0
:10B25000CF910C94F29281E0888380E0DF91CF91CE
:10B260000895CF93DF93EC010E94FE581B82DF917B
:10B27000CF910895CF93DF93EB01FC01238121113E
:10B2800002C080E028C02250223020F48FE2888360
:10B29000198220C060E00E94E258009791F3FC01FF
:10B2A00090E080E02EE23081303269F0883029F47D
:10B2B000DE01A90FB11D2C939F5FDE01A90FB11D07
:10B2C00030813C939F5F8F5F31968B3061F7C90F60
:10B2D000D11D188281E0DF91CF91089540E050E0C8
:10B2E000BA010C94F85761E0FC0180810D9487ACA1
:10B2F0008EBD0DB407FEFDCF08958FEF8EBD0DB44A
:10B3000007FEFDCF8EB508950F931F93CF93DF9364
:10B31000EB010F94257D8B010E947D598F3F49F0F1
:10B320000F94257D601B710B6C177D07A8F380E0DF
:10B3300001C081E0DF91CF911F910F9108958F920D
:10B340009F92AF92BF92EF92FF921F93CF93DF93A2
:10B35000EC01162F49015A019A81892F806A86953E
:10B360008CBD90FD03C081E0963009F480E08DBD76
:10B3700060E088810F9487AC6CE271E0CE010E949E
:10B380008459812F80640E94785988E1E82EF12C3D
:10B39000D501C4010E2C04C0B695A7959795879545
:10B3A0000A94D2F70E94785988E0E81AF10888EFE9
:10B3B000E8168FEFF80661F71123A9F0183011F4A1
:10B3C00087E801C08FEF0E9478591C3011F40E9469
:10B3D0007D5910E00E947D598B8387FF08C01F3F75
:10B3E00031F01F5FF7CF85E90E947859F2CFDF91E6
:10B3F000CF911F91FF90EF90BF90AF909F908F9053
:10B4000008950F931F93CF93DF93EC0189018C81F3
:10B41000833039F089E0440F551F661F771F8A95E6
:10B42000D1F79A01AB0168E1CE010E949F598823B0
:10B4300011F086E031C08EEF8EBDF801C8019E5F2D
:10B440000DB407FEFDCF20812EBD0DB407FEFDCF4C
:10B4500021812EBD32968E179F0791F70DB407FEFE
:10B46000FDCF8FEF0E9478598FEF0E9478590E948C
:10B470007D598B838F71853031F083E18983CE01D3
:10B480000E9473590AC068E572E0CE010E94845997
:10B49000182F811107C087E18983CE010E9473595B
:10B4A00010E012C020E030E0A9016DE0CE010E9462
:10B4B0009F59811104C00E947D59882311F086E1B3
:10B4C000EBCFCE010E947359812FDF91CF911F9155
:10B4D0000F9108952F923F924F925F926F927F92B9
:10B4E0008F929F92AF92BF92CF92DF92EF92FF9294
:10B4F0000F931F93CF93DF9300D01F92CDB7DEB78A
:10B500008C014B011A01DC0113968C911397813049
:10B51000C9F411968C9181FF15C082FF19C0F80102
:10B52000418952896389748980859185A285B38513
:10B5300084179507A607B70759F0C8010E94F85766
:10B54000811106C081E0D8018C938FEF9FEF2DC150
:10B55000610185C059968D919C915A97FC01748028
:10B560002FEF270D2A013B0139E076946794579419
:10B5700047943A95D1F7722E74207A01F1E0FF22B8
:10B58000772009F478C080E092E08E199F09560177
:10B590008C159D0508F45C01D80159962D913C91BC
:10B5A0005A9714968D919D910D90BC91A02D029764
:10B5B000A109B109F901058404C0880F991FAA1FC8
:10B5C000BB1F0A94D2F74685578560897189840F1D
:10B5D000951FA61FB71F9C01AD01270D311D411DF1
:10B5E000511D29013A01A11432E0B30609F08AC0C5
:10B5F0008091201290912112A0912212B0912312D9
:10B60000481659066A067B0669F4109228128FEFD5
:10B610009FEFDC018093201290932112A0932212BD
:10B62000B09323129401B301A20180912912909149
:10B630002A120E94015A882309F484CFF8018085D8
:10B640009185A285B3858A0D9B1DA11DB11D8087A3
:10B650009187A287B3878A0C9B1CCA18DB08D80184
:10B6600018964D915D916D917C911B97C114D104F9
:10B6700009F070CF7DC0E114F10409F084CF149675
:10B680004D915D916D917C91179741155105610523
:10B69000710559F455968D919D910D90BC91A02DF9
:10B6A0000097A105B10541F521C09E012F5F3F4FD5
:10B6B0000E94FD93882309F445CF89819A81AB814B
:10B6C000BC81F801218D328DF9012789203139F4AF
:10B6D000883FFFEF9F07A105B10540F40DC0883FEB
:10B6E0002FEF9207A2072FE0B20730F0C8010E94A7
:10B6F000F356811148CF26CFF80184839583A68322
:10B70000B78341CFE114F10419F5D80118964D9192
:10B710005D916D917C911B9751968D919D910D90AE
:10B72000BC91A02D481759076A077B0788F00E9433
:10B73000F292882309F406CF81E080932812409288
:10B74000201250922112609222127092231208C08D
:10B7500041E0C301B2010E943293882309F4F2CE82
:10B76000A501B401C701805E9F4E0F94CBD366CF75
:10B77000F80181899289A389B48984179507A6075E
:10B78000B70738F4418B528B638B748B818180684F
:10B790008183F801818183FD02C0C10106C0C80117
:10B7A0000E94FE588111F9CFCDCE0F900F900F90CF
:10B7B0000F90DF91CF911F910F91FF90EF90DF904D
:10B7C000CF90BF90AF909F908F907F906F905F9041
:10B7D0004F903F902F900895EF92FF920F931F93F9
:10B7E000CF93DF93EC0179018C81833039F089E0CC
:10B7F000440F551F661F771F8A95D1F79A01AB0139
:10B8000061E1CE010E949F59882331F084E0898351
:10B81000CE010E9473593CC00F94257D8B010E947C
:10B820007D598B838F3F49F40F94257D601B710BED
:10B830006D327140A0F381E103C08E3F49F08FE08B
:10B840008983CE010E9473598FEF0E94785920C0DE
:10B850008FEF8EBDF701D701A150BE4F0DB407FE8B
:10B86000FDCF9EB591938EBDEA17FB07B9F70DB4D6
:10B8700007FEFDCF8EB58C930E947D590E947D59A5
:10B88000CE010E9473598FEF0E94785981E001C068
:10B8900080E0DF91CF911F910F91FF90EF9008957D
:10B8A0002F923F924F925F926F927F928F929F92D0
:10B8B000AF92BF92CF92DF92EF92FF920F931F93BE
:10B8C000CF93DF9300D01F92CDB7DEB79C838B83DD
:10B8D0004B015A01DC0113968C91811103C08FEF4B
:10B8E0009FEFEBC0EB81FC81818180FFF8CFAB81C2
:10B8F000BC8151960D911D912D913C9154971896B4
:10B900004D915D916D917C911B97C501A0E0B0E0D8
:10B9100068017901C41AD50AE60AF70AC816D906D9
:10B92000EA06FB0618F45801A41AB50A75018B81C2
:10B930009C8104969A838983612C42E0742EE114E1
:10B94000F10409F48BC0AB81BC8118964D915D91D7
:10B950006D917C911B976A01B1E0DB22EB81FC8148
:10B960002381818D928D1A012B0139E056944794E1
:10B97000379427943A95D1F7223061F4FC01828DF7
:10B98000938DA48DB58DBC01CD01620D731D841DF9
:10B99000951D4AC0DC0114961C9111501221C1144E
:10B9A000D10401F511111EC0452B462B472B59F42C
:10B9B000EB81FC8185899689A789B08D84839583E5
:10B9C000A683B7830FC0AB81BC8114964D915D9166
:10B9D0006D917C91179729813A810E94FD9388236C
:10B9E00009F47DCFEB81FC81218D328D848195819D
:10B9F000A681B7810297A109B109F901058404C0A4
:10BA0000880F991FAA1FBB1F0A94D2F74685578536
:10BA100060897189840F951FA61FB71FBC01CD01D6
:10BA2000610F711D811D911D93012C193D09870125
:10BA30002E153F0508F489010115F2E01F0779F57D
:10BA40002091201230912112409122125091231204
:10BA5000621773078407950719F421C0C5012DC02B
:10BA60009401AB01BC018091291290912A120E948D
:10BA7000EC5B882309F433CF800E911EEB81FC81AF
:10BA800080859185A285B385800F911FA11DB11D71
:10BA900080879187A287B387E01AF10A50CF40E0F0
:10BAA0000E943293882309F41ACFB601605E7F4E5C
:10BAB000A801C4010F94CBD3DFCF0F900F900F904C
:10BAC0000F90DF91CF911F910F91FF90EF90DF903A
:10BAD000CF90BF90AF909F908F907F906F905F902E
:10BAE0004F903F902F9008954F925F926F927F9268
:10BAF0009F92AF92BF92CF92DF92EF92FF920F93FD
:10BB00001F93CF93DF931F92CDB7DEB78C017B01DC
:10BB10005A01C22EDB0159968D919C915A97F801DA
:10BB2000928F818FCB010E946E59912CF7018085F5
:10BB30009185A285B3854189528963897489841767
:10BB40009507A607B70708F060C025E0B695A7954A
:10BB5000979587952A95D1F7F82FFF70DF2ED7019B
:10BB600013968C91823008F460C041E050E0BE0131
:10BB70006F5F7F4FC7010E94505C019719F4898164
:10BB800090E002C08FEF9FEF019609F44EC0F701DD
:10BB900080859185A285B3854F96A11DB11D8087B3
:10BBA0009187A287B387F0E2DF9EB0011124605E27
:10BBB0007F4E61157105C9F1DB018C91882319F065
:10BBC000853EC1F46CC191100EC0809120129091FD
:10BBD0002112A0912212B0912312F8018487958737
:10BBE000A687B787D08ADB018C91882361F09924DE
:10BBF00093949CCF4BE050E0C5010F94BED3892BAA
:10BC000009F094CF14C0992493948C2D82748234BB
:10BC100061F4992009F48BC0F801D08861E0C80173
:10BC20000E94E258009709F00DC180E03BC1C7FCBB
:10BC3000FCCFF0E2DF9EA00111249A01205E3F4E6E
:10BC4000D9011B968C91817121F08C2D827109F0A4
:10BC50006AC08091201290912112A0912212B0917D
:10BC60002312F80184879587A687B787D08ACA01EF
:10BC7000805E9F4E7C01DC0154964D915C915597FE
:10BC800060E070E0DA0199278827858B968BA78B77
:10BC9000B08FF701428D538D60E070E0482B592B37
:10BCA0006A2B7B2BD80155964D935D936D937C93B6
:10BCB0005897F9018385887161F4F701848D958D1A
:10BCC000A68DB78DF801818B928BA38BB48B81E00D
:10BCD00010C0803141F598012F5E3F4FD801599631
:10BCE0008D919C915A970E947E948823E1F084E084
:10BCF000F80183838C2D8F70D80111968C93119746
:10BD0000F801148215821682178218961D921D92D0
:10BD10001D921C921B97C4FEB5C0C8010F944E51D2
:10BD20008111B0C082CFD80113961C927ECFD7016B
:10BD300013968C911397823009F477CF51968D9199
:10BD40009D910D90BC91A02D803E9F4FAF41B105BC
:10BD500008F06BCFC7010E94F356882309F465CF22
:10BD60000E94F292882309F460CFD70159962D9151
:10BD70003C915A9714968D919D910D90BC91A02D58
:10BD80000297A109B109F901058404C0880F991F20
:10BD9000AA1FBB1F0A94D2F7468457846088718813
:10BDA000480E591E6A1E7B1E81E080932812409225
:10BDB000201250922112609222127092231280E07F
:10BDC00092E0E0E2F0E1DF019C011D922150304061
:10BDD000E1F7DD24D394D7015996ED91FC915A9760
:10BDE0008481D81698F420E230E1B301A2014D0D10
:10BDF000511D611D711D8091291290912A120E947E
:10BE0000015A882309F411CFD394E5CF80E092E062
:10BE1000A0E0B0E0058404C0880F991FAA1FBB1FD3
:10BE20000A94D2F7F7014189528963897489840F92
:10BE3000951FA61FB71F818B928BA38BB48B80E2BB
:10BE400090E1D12C20E2DC011D922A95E9F72BE04C
:10BE5000F501DC0101900D922A95E1F721E238E22B
:10BE6000FC01318B208B40E058E057874687338BAD
:10BE7000228B318F208F578B468B0E94F29281113B
:10BE8000D8CED3CEC5FE09C0F80141895289638955
:10BE90007489C8010E94F85705C081E003C0911061
:10BEA000A6CE93CE0F90DF91CF911F910F91FF906F
:10BEB000EF90DF90CF90BF90AF909F907F906F906A
:10BEC0005F904F9008958F929F92AF92BF92CF92C2
:10BED000DF92EF92FF920F931F93CF93DF93CDB733
:10BEE000DEB728970FB6F894DEBF0FBECDBF7C013A
:10BEF0006B018A01A22EEAEEFBE084914F019FEFD5
:10BF0000891A990A882321F00F941E14F401F5CFA1
:10BF10008091491883FD46C020E030E0A901F80176
:10BF200060817181828193810F9446C8882309F4CE
:10BF300039C0B0904318B11035C0E0914818F0E016
:10BF4000EE0FFF1FEC5BF74E20813181809179026B
:10BF500090917A02281739072CF5E5EDF7E58491E1
:10BF60008F010F5F1F4F882321F00F941E14F801DB
:10BF7000F6CFE9EDFBE084918F010F5F1F4F88231F
:10BF800021F00F941E14F801F6CFAA2029F0609139
:10BF9000481887E00F94699A60E08AEC9BE00E9461
:10BFA00066C4E3C08091311291E0980F90933112F2
:10BFB00090912C13992329F010922C138E5F80936B
:10BFC00031120F94F7A080E1ECEBF8E1A9E2B8E1BF
:10BFD00001900D928A95E1F70E94ECB620E030E0E6
:10BFE000A901F70160817181828193810F9446C814
:10BFF000882339F180914318811115C0E0914818C8
:10C0000084E0E89FF0011124E55CF74E60817181C6
:10C01000828193810F94B8D02091790230917A0275
:10C020006217730774F080E090E0A0E7B2E48983C0
:10C030009A83AB83BC83BE016F5F7F4FC7010E94B1
:10C04000977841E061E081E00F949F14811107C06F
:10C0500082E08983B601CE0101960E9412B820E0E9
:10C0600030E0A901F80160817181828193810F9490
:10C0700046C8882361F00F94A49AB82E81110AC093
:10C08000AA2029F06091481887E00F94699ABB2490
:10C09000B3946BC0AA2029F06091481881E00F94F6
:10C0A000699A80E090E0A0E7B2E48D839E83AF833D
:10C0B000B88780E090E0A0E8B0EC89839A83AB83F6
:10C0C000BC83BE016B5F7F4FCE0101960E949778C3
:10C0D00068E873E180E090E00E944FC380E090E068
:10C0E000A0E8B0E489839A83AB83BC836AEB7AE1EE
:10C0F000CE0101960E949778C0902118D090221806
:10C10000E0902318F090241880E090E0A8ECB1E4CF
:10C110008093211890932218A0932318B093241889
:10C1200080E090E0A4E2B2E489839A83AB83BC838D
:10C13000BE016F5F7F4FC8010E949778C09221189F
:10C14000D0922218E0922318F09224188091481877
:10C15000882321F0813019F4479A01C0129A64E6CD
:10C1600070E080E090E00E944FC38B2D28960FB6C0
:10C17000F894DEBF0FBECDBFDF91CF911F910F911D
:10C18000FF90EF90DF90CF90BF90AF909F908F90F7
:10C1900008954F925F926F927F928F929F92AF928B
:10C1A000BF92CF92DF92EF92FF920F931F93CF93A4
:10C1B000C82FC82ED12C811107C080914818811139
:10C1C00013C00FEF1FEF12C0F601E953F44F0491B3
:10C1D000002E000C110B823049F481E00F94F60E12
:10C1E000882309F4C2C0FAC001E010E07601EE0C29
:10C1F000FF1CEE0CFF1CF701E554F44F45905590E1
:10C2000065907490B801110F880B990B0F944DC86D
:10C210004B015C0120E030E040EC5FE3C301B20180
:10C220000F94ACC8A50194010F94ACC8AB01BC013C
:10C2300000E010E098018C2F0E947179C23009F063
:10C2400088C080E00F942514E0E070E060EA80E4AC
:10C250002E2F372F462F582FC501B4010F94ACC88D
:10C260004B015C0120E030E0A9010F9446C888230F
:10C2700009F446C0C23021F000E010E0980104C08B
:10C2800000E010E020E830E4B501A40170588C2FE4
:10C290000E947179C23009F06EC081E00F942514BC
:10C2A00081119CC0412C512C612C90E4792E15C039
:10C2B0006AE0F701E658F44F459055906590749008
:10C2C00070E080E090E00F944DC89B01AC01C30189
:10C2D000B2010F9446D02B013C01A5019401C50188
:10C2E000B4010F944CCFAB01BC01930182018C2FA0
:10C2F0000E947179C23009F05DC080E00F9425146E
:10C300008C2F0F944B100F944E11F701E053F74E02
:10C31000D701A454B74E8D919D910D90BC91A02D45
:10C3200080839183A283B383C23009F057C080E039
:10C33000CF911F910F91FF90EF90DF90CF90BF9022
:10C34000AF909F908F907F906F905F904F900D94E3
:10C35000F60EF701E155F44F85919591A591B491B1
:10C36000E82F792F6A2F8B2F73CF81E00F9425143C
:10C37000811134C03BCFF601E455F44F6491611153
:10C3800098CFE4E0F8E584918F010F5F1F4F882379
:10C3900021F00F941E14F801F6CFEAE8FBE0849137
:10C3A0008F010F5F1F4F882309F482CF0F941E1453
:10C3B000F801F5CF8C2F0F944B100F944E11D7012D
:10C3C000A053B74EF701E454F74E4081518162818A
:10C3D00073814D935D936D937C931397CF911F91D0
:10C3E0000F91FF90EF90DF90CF90BF90AF909F9014
:10C3F0008F907F906F905F904F9008958CE0EEE467
:10C40000F9E0ACEBB8E101900D928A95E1F708955F
:10C41000CF92DF92EF92FF92CF93DF93EC01C09027
:10C42000A705D090A805E090A905F090AA05A7015E
:10C430009601688179818A819B810F9446C887FF24
:10C4400004C0C882D982EA82FB82C090AB05D0903A
:10C45000AC05E090AD05F090AE05A70196016C81AA
:10C460007D818E819F810F9446C887FF04C0CC8256
:10C47000DD82EE82FF82C0902102D0902202E09005
:10C480002302F0902402A7019601688179818A81B4
:10C490009B810F94ACD1181624F4C882D982EA8209
:10C4A000FB82C0902502D0902602E0902702F090F7
:10C4B0002802A70196016C817D818E819F810F9456
:10C4C000ACD1181624F4CC82DD82EE82FF82C090BB
:10C4D000AF05D090B005E090B105F090B205A7018E
:10C4E0009601688579858A859B850F9446C887FF64
:10C4F00004C0C886D986EA86FB86C0902902D090FF
:10C500002A02E0902B02F0902C02A7019601688588
:10C5100079858A859B850F94ACD1181624F4C8863A
:10C52000D986EA86FB86DF91CF91FF90EF90DF906E
:10C53000CF9008950F931F93CF93DF938C01E4E086
:10C54000F8E58491EF012196882321F00F941E14C1
:10C55000FE01F7CFB8018DE69BE00F948E2382E2B7
:10C560000F941E148AE00F941E1481E0DF91CF9186
:10C570001F910F9108952F923F924F925F926F9269
:10C580007F928F929F92AF92BF92CF92DF92EF9263
:10C59000FF920F931F93CF93DF93CDB7DEB7C254B3
:10C5A000D1090FB6F894DEBF0FBECDBF4C015B01C1
:10C5B0006A01322E19821C821C8E1F8E6115710534
:10C5C00011F410E0A6C0FC0183818111FACFFA01B9
:10C5D00080818F3209F09BC0F501838182508230C7
:10C5E00010F485010CC0F501618D728DCE014C9661
:10C5F0000E948F58882329F38E01045E1F4FC601C5
:10C600006C010196F60120812F32D1F3CE01019603
:10C610007C013C012E019CE1490E511C2396EFAE9A
:10C6200023972F2C9BE09150E7E3F0E0EC0FFD1FE8
:10C63000E90FF11D80E280839111F5CF960147E06B
:10C64000D9018D91882369F18F3259F18E3239F4F5
:10C650004A3009F4B6CF98E04AE09D01F1CFEAEF05
:10C66000FBE02491222321F031968213FACFA9CF47
:10C67000491708F4A6CF813208F4A3CF8F3709F405
:10C68000A0CF21E0290FE7E3F0E0EC0FFD1FE90F59
:10C69000F11D9FE9980F9A3108F480528083922F00
:10C6A000DCCF8FA9803209F48CCF6901F901808138
:10C6B0002F5F3F4F8F32C9F38823F9F021E0AE019D
:10C6C000495C5F4FB801C7010E94745D882309F47B
:10C6D00078CF0A151B0519F0C8010E9431596E1454
:10C6E0007F0441F023969FAD2397822D8701E92E89
:10C6F000F82E98CF942D852DF9CF232DAE01495CCE
:10C700005F4FB801C4010E94745D182F02C08B01F5
:10C710007DCFCE014C960F940D14CE0101960F944F
:10C720000D14812FCE5BDF4F0FB6F894DEBF0FBE26
:10C73000CDBFDF91CF911F910F91FF90EF90DF90D0
:10C74000CF90BF90AF909F908F907F906F905F90B1
:10C750004F903F902F9008952DE433E0FC013183FA
:10C76000208304960D940D14129A479A08955F9AA7
:10C7700080910B01809580728093090180915316FE
:10C780008E7F809353168A9A809153168D7F809363
:10C7900053168091080180958170809306018091E5
:10C7A00053168B7F809353160C94B4638C01E5ED84
:10C7B000F7E58491EF012196882321F00F941E1450
:10C7C000FE01F7CFEBE4FDE08491EF012196882391
:10C7D00021F00F941E14FE01F7CF0F9421A10E94A7
:10C7E000B7630E940DC861E0C8010E9466C40F943F
:10C7F0006962C0913912C695C6950F94A450DC2F7A
:10C80000DD0F1D2F1C0F84E00F94ED6210926F124C
:10C81000C093701266E18FE498E10F94D962109290
:10C820006F12D09370128CE39DE00F94D94F109249
:10C830006F12109370128FE29DE00F94D94F0F94F6
:10C840009A4F8111E0CF2FEF8BE49DE12150804082
:10C850009040E1F700C00000F8942FEF84E39CE0E3
:10C86000215080409040E1F700C000000F9421A1CA
:10C87000A895FECF2F923F924F925F926F927F9238
:10C880008F929F92AF92BF92CF92DF92EF92FF92E0
:10C890000F931F93CF93DF93CDB7DEB7CF55D10959
:10C8A0000FB6F894DEBF0FBECDBF80912D02882356
:10C8B00021F080ED98E10E9408628091491883FD83
:10C8C000ABC0C090DC18D090DD18E090DE18F0907E
:10C8D000DF182091C8183091C9184091CA1850919A
:10C8E000CB18C701B6010F9446C8882309F494C039
:10C8F00080914318811136C0E091481804E0E09F10
:10C90000F0011124E55CF74E608171818281938191
:10C910000F94B8D02091790230917A026217730790
:10C920000CF5C092C818D092C918E092CA18F092BB
:10C93000CB18E4E0F8E584918F010F5F1F4F811160
:10C9400003C0E2E6FCE004C00F941E14F801F3CF2C
:10C9500084918F010F5F1F4F882321F00F941E14C5
:10C96000F801F6CF8090DC189090DD18A090DE18CA
:10C97000B090DF182091C8183091C9184091CA189A
:10C980005091CB18C501B4010F944BCF6B017C01C2
:10C9900020E030E0A9010F94ACD187FF04C0F7FA82
:10C9A000F094F7F8F094E091481814E0E19FF0015A
:10C9B0001124E25DFD4F2081318142815381C70105
:10C9C000B6010F94ACC820E030E048E453E40F9483
:10C9D000ACD118160CF58092C8189092C918A09284
:10C9E000CA18B092CB18E4E0F8E584918F010F5F8C
:10C9F0001F4F811103C0E3E4FCE004C00F941E1438
:10CA0000F801F3CF84918F010F5F1F4F882321F02E
:10CA10000F941E14F801F6CF8091A704882309F41F
:10CA2000F9C080910802813021F0823009F4A6C05B
:10CA3000F1C02091DC183091DD184091DE18509142
:10CA4000DF186091C8187091C9188091CA18909128
:10CA5000CB180F9446C8811139C08091A9049091D8
:10CA6000AA04A091AB04B091AC048F3F9F4FAF4F8D
:10CA7000BF4F61F10E94D299C090D818D090D918B8
:10CA8000E090DA18F090DB18A701960160919F04FE
:10CA90007091A0048091A1049091A2040F9446C8C3
:10CAA00087FF08C0C0929F04D092A004E092A10426
:10CAB000F092A2040F94257D6093A9047093AA04B8
:10CAC0008093AB049093AC040C94766FF12CE090BF
:10CAD000481831E0F3121BC0C090B21AD090B31ABC
:10CAE0000091B41A1091B51A8090AE1A9090AF1AB6
:10CAF000A090B01AB090B11A9401A501B601C80176
:10CB00000F94ACD118165CF46401850108C0C09084
:10CB1000B61AD090B71A0091B81A1091B91AC60176
:10CB2000D80189839A83AB83BC8342E0F41609F46D
:10CB30006AC04FE954E0F11068C06BE974E087E91E
:10CB400094E019A21AA21BA21CA2DE0191966D010B
:10CB50008E010F5F1F4F28EC38E10E9491A78823B8
:10CB600021F0F394B3E0FB12B2CF1092A90410921B
:10CB7000AA041092AB041092AC0442C080914818F1
:10CB8000811148C028EC38E144EC58E160EC78E1D0
:10CB900084E092E00F94722420910002309101020F
:10CBA00040910202509103026091BC187091BD182F
:10CBB0008091BE189091BF180F944CCF69837A83EF
:10CBC0008B839C831DA21EA21FA218A6FE01B596F0
:10CBD0006F01EE24E3940EEA1AE128EC38E144EC0C
:10CBE00058E160EC78E1CE0101960E9491A788237C
:10CBF00089F00E94ECB60F944E1181E08093890F6A
:10CC00001092A70407C044EC58E160EC78E18CEB8B
:10CC100098E197CF8091A318F0904818FFAE00914B
:10CC20003A0210913B02882311F40C94336FC090A8
:10CC3000E015D090E115E090E215F090E31520E0CA
:10CC400030E0A901C701B6010F9446C8882381F0DE
:10CC50002091D8183091D9184091DA185091DB18EA
:10CC6000C701B6010F94ACD1181614F00C94336FB1
:10CC7000B801110F880B990B0F944DC82091090230
:10CC800030910A0240910B0250910C020F94ACC8F3
:10CC90002AE037ED43E25CE30F94ACC86D8F7E8FE2
:10CCA0008F8F98A36091BC187091BD188091BE18A9
:10CCB0009091BF180F94F381E82E880FFF08FAA611
:10CCC000E9A66091C0187091C1188091C218909126
:10CCD000C3180F94F381082F880F110B1AAB09ABFF
:10CCE000C090D018D090D118E090D218F090D318FE
:10CCF000C701B6010F94F3816F968FAF6F97282FFE
:10CD0000022E000C330B3AAF29AF6091D41870910A
:10CD1000D5188091D6189091D7180F94F381A096CA
:10CD20008FAFA097282E880F33088091A8048823FE
:10CD300081F1B701A6018CE19CE00F945923409149
:10CD4000D4185091D5186091D6187091D71886E1F3
:10CD50009CE00F9459234091D8185091D9186091B4
:10CD6000DA187091DB1880E19CE00F945923409110
:10CD7000DC185091DD186091DE187091DF188AE0A0
:10CD80009CE00F94592389E20F941E148AE00F94BB
:10CD90001E1449A55AA589AD9AAD4817590729F51A
:10CDA000A9A9BAA9A215B30501F50F9728F4BFE008
:10CDB0002B16310408F45FC119821A821B821C826F
:10CDC00020E030E0A9016091D8187091D9188091C5
:10CDD000DA189091DB180F944CCF6D837E838F838C
:10CDE0009887FE0131966F017FC2E090BC18F090E9
:10CDF000BD180091BE181091BF18EDA6FEA60FA792
:10CE000018ABA80197016091D0187091D11880914A
:10CE1000D2189091D3180F944BCF6B017C010091E5
:10CE2000C0181091C1182091C2183091C3180BAFCF
:10CE30001CAF2DAF3EAFA90198016091D41870913D
:10CE4000D5188091D6189091D7180F944BCF4B01DD
:10CE50005C0121E030E064963FAF2EAF649720E0A4
:10CE600030E0A9010F9446C887FD04C064961FAE48
:10CE70001EAE649720E030E0A901C701B6010F940F
:10CE800046C887FF3BC2D701C601B05824968CAF75
:10CE90009DAFAEAFBFAF249720E030E0A901C50140
:10CEA000B4010F9446C887FF30C295018401305801
:10CEB00028960CAF1DAF2EAF3FAF289729A53AA5F6
:10CEC00049AD5AAD2417350709F426C220E030E0F9
:10CED000A901C701B6010F9446C887FD20C281E0B1
:10CEE00090E09EAB8DABE9A9FAA9E215F30509F430
:10CEF0001BC220E030E0A901C501B4010F9446C86F
:10CF000087FD17C201E010E02E961FAF0EAF2E97DF
:10CF100028962CAD3DAD4EAD5FAD289724966CADF7
:10CF20007DAD8EAD9FAD24970F94ACD118160CF04B
:10CF300007C2260137012091C8183091C9184091C5
:10CF4000CA185091CB186091DC187091DD1880914F
:10CF5000DE189091DF180F944BCF698F7A8F8B8FEB
:10CF60009C8F9201A3010F9446D062966CAF7DAF67
:10CF70008EAF9FAF62972091C4183091C518409131
:10CF8000C6185091C7186091D8187091D91880911F
:10CF9000DA189091DB180F944BCF9201A3010F94F4
:10CFA00046D068966CAF7DAF8EAF9FAF6897A701F4
:10CFB0009601C501B4010F9446D02C966CAF7DAF9D
:10CFC0008EAF9FAF2C979B01AC016DA57EA58FA561
:10CFD00098A90F94ACC89B01AC016BAD7CAD8DAD35
:10CFE0009EAD0F944BCF6C966CAF7DAF8EAF9FAF65
:10CFF0006C9762968CAD9DADAEADBFAD6297BF77BD
:10D000008DA79EA7AFA7B8ABADA9BEA9AB2B09F062
:10D0100010C364966EAC7FAC6497E9A9FAA96E0E52
:10D020007F1E64964EAC5FAC6497420C531C2C96EA
:10D030000CAD1DAD2EAD3FAD2C973F770DAB1EABAC
:10D040002FAB38AF4614570409F07DC12091D0189A
:10D050003091D1184091D2185091D3186091BC18DA
:10D060007091BD188091BE189091BF180F9446C85A
:10D07000882309F4E3C68090D0189090D118A0902E
:10D08000D218B090D3186F96FFAC6F97EF2DF0E0E9
:10D09000EF3068F4EE0FFF1FEE0FFF1FE855F84C5E
:10D0A0000591159125913491B801D90113C0BF01A3
:10D0B000FF0F880B990B0F944DC82EE63BED4EEDFC
:10D0C00051E40F94ACC820E030E040EA50E40F9403
:10D0D0004CCFDC0149AD5AAD4F5F5F4F8FE0849F6D
:10D0E0009001859F300D1124F901E20DF31DEE0F23
:10D0F000FF1FEE0FFF1FE653FA4FE080F180028121
:10D100001381EDA6FEA60FA718AB09AD1AAD809F3F
:10D11000A001819F500D1124FA01E20DF31DEE0FC5
:10D12000FF1FEE0FFF1FE653FA4F408051806280D1
:10D130007380C1010196F901E80FF91FEE0FFF1F7F
:10D14000EE0FFF1FE653FA4FE080F180028113815A
:10D15000E9AAFAAA0BAB1CABFA01E80FF91FEE0F14
:10D16000FF1FEE0FFF1FE653FA4FC080D180E28011
:10D17000F38009AD1AAD0E3011059CF59B01AD0190
:10D18000C501B4010F944BCF20E339E043E15DE3E7
:10D190000F94ACC84B015C01A30192016DA57EA563
:10D1A0008FA598A90F944BCFA50194010F94ACC8FB
:10D1B000A30192010F944CCF2B013C01A7019601D2
:10D1C00069A97AA98BA99CA90F944BCFA5019401B9
:10D1D0000F94ACC8A70196010F944CCF6B017C0152
:10D1E00005C0C12CD12C760126013701A0961FADB8
:10D1F000A097E12FF0E01F3068F4EE0FFF1FEE0F55
:10D20000FF1FE859F84C4591559165917491FA01C9
:10D21000CB0113C0BF01FF0F880B990B0F944DC8B2
:10D220002EE63BED4EED51E40F94ACC820E030E02B
:10D2300040EA50E40F944CCFFB010EE0201631047D
:10D240000CF044C69F01AC016091D4187091D518C0
:10D250008091D6189091D7180F944BCF20E339E0E6
:10D2600043E15DE30F94ACC84B015C01A301920163
:10D27000C701B6010F944BCF9B01AC01C501B401AE
:10D280000F94ACC8A30192010F944CCF6B017C01A9
:10D2900088ED98E10E9498B79B01AC01C701B601E7
:10D2A0000F94ACC86B017C0119821A821B821C820C
:10D2B0008090D8189090D918A090DA18B090DB1808
:10D2C0009B01AC010F9499D281110CC6A501940168
:10D2D000C701B6010F944CCF6D837E838F839887EF
:10D2E0009E012F5F3F4F6901EFAC8E01035E1F4F20
:10D2F0002CED38E1AE014B5F5F4FDFC52496CCAE1D
:10D30000DDAEEEAEFFAE2497C7CD28968CAE9DAEB7
:10D31000AEAEBFAE2897D2CD1EAA1DAAE4CDAFEF08
:10D32000BFEFBEABADABDFCD2E961FAE1EAE2E97C0
:10D33000EFCD2FEF3FEF2E963FAF2EAF2E97E8CDDC
:10D3400024013501F8CD2E962EAD3FAD2E97620EFD
:10D35000731E162DF301FF271F3078F4EE0FFF1F09
:10D36000EE0FFF1FE859F84C85919591A591B49166
:10D37000D82EE92EFA2E0B2F16C0BF01FF0F880BF7
:10D38000990B0F944DC82EE63BED4EED51E40F94F2
:10D39000ACC820E030E040EA50E40F944CCFD62EE9
:10D3A000E72EF82E092F2FEF3FEF4FE75FE76DA92C
:10D3B0007EA98FA998AD0F9499D2811115C02FEF36
:10D3C0003FEF4FE75FE76DA97EA98FA998AD0F9456
:10D3D00046C818164CF46091BC187091BD18809125
:10D3E000BE189091BF1814C06C962CAD3DAD4EADDB
:10D3F0005FAD6C976D2D7E2D8F2D902F0F944BCFA1
:10D400002C962CAD3DAD4EAD5FAD2C970F9446D014
:10D410006D877E878F87988B49A55AA54F30510518
:10D4200070F45FE06516710450F4A30169A57AA554
:10D43000CE010D960F9468816B017C0103C0C12C55
:10D44000D12C760188ED98E10E9498B7A70196014A
:10D450000F94ACC86B017C019B01AC010F9499D275
:10D46000882319F0C12CD12C7601F301FF271F303E
:10D4700068F4EE0FFF1FEE0FFF1FE859F84C85917F
:10D480009591A591B4914C015D0114C0BF01FF0FAE
:10D49000880B990B0F944DC82EE63BED4EED51E4F1
:10D4A0000F94ACC820E030E040EA50E40F944CCF39
:10D4B0004B015C01C401D50189879A87AB87BC8782
:10D4C0008091C0189091C118A091C218B091C31852
:10D4D00089AB9AABABABBCAB9C01AD01B401C50150
:10D4E0000F9446C8882309F4ADCD2FEF3FEF4FE7E7
:10D4F0005FE76DA57EA58FA598A90F9499D281119C
:10D500000DC02FEF3FEF4FE75FE76DA57EA58FA51D
:10D5100098A90F9446C818160CF456C028962CAD3E
:10D520003DAD4EAD5FAD289724966CAD7DAD8EAD13
:10D530009FAD24970F94ACD118166CF42091BC18B1
:10D540003091BD184091BE185091BF186D857E85F1
:10D550008F85988906C029A93AA94BA95CA9B4016D
:10D56000C5010F944BCF4B015C019B01AC0162964E
:10D570006CAD7DAD8EAD9FAD62970F94ACC89B0135
:10D58000AC016091C8187091C9188091CA18909127
:10D59000CB180F944CCF698F7A8F8B8F9C8FA501FE
:10D5A000940168966CAD7DAD8EAD9FAD68970F947C
:10D5B000ACC82091C4183091C5184091C61850913C
:10D5C000C7180F944CCF14C08091DC189091DD18CF
:10D5D000A091DE18B091DF18898F9A8FAB8FBC8F26
:10D5E0006091D8187091D9188091DA189091DB1851
:10D5F00019821A821B821C82A70196010F944CCFBC
:10D600006D837E838F839887DE0111966D01EFAC69
:10D610008E01035E1F4F9E01275E3F4FAE014B5FA1
:10D620005F4FBE01675F7F4FCE010D960E9491A7AD
:10D6300009CDE1E0F0E0FCAFEBAF20E030E0A90184
:10D64000C701B6010F9446C887FD02C01CAE1BAED1
:10D6500049A45AA4EBACFCAC4E0C5F1C2E960EAD4C
:10D660001FAD2E97012B09F058C1320149AC5AACBD
:10D670004E0C5F1C4614570409F4E8CC2DA93EA9B2
:10D68000620E731E162DF301FF271F3070F4EE0F8C
:10D69000FF1FEE0FFF1FE855F84C4591559165911E
:10D6A0007491F42FE52FCB0114C0BF01FF0F880B3D
:10D6B000990B0F944DC82EE63BED4EED51E40F94BF
:10D6C000ACC820E030E040EA50E40F944CCFF62F95
:10D6D000E72F2F2F3E2FAC012C966CAD7DAD8EAD7C
:10D6E0009FAD2C970F94ACC86C962CAD3DAD4EAD54
:10D6F0005FAD6C970F944CCF6D877E878F87988B2B
:10D700003FE06316710468F449A95AA94F305105E6
:10D7100040F4B301CE010D960F94DD806B017C01C6
:10D7200003C0C12CD12C760188ED98E10E9498B7F6
:10D73000A70196010F94ACC86B017C019B01AC0161
:10D740000F9499D2882319F0C12CD12C7601F301C2
:10D75000FF271F3068F4EE0FFF1FEE0FFF1FE85585
:10D76000F84C85919591A591B4914C015D0114C03F
:10D77000BF01FF0F880B990B0F944DC82EE63BEDB0
:10D780004EED51E40F94ACC820E030E040EA50E4A4
:10D790000F944CCF4B015C01C401D50189879A8756
:10D7A000AB87BC878091BC189091BD18A091BE1822
:10D7B000B091BF1889A79AA7ABA7BCA79C01AD01E0
:10D7C000B401C5010F9446C8882309F453CF2FEF45
:10D7D0003FEF4FE75FE76DA57EA58FA598A90F9452
:10D7E00099D281110DC02FEF3FEF4FE75FE76DA595
:10D7F0007EA58FA598A90F9446C818160CF456C09C
:10D8000028962CAD3DAD4EAD5FAD289724966CADFE
:10D810007DAD8EAD9FAD24970F94ACD118163CF41E
:10D8200029A53AA54BA55CA5B401C5010CC0209162
:10D83000C0183091C1184091C2185091C3186D851D
:10D840007E858F8598890F944BCF4B015C019B019E
:10D85000AC0162966CAD7DAD8EAD9FAD62970F94BD
:10D86000ACC89B01AC016091C8187091C918809137
:10D87000CA189091CB180F944CCF698F7A8F8B8FE9
:10D880009C8FA501940168966CAD7DAD8EAD9FAD6A
:10D8900068970F94ACC82091C4183091C518409176
:10D8A000C6185091C7180F944CCF14C08091DC1843
:10D8B0009091DD18A091DE18B091DF18898F9A8FB2
:10D8C000AB8FBC8F6091D8187091D9188091DA18FD
:10D8D0009091DB1819821A821B821C82A701960183
:10D8E0000F944CCF6D837E838F839887DE011196D2
:10D8F0006D01EFAC8E01035E1F4F9E01275E3F4F0F
:10D90000AE014B5F5F4FBE01635F7F4FCE01099653
:10D910000E9491A78111AECE99CB29A93AA92219CB
:10D92000330989A59AA5E9ADFAAD8E1B9F0B97FF28
:10D9300003C09195819591099AA789A7C90137FFDD
:10D9400003C09195819591096E969FAF8EAF6E97AA
:10D9500064966EAC7FAC6497E9A8FAA86E0C7F1C45
:10D9600009A51AA5012B39F46E962EAD3FAD6E9721
:10D97000232B09F46BCB8DA9840DE82FF0E08F30B9
:10D9800068F4EE0FFF1FEE0FFF1FE855F84C85916E
:10D990009591A591B4916C017D0114C0BF01FF0F59
:10D9A000880B990B0F944DC82EE63BED4EED51E4DC
:10D9B0000F94ACC820E030E040EA50E40F944CCF24
:10D9C0006B017C01C601D7018D8B9E8BAF8BB88F0D
:10D9D0002D968FAD2D97860DE82FF0E08F3068F4EF
:10D9E000EE0FFF1FEE0FFF1FE859F84C8591959140
:10D9F000A591B4915C018D0114C0BF01FF0F880B8C
:10DA0000990B0F944DC82EE63BED4EED51E40F946B
:10DA1000ACC820E030E040EA50E40F944CCF5B010A
:10DA20008C01C501D801898B9A8BAB8BBC8B96017D
:10DA3000A7012C966CAD7DAD8EAD9FAD2C970F944C
:10DA4000ACC86C962CAD3DAD4EAD5FAD6C970F94F0
:10DA50004CCF6D877E878F87988B6C962CAD3DADB4
:10DA60004EAD5FAD6C97B501C8010F944BCF2C96AE
:10DA70002CAD3DAD4EAD5FAD2C970F9446D09B01C4
:10DA8000AC0169877A878B879C8701E010E0B6013B
:10DA9000C7010F9446C887FD02C000E010E04BADFF
:10DAA0005CAD0417150709F0E4C02E968EAD9FAD4E
:10DAB0002E97680E791EB201641B750B6F307105CD
:10DAC00060F49FE06916710440F4A301CE01099649
:10DAD0000F9468816B017C0103C0C12CD12C7601AD
:10DAE00088ED98E10E9498B7A70196010F94ACC801
:10DAF0006B017C019B01AC010F9499D2882319F032
:10DB0000C12CD12C76012FEF3FEF4FE75FE76DA5DA
:10DB10007EA58FA598A90F9499D281110DC02FEFE2
:10DB20003FEF4FE75FE76DA57EA58FA598A90F94FE
:10DB300046C818160CF45CC028962CAD3DAD4EAD11
:10DB40005FAD289724966CAD7DAD8EAD9FAD2497CB
:10DB50000F94ACD118166CF42091BC183091BD18FC
:10DB60004091BE185091BF1869857A858B859C8538
:10DB70000CC02091C0183091C1184091C21850912A
:10DB8000C31869897A898B899C890F944BCF4B0183
:10DB90005C019B01AC0162966CAD7DAD8EAD9FAD1D
:10DBA00062970F94ACC89B01AC016091C81870914A
:10DBB000C9188091CA189091CB180F944CCF698FD7
:10DBC0007A8F8B8F9C8FA501940168966CAD7DAD8B
:10DBD0008EAD9FAD68970F94ACC82091C41830915A
:10DBE000C5184091C6185091C7180F944CCF14C057
:10DBF0008091DC189091DD18A091DE18B091DF18AB
:10DC0000898F9A8FAB8FBC8F6091D8187091D9187B
:10DC10008091DA189091DB1819821A821B821C827B
:10DC2000A70196010F944CCF6D837E838F839887D5
:10DC3000DE0111966D01EFAC8E01035E1F4F9E0158
:10DC4000275E3F4FAE014B5F5F4FBE016F5E7F4F60
:10DC5000CE0109960E9491A7882309F4F7C96E9610
:10DC6000EEADFFAD6E9731976E96FFAFEEAF6E974C
:10DC7000E1C02DA93EA9420E531E3FE043165104B8
:10DC800090F4A30164968EAD9FAD6497481B590B29
:10DC90004F30510540F4B201CE010D960F94DD8056
:10DCA0006B017C0103C0C12CD12C760188ED98E179
:10DCB0000E9498B7A70196010F94ACC86B017C0134
:10DCC0009B01AC010F9499D2882319F0C12CD12C5F
:10DCD00076012FEF3FEF4FE75FE76DA57EA58FA59C
:10DCE00098A90F9499D281110DC02FEF3FEF4FE704
:10DCF0005FE76DA57EA58FA598A90F9446C8181655
:10DD00000CF45CC028962CAD3DAD4EAD5FAD2897B0
:10DD100024966CAD7DAD8EAD9FAD24970F94ACD1A4
:10DD200018166CF42091BC183091BD184091BE18A3
:10DD30005091BF186D897E898F89988D0CC0209174
:10DD4000C0183091C1184091C2185091C3186D8508
:10DD50007E858F8598890F944BCF4B015C019B0189
:10DD6000AC0162966CAD7DAD8EAD9FAD62970F94A8
:10DD7000ACC89B01AC016091C8187091C918809122
:10DD8000CA189091CB180F944CCF698F7A8F8B8FD4
:10DD90009C8FA501940168966CAD7DAD8EAD9FAD55
:10DDA00068970F94ACC82091C4183091C518409161
:10DDB000C6185091C7180F944CCF14C08091DC182E
:10DDC0009091DD18A091DE18B091DF18898F9A8F9D
:10DDD000AB8FBC8F6091D8187091D9188091DA18E8
:10DDE0009091DB1819821A821B821C82A70196016E
:10DDF0000F944CCF6D837E838F839887DE011196BD
:10DE00006D01EFAC8E01035E1F4F9E01275E3F4FF9
:10DE1000AE014B5F5F4FBE01635F7F4FCE01459602
:10DE20000E9491A7882309F411C9E9A5FAA53197A1
:10DE3000FAA7E9A7319609F093CD08C92091D41823
:10DE40003091D5184091D6185091D7186091C018CC
:10DE50007091C1188091C2189091C3180F9446C850
:10DE6000811109C930C0B801110F880B990B0F94AB
:10DE70004DC82091090230910A0240910B02509145
:10DE80000C020F94ACC82AE037ED43E25CE30F9438
:10DE9000ACC86D837E838F83988719821A821B8218
:10DEA0001C829E012F5F3F4F6901EFAC8E010B5F1B
:10DEB0001F4F2CED38E148ED58E164ED78E180ED3D
:10DEC00098E10E9491A70E94D29910C019821A82EB
:10DED0001B821C828090D8189090D918A090DA18D4
:10DEE000B090DB18C12CD12C7601F0C9C15ADF4F9C
:10DEF0000FB6F894DEBF0FBECDBFDF91CF911F915B
:10DF00000F91FF90EF90DF90CF90BF90AF909F90D8
:10DF10008F907F906F905F904F903F902F900895DB
:10DF20002F923F924F925F926F927F928F929F9229
:10DF3000AF92BF92CF92DF92EF92FF920F931F9317
:10DF4000CF93DF9300D01F92CDB7DEB78A830E94B4
:10DF5000CAC40F94257D6B017C0180911B10811137
:10DF60006DC080910D02882309F468C08091261845
:10DF7000882309F463C04091BF045091C0046091AC
:10DF8000C1047091C20497018601041B150B260B76
:10DF9000370B37FD66C0833019F134F481300CF44F
:10DFA0004DC0E4E0F8E506C0843009F047C0E4E085
:10DFB000F8E52EC084918F010F5F1F4F882321F059
:10DFC0000F941E14F801F6CFECEAFCE084918F0167
:10DFD0000F5F1F4F882391F10F941E14F801F6CFA5
:10DFE000E4E0F8E584918F010F5F1F4F882321F053
:10DFF0000F941E14F801F6CFE5E9FCE084918F013F
:10E000000F5F1F4F8823D1F00F941E14F801F6CF35
:10E0100084918F010F5F1F4F882321F00F941E14EE
:10E02000F801F6CFEDE7FCE084918F010F5F1F4F01
:10E03000882321F00F941E14F801F6CF20910D02D1
:10E0400030E0A8EEB3E00F9400CFC60ED71EE81E56
:10E05000F91EC092BF04D092C004E092C104F092B5
:10E06000C20480912C13811104C08091D50F81309E
:10E0700071F580914818882339F0813049F429B12D
:10E0800028272170298304C010B1109511701983BD
:10E090000981002341F0809128188F5F8093281810
:10E0A000863020F414C01092281811C080912718CF
:10E0B00081110DC081E0809327188AE29DE0909342
:10E0C0000D1880930C180F94EE100E94ECB68091FE
:10E0D000EA17843010F40F9451150F94257D6B01CD
:10E0E0007C014091B1045091B2046091B3047091ED
:10E0F000B404411551056105710589F18091AD04A4
:10E100009091AE04A091AF04B091B004840F951F1C
:10E11000A61FB71FA7019601281B390B4A0B5B0BE3
:10E1200057FD1DC0E5EDF7E584918F010F5F1F4F8F
:10E130001B830A83882329F00F941E14EA81FB8134
:10E14000F3CF609117187091181880EF9CE00F942E
:10E150008E238AE00F941E1487EE9CE096C04091B7
:10E160000E0250910F026091100270911102411540
:10E1700051056105710509F451C0909176128091A5
:10E180007712981749F0C092AD04D092AE04E09295
:10E19000AF04F092B00442C08091311281113EC0B0
:10E1A0001A8111113BC08091AD049091AE04A091F1
:10E1B000AF04B091B004840F951FA61FB71FA7012D
:10E1C0009601281B390B4A0B5B0B57FD27C05F9A42
:10E1D00080910B0180958072809309018091531684
:10E1E0008E7F809353168A9A809153168D7F8093E9
:10E1F000531680910801809581708093060180916B
:10E2000053168B7F809353160E94B4638091C90587
:10E21000882321F010924A181092C9058091CF04EA
:10E220009091D004909902C0019604C01816190666
:10E230002CF401979093D0048093CF048091CF0465
:10E240009091D0048E3E924014F1E5EDF7E5849173
:10E250008F010F5F1F4F1B830A83882329F00F94C0
:10E260001E14EA81FB81F3CFE7ECFCE084918F017F
:10E270000F5F1F4F1B830A83882329F00F941E14FE
:10E28000EA81FB81F3CF8EEB9CE00E94D663809104
:10E29000A9049091AA04A091AB04B091AC0400979A
:10E2A000A105B10581F0C81AD90AEA0AFB0A18EEDD
:10E2B000C11A13E0D10AE108F108F7FC04C080910B
:10E2C00080028111FFC1909176128091771298138C
:10E2D00007C00091EB170A831091ED1719831CC03A
:10E2E000E09177128FE48E9FF0011124E152F54FF7
:10E2F00000810A83E09177128E9FF0011124EF5183
:10E30000F54F1081198380917712909176129817AA
:10E3100019F08F5F8F70F9CF0A81002349F10F94B4
:10E32000257D0091C7041091C8042091C904309143
:10E33000CA04DC01CB01011511052105310579F471
:10E340008C599F4FAF4FBF4F8093C7049093C80421
:10E35000A093C904B093CA041FEF1A8311C0801B95
:10E36000910BA20BB30BB7FF0BC00FEF0A8308C0D2
:10E370001092C7041092C8041092C9041092CA04E3
:10E380001981112349F10F94257D0091CB0410913F
:10E39000CC042091CD043091CE04DC01CB010115D9
:10E3A00011052105310579F48C599F4FAF4FBF4FAF
:10E3B0008093CB049093CC04A093CD04B093CE046F
:10E3C0000FEF098311C0801B910BA20BB30BB7FF9A
:10E3D0000BC01FEF198308C01092CB041092CC041D
:10E3E0001092CD041092CE040A81602F70E089E073
:10E3F0000F94F2AC1981612F70E08CE00F94F2ACB5
:10E4000080918609882309F4FAC000915D02109179
:10E410005E0220915F022C83309160023A8360910A
:10E420004418709145186E5F7F4F072E000C880BC3
:10E43000990B0F944DC898014C815A810F9446C88E
:10E4400087FDDDC0F0907712212C312CE12C198250
:10E45000809176128F1509F460C08F2D90E04FE403
:10E46000489FF001499FF00D1124E856F54F45896A
:10E4700056896789708D452B462B472B81F4418D3A
:10E48000528D638D748D452B462B472B41F4458D62
:10E49000568D678D70A1452B462B472BC9F15FE444
:10E4A000589F9001599F300D1124B9016856754F3E
:10E4B0006B01FB0161817281838194810F944AD247
:10E4C0004B015C01F60161A172A183A194A10F949B
:10E4D0004BC82B013C01F60165A176A187A190A54F
:10E4E0000F944BC89B01AC01C301B2010F9446D0FD
:10E4F000A50194010F94ACC85B016C0191014E2DF4
:10E5000059810F94ACD118161CF41501EC2CD9824A
:10E5100081E08F0D8F70F82E9BCF209155023091A6
:10E5200056024091570250915802B1018E2D9981A7
:10E530000F94ACC898014C815A810F944CCF6B0159
:10E540007C019B01AC01B8018C819A810F94ACD104
:10E550001816B4F00091590210915A02F0915B0222
:10E56000FC8320915C022A8398014F2F5A81B601C7
:10E57000C7010F94ACD118161CF08601EC82FA8208
:10E58000C090C304D090C404E090C504F090C604C9
:10E5900098014C815A81C701B6010F94ACD118166D
:10E5A000D4F420E037ED43EA5CE3B8018C819A8132
:10E5B0000F94ACC84B015C0128E431EE4AE75FE3FD
:10E5C000C701B6010F94ACC8A50194010F944CCFBC
:10E5D0008B018C839A83C801AC81BA818093C30478
:10E5E0009093C404A093C504B093C604B801CD01B0
:10E5F0000F94B8D0DC01CB0160E00E9474980F94B6
:10E60000FFA48CE093E10F94320D80911B108111D7
:10E6100086C00091BE040983002391F00F94257DEC
:10E620000091BA041091BB042091BC043091BD0448
:10E63000DC01CB01801B910BA20BB30BB7FF52C0C7
:10E640000F94257D6B017C012091B904222309F4EC
:10E6500066C08091B5049091B604A091B704B091C2
:10E66000B804B701A601481B590B6A0B7B0B77FD59
:10E6700056C030E0A8EEB3E00F9400CFC60ED71E10
:10E68000E81EF91EC092B504D092B604E092B70419
:10E69000F092B8040F900F900F900F90DF91CF91F0
:10E6A0001F910F91FF90EF90DF90CF90BF90AF90B0
:10E6B0009F908F907F906F905F904F903F902F90A2
:10E6C0000D940B518FEF9FEFDC018093A904909381
:10E6D000AA04A093AB04B093AC040E948B980E9450
:10E6E0003A64F1CD0F94257D6B017C010981202FC7
:10E6F00030E0A8EEB3E00F9400CFC60ED71EE81EA0
:10E70000F91EC092BA04D092BB04E092BC04F0920D
:10E71000BD040F947E438AE00F941E1491CF0F9096
:10E720000F900F900F90DF91CF911F910F91FF905D
:10E73000EF90DF90CF90BF90AF909F908F907F90A1
:10E740006F905F904F903F902F9008952F923F923F
:10E750004F925F926F927F928F929F92AF92BF92F1
:10E76000CF92DF92EF92FF920F931F93CF93DF939D
:10E77000CDB7DEB7C655D1090FB6F894DEBF0FBED0
:10E78000CDBF1C0123967FAF6EAF2397142FDB0103
:10E790008D909D90AD90BC901397A5019401505819
:10E7A0002DA73EA74FA758AB1496CD90DD90ED90C6
:10E7B000FC901797D701C601B0588DA39EA3AFA3B5
:10E7C000B8A7CA01B9010F94ACC82B013C012DA117
:10E7D0003EA14FA158A5CA01B9010F94ACC89B0135
:10E7E000AC01C301B2010F944CCF0F944AD22796CB
:10E7F0006CAF7DAF8EAF9FAF27972091BC18309143
:10E80000BD184091BE185091BF1829AB3AAB4BAB25
:10E810005CABC501B4010F944CCF2B966CAF7DAFB0
:10E820008EAF9FAF2B978091C0189091C118A09187
:10E83000C218B091C3188DAB9EABAFABB8AF9C0103
:10E84000AD01C701B6010F944CCF2F966CAF7DAFD1
:10E850008EAF9FAF2F97D1012D913D914D915C913E
:10E8600029AF3AAF4BAF5CAF2B962CAD3DAD4EAD63
:10E870005FAD2B9769AD7AAD8BAD9CAD0F944BCF4F
:10E880006B017C01D10114962D913D914D915C91CC
:10E89000179721962CAF3DAF4EAF5FAF21972F96C4
:10E8A0002CAD3DAD4EAD5FAD2F9721966CAD7DADDE
:10E8B0008EAD9FAD21970F944BCF4B015C01209102
:10E8C000C4183091C5184091C6185091C718639666
:10E8D0002CAF3DAF4EAF5FAF6397D10118966D91EE
:10E8E0007D918D919C911B970F944BCF69A77AA72F
:10E8F0008BA79CA7A70196016DA57EA58FA598A9BA
:10E900000F94ACC82B013C01A50194016DA17EA11F
:10E910008FA198A50F94ACC89B01AC01C301B201B3
:10E920000F944CCF2B013C01A50194016DA57EA550
:10E930008FA598A90F94ACC84B015C01A701960163
:10E940006DA17EA18FA198A50F94ACC89B01AC01CD
:10E95000C501B4010F944BCFA30192010F94CBCF0B
:10E960004B015C0120E030E0A9010F9446C887FF0D
:10E970000AC02BED3FE049EC50E4C501B4010F940F
:10E980004CCF4B015C01112351F02BED3FE049ECE2
:10E9900050E4C501B4010F944BCF4B015C0120E062
:10E9A00030E0A901C501B4010F9446C8811122C00D
:10E9B00029AD3AAD4BAD5CAD69A97AA98BA99CA9EB
:10E9C0000F9446C8811116C021962CAD3DAD4EADB9
:10E9D0005FAD21976DA97EA98FA998AD0F9446C808
:10E9E000811108C08BED882E8FE0982E89ECA82E1F
:10E9F00080E4B82E27962CAD3DAD4EAD5FAD279788
:10EA0000C501B4010F94ACC86B017C0120E030E07B
:10EA1000A90169A57AA58BA59CA50F9446C8882352
:10EA2000D9F0A7019601C701B6010F94ACC86B01DC
:10EA30007C0129A53AA54BA55CA5CA01B9010F9493
:10EA4000ACC89B01AC01C701B6010F944CCF0F9429
:10EA50004AD26B017C010DC020E030E0A901C70162
:10EA6000B6010F94ACD187FF04C0F7FAF094F7F821
:10EA7000F0942FE632E143E85AE3C701B6010F9460
:10EA800046C887FD60C2C701B6010F94EED00F944F
:10EA9000BFD07AAB69ABFB01EF2B21F421E030E072
:10EAA0003AAB29AB4090C8185090C9186090CA186A
:10EAB0007090CB1849A95AA9BA0180E090E00F9450
:10EAC0004BC86B017C019B01AC01C501B4010F94E3
:10EAD00046D04B015C01A701960169A57AA58BA5DB
:10EAE0009CA50F9446D027966CAF7DAF8EAF9FAF9D
:10EAF0002797A3019201D1011C966D917D918D9173
:10EB00009C911F970F944BCFA70196010F9446D06D
:10EB100067966CAF7DAF8EAF9FAF6797A5019401ED
:10EB2000C501B4010F94ACC820E030E040E05FE3E1
:10EB30000F94ACC89B01AC0160E070E080E89FE3FB
:10EB40000F944BCF21966CAF7DAF8EAF9FAF2197C7
:10EB500063962CAD3DAD4EAD5FAD639729873A8787
:10EB60004B875C874D865E866F86788A60913A0215
:10EB700070913B02072E000C880B990B0F944DC827
:10EB80002091090230910A0240910B0250910C022F
:10EB90000F94ACC82AE037ED43E25CE30F94ACC8B5
:10EBA00069A37AA38BA39CA30F94257D9B01AC0141
:10EBB00028533F4F4F4F5F4F29AF3AAF4BAF5CAF3A
:10EBC00041E050E05EAB4DAB59E159A789A99AA944
:10EBD000ADA9BEA98A179B0709F469C10F94FFA4C8
:10EBE0000F94257DDC01CB0129AD3AAD4BAD5CAD79
:10EBF000821B930BA40BB50BB7FD0FC00F94257DA3
:10EC00009B01AC0128533F4F4F4F5F4F29AF3AAFA5
:10EC10004BAF5CAF80E00E94906F39A5315039A7AF
:10EC2000332309F443C021962CAD3DAD4EAD5FAD0D
:10EC300021976DA17EA18FA198A50F94ACC86B01FF
:10EC40007C01A50194016DA57EA58FA598A90F94BF
:10EC5000ACC8A70196010F944CCF6B017C012196A3
:10EC60002CAD3DAD4EAD5FAD21976DA57EA58FA5B9
:10EC700098A90F94ACC82B013C01A50194016DA18A
:10EC80007EA18FA198A50F94ACC89B01AC01C301D4
:10EC9000B2010F944BCF6DA77EA78FA798ABC6018B
:10ECA000D7018DA39EA3AFA3B8A76EC04DA95EA93F
:10ECB000BA0180E090E00F944BC8A50194010F9435
:10ECC000ACC86B017C010F9441D02B013C01C70102
:10ECD000B6010F943CD26DA37EA38FA398A7239671
:10ECE000AEADBFAD2397CD90DD90ED90FC90139726
:10ECF000F7FAF094F7F8F09414962D913D914D9118
:10ED00005C91179729A73AA74BA75CA7A701960183
:10ED1000C301B2010F94ACC86DA77EA78FA798ABB3
:10ED200029A53AA54BA55CA56DA17EA18FA198A5AB
:10ED30000F94ACC89B01AC016DA57EA58FA598A9C9
:10ED40000F944CCF6DA77EA78FA798ABA701960114
:10ED50006DA17EA18FA198A50F94ACC86B017C0119
:10ED600029A53AA54BA55CA5C301B2010F94ACC877
:10ED70009B01AC01C701B6010F944BCF6DA37EA3DD
:10ED80008FA398A7B9E1B9A72B962CAD3DAD4EAD99
:10ED90005FAD2B976DA57EA58FA598A90F944CCF3D
:10EDA00069837A838B839C832F962CAD3DAD4EADCA
:10EDB0005FAD2F976DA17EA18FA198A50F944CCF29
:10EDC0006D837E838F83988727962CAD3DAD4EADA6
:10EDD0005FAD279769857A858B859C850F944CCF8D
:10EDE00069877A878B879C8767962CAD3DAD4EAD42
:10EDF0005FAD67976D857E858F8598890F944CCF21
:10EE00006D877E878F87988B80912D02882321F0D4
:10EE1000CE0101960E94086289819A81AB81BC81F2
:10EE2000898B9A8BAB8BBC8B8D819E81AF81B88592
:10EE30008D8B9E8BAF8BB88F89859A85AB85BC8572
:10EE4000898F9A8FAB8FBC8F8091A318882351F044
:10EE5000AE01475E5F4FBE016B5E7F4FCE014196B4
:10EE60000F94A92320E030E040E85FE32D8F3E8F30
:10EE70004F8F58A3AE01435E5F4F6A01E090481880
:10EE80008E010F5D1F4F9E01235F3F4F445051097C
:10EE9000BE016B5E7F4FCE0141960E9491A78823F1
:10EEA00031F08DA99EA901969EAB8DAB8FCEF1015D
:10EEB00080819181A281B381898B9A8BAB8BBC8B32
:10EEC00084819581A681B7818D8B9E8BAF8BB88F06
:10EED00080859185A285B385898F9A8FAB8FBC8FF2
:10EEE0008091A318882351F0AE01475E5F4FBE01A9
:10EEF0006B5E7F4FCE0141960F94A92380E090E096
:10EF0000A0E8BFE38D8F9E8FAF8FB8A39101245FE0
:10EF10003F4FAE01435E5F4F6A01E09048188E019B
:10EF20000F5D1F4F44505109BE016B5E7F4FCE01F4
:10EF300041960E9491A780E1F101ACEBB8E101900C
:10EF40000D928A95E1F7CA5ADF4F0FB6F894DEBFEB
:10EF50000FBECDBFDF91CF911F910F91FF90EF902A
:10EF6000DF90CF90BF90AF909F908F907F906F90E9
:10EF70005F904F903F902F9008951F93CF93DF9312
:10EF8000CDB7DEB728970FB6F894DEBF0FBECDBF62
:10EF900069837A838B839C832D833E834F83588739
:10EFA00081E00F942514882311F081E02BC0BE016D
:10EFB0006B5F7F4FCE0101960F94D70E809168163C
:10EFC000182F147082FF05C080E00F942514811162
:10EFD000ECCF109268160F94DDB480915609909191
:10EFE0005709A0915809B09159098093C41890937A
:10EFF000C518A093C618B093C7180F944E1181E09E
:10F00000111180E028960FB6F894DEBF0FBECDBF79
:10F01000DF91CF911F9108956F927F928F929F926F
:10F02000AF92BF92EF92FF920F931F93CF93DF9314
:10F0300000D01F92CDB7DEB7B82E662351F01092E4
:10F04000D5041092D1041092D2041092D3041092DD
:10F05000D4040F94257D0091D1041091D204209105
:10F06000D3043091D4043B014C01601A710A820A26
:10F07000930A97FC4BC01091D504B7FC16C02B2DFA
:10F080000B2C000C330B2C5F3F4F412F012E000C3B
:10F09000550B24173507D4F11B153CF034EF832EA4
:10F0A00099249394A12CB12C06C028EE822E23E043
:10F0B000922EA12CB12CDC01CB01880D991DAA1D2B
:10F0C000BB1D8093D1049093D204A093D304B0933A
:10F0D000D40410FBEE24E0F8F12C24E22E9DC001B4
:10F0E0002F9D900D9E19112480599C4F9C838B83DA
:10F0F00082E390E09A838983BE016D5F7F4FCE01EA
:10F1000001960F94D7501F5F1093D5040F900F9066
:10F110000F900F90DF91CF911F910F91FF90EF9083
:10F12000BF90AF909F908F907F906F900895AF9217
:10F13000BF92CF92DF92EF920F931F93CF93DF9303
:10F1400000D01F92CDB7DEB75C018B010E948B9877
:10F15000E090481880EDC82E88E1D82E84E0E89E23
:10F16000F0011124E25DFD4F208131814281538104
:10F17000F50160817181828193810F9446D0F601FF
:10F1800024853585468557850F944CCFF6016487D5
:10F1900075878687978719821A821B821C82CE0107
:10F1A00001966C012CED38E148ED58E164ED78E111
:10F1B000CF010E9491A70E94D2990E94ECB60F90B5
:10F1C0000F900F900F90DF91CF911F910F91EF90C3
:10F1D000DF90CF90BF90AF9008959F92AF92BF9273
:10F1E000CF92DF92EF92FF920F931F93CF93DF9313
:10F1F00081E6A82E83E0B82E00ED18E1CCEBD8E133
:10F200009BE9C92E95E0D92E22E9E22E24E0F22EC8
:10F21000912CF50181915F010E941098882309F1DA
:10F220000E94D997F7012081211104C020919604F2
:10F23000222339F0288139814A815B810F944CCF98
:10F240000AC0F3E09F1639F0F60120813181428136
:10F2500053810F944BCFF801608371838283938332
:10F2600009C088819981AA81BB81F801808391833B
:10F27000A283B38393940C5F1F4F2496F4E0CF0EC8
:10F28000D11C2FEFE21AF20A84E09812C2CF86E472
:10F290000E9459988823C9F00E94D99720E030E055
:10F2A000A9010F94ACD1181684F40E94D99720E0DC
:10F2B00030E040E752E40F9446D060930902709327
:10F2C0000A0280930B0290930C02DF91CF911F9161
:10F2D0000F91FF90EF90DF90CF90BF90AF909F90F5
:10F2E00008952F923F924F925F926F927F929F92DA
:10F2F000AF92BF92CF92DF92EF92FF920F931F9344
:10F30000CF93DF93CDB7DEB728970FB6F894DEBF63
:10F310000FBECDBF1A012B01922EF32EC82ED12C79
:10F32000811108C080914818811102C0EFEF06C01A
:10F33000E1E004C0F601E953F44FE491AA24A39458
:10F340001E160CF4A12CBB24B39420E030E0A901DC
:10F35000C201B1010F94ACD118160CF0B12CCC0C39
:10F36000DD1CCC0CDD1CC6018454974E3C01FC0115
:10F3700010821182128213820F944E11F3012082A7
:10F38000318242825382E090481820E030E0A901A7
:10F39000B801892D9F2D0F9446C881110AC0F6012E
:10F3A000E658F44F85919591A591B4918C019A2ED0
:10F3B000FB2EC801A92DBF2D8D839E83AF83B887F7
:10F3C00019821A821B821C82CE0101966C018E0169
:10F3D0000B5F1F4F28EC38E144EC58E160EC78E11A
:10F3E0008CEB98E10E9491A70E94ECB6AB100F94B1
:10F3F000175928960FB6F894DEBF0FBECDBFDF9128
:10F40000CF911F910F91FF90EF90DF90CF90BF9021
:10F41000AF909F907F906F905F904F903F902F9014
:10F4200008959091A318981709F440C00E94ECB673
:10F430008091A3188823E9F060EC78E18CEB98E1E7
:10F440000F9484119B01AC016091C4187091C51890
:10F450008091C6189091C7180F944CCF6093C41830
:10F460007093C5188093C6189093C7181092A3186C
:10F47000089581E08093A31860EC78E18CEB98E12B
:10F480000F9484119B01AC016091C4187091C51850
:10F490008091C6189091C7180F944BCF6093C418F1
:10F4A0007093C5188093C6189093C71808952F922B
:10F4B0003F924F925F926F927F928F929F92AF9204
:10F4C000BF92CF92DF92EF92FF920F931F93CF9351
:10F4D000DF93CDB7DEB76B970FB6F894DEBF0FBEE4
:10F4E000CDBF182F809153168770873069F48FE451
:10F4F0000E945998882319F00E94C99703C08FE48D
:10F500000E94109881111EC20E94ECB62091A3188F
:10F510002A8F80E00E94117A80EA90E00F947F0D9C
:10F5200080E00F942514309148183B8F21E040E093
:10F5300050E0BA0180E00F94A6691092890F0F94F1
:10F54000A30D81E08093521611111BC088E50E9423
:10F550001098382E89E50E941098282E8AE50E947E
:10F5600010988D8B311006C0211009C0811107C081
:10F57000322C0DC0222019F0322C0D8909C000E078
:10F5800007C0332433942224239421E02D8B01E0FF
:10F590000E948B9882E50E945998882361F00E940E
:10F5A000D9976B017C0120E030E0A9010F9446C897
:10F5B000882379F106C0C12CD12C80E8E82E80E4A4
:10F5C000F82E011105C0311003C0222009F440C1FA
:10F5D000C092D818D092D918E092DA18F092DB18BD
:10F5E000A70196016091C4187091C5188091C61842
:10F5F0009091C7180F9446C887FF0BC019821A82D2
:10F600001B821C82BE016F5F7F4F88ED98E10F94D3
:10F61000D70E011138C0311003C0211014C118C118
:10F62000211031C011E01093481880E00E94C96099
:10F630008091BC189091BD18A091BE18B091BF18D0
:10F640008093040290930502A0930602B0930702F0
:10F650001092481880E00E94C96080E1ECEBF8E16C
:10F66000A7E9B4E001900D928A95E1F71092A90400
:10F670001092AA041092AB041092AC041093A70449
:10F68000002359F2E0C01092C0181092C1181092D5
:10F69000C2181092C3181092BC181092BD18109284
:10F6A000BE181092BF180F944E1180914818811106
:10F6B00005C08FEF9FEF9F8B8E8B04C0A1E0B0E061
:10F6C000BF8BAE8BEBEBFBE0459055906590749053
:10F6D000EFEBFBE085909590A590B490A30192018B
:10F6E000C501B4010F9446C887FF05C0A30192016C
:10F6F000C501B40104C0A5019401C301B2010F9476
:10F7000046D06B017C01EEE7FBE085919591A591D8
:10F71000B4918D879E87AF87B88BEAE7FBE0859130
:10F720009591A591B491898B9A8BAB8BBC8B9C01E5
:10F73000AD016D857E858F8598890F94ACD11816A3
:10F7400044F01D859E85988FAF85A98FB889BD87A8
:10F7500007C019892A89288F3B89398F8C898D8721
:10F76000A7019601C701B6010F94ACC820E030E0B4
:10F7700040E85FE30F944CCF0F944AD2212F388D8D
:10F78000498D5D850F94ACC869877A878B879C8784
:10F79000E8ECFBE0149120E030E040EC5FE3C501D1
:10F7A000B4010F94ACC86B017C01612F110F770B72
:10F7B000880B990B0F944DC89B01AC01C701B60192
:10F7C0000F94ACC869837A838B839C8320E030E0FC
:10F7D00040EC5FE3C301B2010F94ACC86B017C0144
:10F7E000AE89BF89BD01BB0F880B990B0F944DC823
:10F7F0009B01AC01C701B6010F94ACC86D837E8339
:10F800008F839887AE01475F5F4FBE016F5F7F4F69
:10F81000CE0105960F94B50E0F9417591092C0188B
:10F820001092C1181092C2181092C3181092BC18EE
:10F830001092BD181092BE181092BF180111F2CE8E
:10F840003110F0CEEACE81E00E94C960011104C0FF
:10F85000BD89BB2309F45FC0809153168370833048
:10F86000F1F060E08BEA9DE00E9466C4E4E0F8E518
:10F8700084918F010F5F1F4F882321F00F941E1476
:10F88000F801F6CFECE9FDE084918F010F5F1F4F87
:10F89000882309F440C00F941E14F801F5CF0F948B
:10F8A0004E118091C4189091C518A091C618B091BE
:10F8B000C7188093D8189093D918A093DA18B093EA
:10F8C000DB1880E090E0AFE4B3E48093D01890932D
:10F8D000D118A093D218B093D31880E090E0A9E299
:10F8E000B3E48093D4189093D518A093D618B0930E
:10F8F000D7181092A70419821A821B821C82AE01AB
:10F900004F5F5F4F64ED78E180ED98E10F94B50EA5
:10F9100082E00E94C9600F944E118091511680932D
:10F9200052168A8D0E94117A0F948A0D21E040E0D0
:10F9300050E0BA018B8D0F94A66983E080937B021F
:10F940000F9476366B960FB6F894DEBF0FBECDBF20
:10F95000DF91CF911F910F91FF90EF90DF90CF90AB
:10F96000BF90AF909F908F907F906F905F904F90DF
:10F970003F902F90089581E00C94577ACF92DF92B8
:10F98000EF92FF920F931F93CF93DF93CDB7DEB724
:10F990002C970FB6F894DEBF0FBECDBF7B018C0154
:10F9A000D42E9B01AC016091E0157091E11580911E
:10F9B000E2159091E3150F9446C8882309F496C088
:10F9C000C090A31880E00E94117A20E030E0A901E5
:10F9D000B701C8010F94ACD1181624F0E12CF12C1A
:10F9E00000E010E0C701D8018093E0159093E11585
:10F9F000A093E215B093E3152DEB37E346E855EB02
:10FA0000B701C8010F94ACD187FD0AC02DEB37E3D5
:10FA100046E855E3B701C8010F9446C818164CF4E0
:10FA20009701A80160E070E080E89FE30F9446D062
:10FA300003C060E070E0CB01609317107093181062
:10FA40008093191090931A1080EF9FEFA9E7B4EC00
:10FA50008093131090931410A0931510B093161068
:10FA6000CC2009F443C08091BC189091BD18A0919E
:10FA7000BE18B091BF1889839A83AB83BC838091F1
:10FA8000C0189091C118A091C218B091C3188D836D
:10FA90009E83AF83B8878091C4189091C518A091B8
:10FAA000C618B091C71889879A87AB87BC8781E051
:10FAB0000E94117ADD20D1F04CE050E06CEB78E14F
:10FAC000CE0101960F94BED3892B81F02C960FB6F0
:10FAD000F894DEBF0FBECDBFDF91CF911F910F9184
:10FAE000FF90EF90DF90CF900D9476362C960FB666
:10FAF000F894DEBF0FBECDBFDF91CF911F910F9164
:10FB0000FF90EF90DF90CF9008952F923F924F9209
:10FB10005F926F927F928F929F92AF92BF92CF929D
:10FB2000DF92EF92FF920F931F93CF93DF93CDB7A6
:10FB3000DEB760970FB6F894DEBF0FBECDBF3C01B5
:10FB40007F876E874D87288BFC0120803180428023
:10FB50005380FB01C080D180E280F380C986DA86C1
:10FB6000EB86FC86002301F1A7019601C201B101D9
:10FB70000F944682882309F4A0C120E030E040E4DD
:10FB800050E4C201B1010F944CCF1B012C0120E0C5
:10FB900030E048EF51E4C701B6010F944BCF6987BD
:10FBA0007A878B879C870AC0AE01475F5F4FC2018F
:10FBB000B1010F940982882309F47FC1E090C41831
:10FBC000F090C5180091C6181091C71880900902CE
:10FBD00090900A02A0900B02B0900C0280916A02F1
:10FBE00090916B02A0916C02B0916D02809309021A
:10FBF00090930A02A0930B02B0930C0219821A820E
:10FC00001B821C8229853A854B855C85CE01019635
:10FC10006C01C201B1010F94C20D81E00F94F60E88
:10FC20008111C0C08091531682FF11C02091F40F42
:10FC30003091F50F4091F60F5091F70F60E070E0B2
:10FC400080E490EC0F944BCF1B012C0106C0212CBB
:10FC5000312C80E2482E81EC582E20E030E040E844
:10FC600050E4C201B1010E94BD77882329F060E011
:10FC700070E080EC9FE74FC0C090C418D090C518CA
:10FC8000E090C618F090C71880E090E0A0E8B0E4DB
:10FC900089839A83AB83BC8320E030E040EA50E460
:10FCA000C701B6010F944CCF6D837E838F839887F5
:10FCB000BE016F5F7F4FCE0105960F94D70E20E0F7
:10FCC00030E040E050E4C201B1010E94BD778111F3
:10FCD000CECF20E030E040E450E46091C418709151
:10FCE000C5188091C6189091C7180F94ACC81B0115
:10FCF0002C01A7019601C701B6010F944CCF9B01BF
:10FD0000AC01C201B1010F944CCF2DEC3CEC4CE4A2
:10FD10005EE30F94ACC82091F40F3091F50F409141
:10FD2000F60F5091F70F0F944CCF6B018C018D851E
:10FD30008250823050F580E090E0A0E8B0E48D83FE
:10FD40009E83AF83B8872091C4183091C518409125
:10FD5000C6185091C7189D85933029F060E070E077
:10FD600080EA90E404C060E070E088EC91E40F94D5
:10FD70004CCF69837A838B839C83BE016B5F7F4FFB
:10FD8000CE0101960F94D70E08C0ED85E13029F41D
:10FD900080E00F94F60E811105C0F889F33008F465
:10FDA0005DC008C0E889E33008F48CC0C12CD12CB8
:10FDB00000EC1FE7E4E9FDE084917F019FEFE91A81
:10FDC000F90A882321F00F941E14F701F5CF209132
:10FDD0009B0530919C0540919D0550919E05F30136
:10FDE00060817181828193810F944CCF43E00F94A5
:10FDF000B618EFE8FDE084917F019FEFE91AF90A58
:10FE0000882321F00F941E14F701F5CF20919F0550
:10FE10003091A0054091A1055091A205EE85FF8586
:10FE200060817181828193810F944CCF43E00F9464
:10FE3000B618EAE8FDE084917F019FEFE91AF90A1C
:10FE4000882321F00F941E14F701F5CF43E0B6018B
:10FE5000C8010F94B6188AE00F941E14809209020C
:10FE600090920A02A0920B02B0920C029601A80195
:10FE7000B601C8010F9499D2882389F160E08BE71D
:10FE80009DE00E9466C4E5EDF7E584917F019FEF58
:10FE9000E91AF90A882321F00F941E14F701F5CF0F
:10FEA000EBE6FDE084917F019FEFE91AF90A8823D0
:10FEB000B1F00F941E14F701F5CFC12CD12C00EC3A
:10FEC0001FE70DC08092090290920A02A0920B02D5
:10FED000B0920C02C12CD12C00EC1FE7CFCFB601A1
:10FEE000C80160960FB6F894DEBF0FBECDBFDF919C
:10FEF000CF911F910F91FF90EF90DF90CF90BF9027
:10FF0000AF909F908F907F906F905F904F903F90B9
:10FF10002F9008952F923F924F925F926F927F920F
:10FF20008F929F92AF92BF92CF92DF92EF92FF9209
:10FF30000F931F93CF93DF93CDB7DEB7EF970FB635
:10FF4000F894DEBF0FBECDBF2DB73EB73AAB29AB9D
:10FF500041E061E081E00F949F14811120C586E5A6
:10FF60000E945998882391F00E94B5978D8B853017
:10FF700080F0E7E4FFE084918F010F5F1F4F88233B
:10FF800009F40DC50F941E14F801F5CF31E03D8B37
:10FF900003C08D89882361F0E7E2FFE084918F013F
:10FFA0000F5F1F4F882321F00F941E14F801F6CF26
:10FFB00080E50E945998882321F00E94B597F82E79
:10FFC00002C0EAE0FE2E8CEF8F0D8F3268F0E3E086
:10FFD000FFE084918F010F5F1F4F882309F4DFC476
:10FFE0000F941E14F801F5CF85E40E9459988823D8
:10FFF00039F00E94C997882339F091E098A706C08C
:020000021000EC
:1000000085E40E941098F7CFA2E0A8A78090BC18C2
:100010009090BD18A090BE18B090BF188D829E829F
:10002000AF82B8868091C0189091C118A091C21873
:10003000B091C31889879A87AB87BC8788E50E94EF
:100040005998811109C020E030E040E450E4C50136
:10005000B4010F944BCF02C00E94D9976D877E8761
:100060008F87988B89849A84AB84BC8489E50E94AD
:100070005998811109C020E030E048EF51E4C501F2
:10008000B4010F944CCF02C00E94D9979B01AC01E0
:10009000698B7A8B8B8B9C8B6D857E858F85988900
:1000A0000F9446828EA381110DC0EBEEFEE0849189
:1000B0008F010F5F1F4F882309F471C40F941E1422
:1000C000F801F5CF8CE40E941098182F8823C1F016
:1000D0000E94B5978E8B803168F0E8EBFEE084914A
:1000E0008F010F5F1F4F882309F459C40F941E140A
:1000F000F801F5CFBE89B13021F422E02E8B01C08A
:100100001E8A83E50E945998882349F00E94C99766
:10011000882349F0111108C037E03E8B05C083E504
:100120000E941098F5CF1EA28D89833060F0EEE911
:10013000FEE084918F010F5F1F4F882321F00F9401
:100140001E14F801F6CF9091A3189DAF80E00E9495
:10015000117A0F94A30DAF2DB0E0B8AFAFAB2DB7B0
:100160003EB784E0F89E2019310911240FB6F894A7
:100170003EBF0FBE2DBFADB7BEB71196B8ABAFA790
:1001800001E02D8948A5BE016F5E7F4FCE010D961F
:100190000E94857D9B01AC010F9499D2811151C3BE
:1001A0000F94257D611571058105910511F00F945E
:1001B000A7C31DA299249394B3EFBB8F2FE42C8F78
:1001C00063EC362E77EC272E33EF3F8B8FE4888F4E
:1001D00093EC998FA7E4AA8F1D8E1E8E1F8E18A2F6
:1001E00019A21AA21BA21CA2BE898B2F90E09C010F
:1001F000215031093FAF2EAF9DA1892F90E09AA7E2
:1002000089A7AFA9B8AD8A179B070CF033C3BE8985
:10021000BB2309F4C2C10F9459C32AE030E040E087
:1002200050E00F94CECE0F944DC820E030E040EA6D
:1002300050E40F94ACD118161CF001E010E002C09D
:100240000FEF1FEF0F9459C328E631E040E050E074
:100250000F94CECE0F944DC82B013C010F9459C37F
:100260002DE230E040E050E00F94CECE6B5F7F4F48
:100270008F4F9F4F0F944DC86BA77CA78DA79EA74C
:100280002D89243051F01FA2C801110FAA0BBB0BFE
:1002900089AF9AAFABAFBCAF6AC04BA55CA56DA5EB
:1002A0007EA58CE89EE00F945923B301A20181E85A
:1002B0009EE00F945923E4E7FEE084917F019FEFD5
:1002C000E91AF90A882321F00F941E14F701F5CFDB
:1002D0000130110519F0E0E6FEE00DC0EBE6FEE0AE
:1002E00084917F01AFEFEA1AFA0A8823A1F30F94F1
:1002F0001E14F701F5CF84917F01BFEFEB1AFB0AC3
:10030000882309F4C0CF0F941E14F701F4CF4D8158
:100310005E816F81788583E59EE00F94592349853E
:100320005A856B857C8580E59EE00F94592340912A
:10033000C4185091C5186091C6187091C7188DE403
:100340009EE00F9459238AE00F941E1419821A829A
:100350001B821C82AE014F5F5F4FBE01675F7F4F04
:10036000CE0105960F94B50E8FA18F5F8FA32FA19D
:10037000822F90E0AEADBFAD8A179B070CF00DC188
:10038000BEA1BB2379F069AD7AAD8BAD9CAD0F9466
:100390004DC89B01AC010F944CCF20E030E040E908
:1003A00052E41AC00F9459C324E130E040E050E019
:1003B0000F94CECE675E7F4F8F4F9F4F0F944DC8E7
:1003C0006B017C0169AD7AAD8BAD9CAD0F944DC8CE
:1003D0009B01AC01C701B6010F94ACC89B01AC01F5
:1003E000C301B2010F944CCF2B013C0120E030E05F
:1003F00044EB53E40F94ACD118164CF420E030E0F9
:1004000044EB53E4C301B2010F944BCFEDCF20E096
:1004100030E0A901C301B2010F9446C887FF0BC0A9
:1004200020E030E044EB53E4C301B2010F944CCF21
:100430002B013C01ECCF2BED3FE049E450E4C3013C
:10044000B2010F94ACC820E030E044E353E40F94D1
:1004500046D04B015C010F9441D06BAB7CAB8DABB4
:100460009EAB20E030E040E450E46D857E858F85D2
:1004700098890F944CCF6B017C012BA93CA94DA905
:100480005EA96BA57CA58DA59EA50F94ACC89B010C
:10049000AC01C701B6010F944CCF6B017C01C501C3
:1004A000B4010F943CD26BAB7CAB8DAB9EAB20E028
:1004B00030E048EF51E469897A898B899C890F94EF
:1004C0004BCF4B015C012BA93CA94DA95EA96BA5A3
:1004D0007CA58DA59EA50F94ACC89B01AC01C50160
:1004E000B4010F944CCF4B015C0120E030E048E2B6
:1004F00052ECC701B6010F9446C887FD11C020E039
:1005000030E041EE53E4C701B6010F94ACD11816A8
:100510006CF4C12CD12C41EEE42E43E4F42E06C041
:10052000C12CD12C58E2E52E52ECF52ECD82DE8284
:10053000EF82F88620E030E0A901C501B4010F94F4
:1005400046C887FD11C020E030E048EC53E4C50107
:10055000B4010F94ACD1181654F4812C912C38ECC2
:10056000A32E33E4B32E03C0812C912C5401898631
:100570009A86AB86BC862D89243009F0E7CEE6E565
:10058000FEE084917F013FEFE31AF30A882309F428
:10059000BECE0F941E14F701F4CF01E020E048A571
:1005A000BE016F5E7F4FCE010D960E94857D5B017F
:1005B0007C01E9A5FAA5EE0FFF1FEE0FFF1FAFA507
:1005C000B8A9EA0FFB1FCB01D70180839183A283D7
:1005D000B383912C9501A701B501C7010F9499D25E
:1005E000811102C0992493949501A701B501C70117
:1005F0000F9499D281113EC110E0412C512C32014F
:10060000EFA5F8A9B4E01B9FE00DF11D1124208196
:10061000318142815381C301B2010F944CCF2B0130
:100620003C011F5F2DA1211758F709A51AA50F5FDF
:100630001F4FB801012E000C880B990B0F944DC869
:100640006D8F7E8F8F8F98A39B01AC01C301B20188
:100650000F9446D069A37AA38BA39CA39501A7010D
:100660006F89788D898D9A8D0F94ACD1181624F4EA
:10067000AF8AB88EE98EFA8E9501A7016B8D7C8DBD
:10068000832D922D0F9446C887FF04C0AB8EBC8E7D
:100690003E2C2F2CD12C412C512C3201EFA5F8A946
:1006A00034E0D39EE00DF11D112429A13AA14BA104
:1006B0005CA160817181828193810F944BCF9B01FA
:1006C000AC010F94ACC89B01AC01C301B2010F9403
:1006D0004CCF2B013C01D3948DA18D15F8F62D8DB7
:1006E0003E8D4F8D58A1C301B2010F9446D00F9497
:1006F0004AD26D8F7E8F8F8F98A38D8982508E37CF
:1007000008F09BC06AE070E0C8010F94A618E8E406
:10071000FEE084916F019FEFC91AD90A882321F066
:100720000F941E14F601F5CF6AE070E08FA998AD22
:100730000F94A618E2E4FEE084916F01AFEFCA1AAD
:10074000DA0A882321F00F941E14F601F5CF43E056
:10075000B501C7010F94B618BD89B23009F46AC05B
:10076000EAE3FEE084917F012FEFE21AF20A882388
:1007700021F00F941E14F701F5CF44E069A17AA18E
:100780008BA19CA10F94B618E1E3FEE084917F0158
:100790003FEFE31AF30A882321F00F941E14F701A8
:1007A000F5CF46E06D8D7E8D8F8D98A10F94B61894
:1007B000EAE2FEE084917F019FEFE91AF90A8823BB
:1007C00021F00F941E14F701F5CF43E06F89788D67
:1007D000898D9A8D0F94B618E3E2FEE084917F0133
:1007E000AFEFEA1AFA0A882321F00F941E14F701DA
:1007F000F5CF43E06B8D7C8D832D922D0F94B61831
:10080000EAE1FEE084917F01BFEFEB1AFB0A882347
:1008100021F00F941E14F701F5CF2F89388D498DE3
:100820005A8D6B8D7C8D832D922D0F944BCF43E091
:100830000F94B6188AE00F941E142DA12F5F2DA3DC
:10084000DBCC912C33EF3B8F8FE48C8F83EC382EF5
:1008500097EC292E93EF9F8BAFE4A88FB3ECB98F61
:1008600027E42A8F1D8E1E8E1F8E18A219A21AA28F
:100870001BA21CA280E00F94F60E992009F480C000
:10088000EFE0FEE084917F013FEFE31AF30A882353
:1008900021F00F941E14F701F5CF8D89882309F4F8
:1008A00056C0E8E0FEE084917F019FEFE91AF90A63
:1008B000882321F00F941E14F701F5CF46E069A1BB
:1008C0007AA18BA19CA10F94B618E1E0FEE084917F
:1008D0008F010F5F1F4F882321F00F941E14F80122
:1008E000F6CF43E06F89788D898D9A8D0F94B61875
:1008F000EAEFFDE084918F010F5F1F4F882321F005
:100900000F941E14F801F6CF43E06B8D7C8D832D80
:10091000922D0F94B618E1EFFDE084918F010F5FE7
:100920001F4F882321F00F941E14F801F6CF2F8952
:10093000388D498D5A8D6B8D7C8D832D922D0F9422
:100940004BCF43E00F94B6188AE00F941E14ECEDE1
:10095000FDE084918F010F5F1F4F882321F00F94DA
:100960001E14F801F6CF46E06D8D7E8D8F8D98A117
:100970000F94B6188AE00F941E148AE00F941E1488
:100980000F948A0D8DAD0E94117A0F947636A9A925
:10099000BAA90FB6F894BEBF0FBEADBF07C029A954
:1009A0003AA90FB6F8943EBF0FBE2DBF89A99AA9E8
:1009B0000FB6F8949EBF0FBE8DBFEF960FB6F8949A
:1009C000DEBF0FBECDBFDF91CF911F910F91FF9082
:1009D000EF90DF90CF90BF90AF909F908F907F90DF
:1009E0006F905F904F903F902F9008956F927F92FD
:1009F0008F929F92AF92BF92CF92DF92EF92FF922F
:100A00000F931F93CF93DF93CDB7DEB7EE970FB65B
:100A1000F894DEBF0FBECDBF0091F41A1091F51A05
:100A200082E08093D115F80101900020E9F7319719
:100A30005F01A01AB10AF801CF01801B910B8A1542
:100A40009B0534F480818F3209F410823196F4CF03
:100A500060E873E1CE0180960F94E051E12CF12C17
:100A60008DE4682E83E0782EEA14FB040CF09DC020
:100A7000F801EE0DFF1D8081811103C08FEFE81A90
:100A8000F80A6801CE0CDF1CF6018081882309F486
:100A90008CC0FFEFEF1AFF0AF801EE0DFF1D7F017A
:100AA000E01AF10A81918111FACFCE0184960E9459
:100AB0006E59BE01605E7F4FCE0101960F94E051EA
:100AC000A601BE016F5F7F4F80E090E00F949053CE
:100AD000CE0101960E94AC638FE20F941E148091A8
:100AE0003D13882319F08DE393E102C088E793E07A
:100AF0004C01F40181914F01882319F00F941E14C9
:100B0000F8CF80912E13882309F44FC01D821886D8
:100B10001C821B827A82698221E0A601BE016C5D83
:100B20007F4FCE0105960E94BB62811128C08AE0EA
:100B30000F941E14E4E0F8E584918F010F5F1F4FBE
:100B4000882321F00F941E14F801F6CFE9EBFDE0A5
:100B500084918F010F5F1F4F882321F00F941E1483
:100B6000F801F6CFF60181916F01882319F00F94F7
:100B70001E14F8CFCE0101960E94AC6316C0CE01C0
:100B800084960E9431598BE1FE013596DE019496E0
:100B900001900D928A95E1F78B819C819BA38AA39A
:100BA000CE0101960E94AC635FCF8AE00F941E14C1
:100BB000CE0180960E94AC63EE960FB6F894DEBF2D
:100BC0000FBECDBFDF91CF911F910F91FF90EF909E
:100BD000DF90CF90BF90AF909F908F907F906F905D
:100BE0000895CF93DF938B399240B1F0E5EDF7E5AF
:100BF0008491EF012196882321F00F941E14FE01A9
:100C0000F7CFE9E8FFE08491EF012196882331F0E6
:100C10000F941E14FE01F7CF80E001C081E0DF9148
:100C2000CF910895CF93DF931F92CDB7DEB769833D
:100C300041E050E0BE016F5F7F4F04960E946A5A08
:100C40000F90DF91CF9108958F929F92AF92BF92B4
:100C5000CF92DF92EF92FF920F93CF93DF931F9289
:100C6000CDB7DEB77C015B016A0149018091D604F2
:100C70008823E9F0F70180819181C80ED91ED182C5
:100C8000C08222C001111DC0BE016F5F7F4FC40131
:100C90000F94B399F70180819181019691838083AC
:100CA000FFEFAF1ABF0A81E0C81AD10869F0F70157
:100CB000808191810F9486CE89839091DA1591116C
:100CC000E1CFF5018083E0CF0F90DF91CF910F91BD
:100CD000FF90EF90DF90CF90BF90AF909F908F905C
:100CE00008957F928F929F92AF92BF92CF92DF92A0
:100CF000EF92FF920F931F93CF93DF931F92CDB785
:100D0000DEB7E091D604EE2341F0FC012081318171
:100D1000420F531F5183408349C069017C015B012D
:100D20008B01040F151FA016B10609F43FC0F7018F
:100D300080809180F50171905F017982C4010F94E8
:100D400086CE781631F1672DC4010F948ECEC40182
:100D50000F9486CE99818917E1F0E4E0F8E584915B
:100D60008F010F5F1F4F882321F00F941E14F8018D
:100D7000F6CFEFE6FFE084918F010F5F1F4F8823CE
:100D800021F00F941E14F801F6CF81E08093D60471
:100D90000DC0BE016F5F7F4FC6010F94B399F7017D
:100DA00080819181019691838083BDCF0F90DF91E7
:100DB000CF911F910F91FF90EF90DF90CF90BF9058
:100DC000AF909F908F907F9008952F923F924F9277
:100DD0005F926F927F928F929F92AF92BF92CF92CB
:100DE000DF92EF92FF920F931F93CF93DF93CDB7D4
:100DF000DEB7C85AD1090FB6F894DEBF0FBECDBF1B
:100E0000CB57DF4F188219821A821B82C558D040F7
:100E100080917C0390917D03A0917E03B0917F032C
:100E2000C757DF4F88839983AA83BB83C958D040B3
:100E3000C556DF4F19821882CB59D04084E690E026
:100E4000C356DF4F99838883CD59D0401092D60482
:100E50009E0125563F4F44E050E0BE0167577F4F4B
:100E6000CE0183569F4F0E947186C356DF4F888103
:100E70009981CD59D0400296C356DF4F998388831C
:100E8000CD59D040C556DF4F19821882CB59D0407A
:100E900081E0CD55DF4F8883C35AD0409E0125564F
:100EA0003F4F41E050E0BE016D557F4FCE0183566C
:100EB0009F4F0E9471869E0125563F4F40E150E0B2
:100EC0006EEB7AE1CE0183569F4F0E9471869E01A0
:100ED00025563F4F44E050E062E575E0CE01835671
:100EE0009F4F0E9471869E0125563F4F40E150E082
:100EF00064EA78E1CE0183569F4F0E9471869E017D
:100F000025563F4F40E150E06EEA7AE1CE0183562C
:100F10009F4F0E9471869E0125563F4F44E050E04E
:100F200062ED7AE1CE0183569F4F0E9471869E0149
:100F300025563F4F44E050E061E278E1CE01835610
:100F40009F4F0E9471869E0125563F4F44E050E01E
:100F50006EEC7AE1CE0183569F4F0E9471869E010E
:100F600025563F4F44E050E06AEA7AE1CE018356CD
:100F70009F4F0E9471869E0125563F4F44E050E0EE
:100F800066EA7AE1CE0183569F4F0E94718680E126
:100F9000E9E9F2E0DE01AD59BF4F01900D928A956B
:100FA000E1F79E0125563F4F40E150E0BE016D59EB
:100FB0007F4FCE0183569F4F0E9471869E0125561A
:100FC0003F4F44E050E069E276E1CE0183569F4F07
:100FD0000E9471869E0125563F4F4CE050E067E528
:100FE00076E1CE0183569F4F0E94718600E010E0AB
:100FF000B8016652704F9E0125563F4F44E050E0C5
:10100000CE0183569F4F0E947186085F1F4F0831A3
:10101000110571F78091E0159091E115A091E2150D
:10102000B091E315C357DF4F88839983AA83BB83AD
:10103000CD58D0409E0125563F4F44E050E0BE01C0
:1010400063577F4FCE0183569F4F0E947186CB57C7
:10105000DF4F188219821A821B82C558D04083E064
:10106000CC55DF4F8883C45AD040CB55DF4F88839F
:10107000C55AD0409E0125563F4F44E050E0BE0186
:101080006B577F4FCE0183569F4F0E9471869E0102
:1010900025563F4F41E050E0BE016C557F4FCE01D9
:1010A00083569F4F0E9471869E0125563F4F41E017
:1010B00050E0BE016B557F4FCE0183569F4F0E947B
:1010C00071861AE011509E0125563F4F44E050E0D2
:1010D000112349F0BE016B577F4FCE0183569F4FBE
:1010E0000E947186EFCF64EF7FE0CE0183569F4F61
:1010F0000E947186CB57DF4F188219821A821B8299
:10110000C558D0401AE0115071F09E0125563F4F4E
:1011100044E050E0BE016B577F4FCE0183569F4F96
:101120000E947186F0CF83E0CA55DF4F8883C65A8C
:10113000D040C955DF4F8883C75AD040CF56DF4FC4
:10114000188219821A821B82C159D040CB56DF4FB8
:10115000188219821A821B82C559D040CB57DF4FA3
:10116000188219821A821B82C558D0409E012556CA
:101170003F4F41E050E0BE016A557F4FCE0183569C
:101180009F4F0E9471869E0125563F4F41E050E0DF
:10119000BE0169557F4FCE0183569F4F0E947186D5
:1011A0009E0125563F4F44E050E0BE016B567F4FF5
:1011B000CE0183569F4F0E9471869E0125563F4F58
:1011C00044E050E0BE016F567F4FCE0183569F4FE3
:1011D0000E9471860AE010E0015011099E01255617
:1011E0003F4F0115110559F044E050E0BE016B5727
:1011F0007F4FCE0183569F4F0E947186EDCF41E015
:1012000050E063EA78E1CE0183569F4F0E947186D9
:101210009E0125563F4F41E050E06AE078E1CE0163
:1012200083569F4F0E9471869E0125563F4F44E092
:1012300050E06EE97AE1CE0183569F4F0E9471869D
:101240009E0125563F4F44E050E06AE97AE1CE0125
:1012500083569F4F0E9471869E0125563F4F44E062
:1012600050E062EA7AE1CE0183569F4F0E94718678
:101270003EE6232E39E0332E4EE7C42E49E0D42E2D
:1012800056E7E52E59E0F52E10E0412C60E8562E89
:101290006BE3662E65E4762E812C912C70E8A72EE8
:1012A0007FE3B72E1230B8F59E0125563F4F44E03C
:1012B00050E0B101CE0183569F4F0E9471869E017E
:1012C00025563F4F44E050E0B601CE0183569F4F74
:1012D0000E9471869E0125563F4F44E050E0B701C1
:1012E000CE0183569F4F0E947186CB57DF4F888275
:1012F0009982AA82BB82C558D0409E0125563F4F95
:1013000044E050E0BE016B577F4FCE0183569F4FA4
:101310000E9471862EC0CB57DF4F488259826A8265
:101320007B82C558D0409E0125563F4F44E050E097
:10133000BE016B577F4FCE0183569F4F0E9471862F
:10134000CB57DF4F188219821A821B82C558D040B2
:1013500004E0015071F09E0125563F4F44E050E0FB
:10136000BE016B577F4FCE0183569F4F0E947186FF
:10137000F0CF1F5F84E0280E311CE4E0CE0ED11CBC
:10138000F4E0EF0EF11C153009F08CCF84E190E011
:10139000C156DF4F99838883CF59D0409E0125568F
:1013A0003F4F42E050E0BE0161567F4FCE01835671
:1013B0009F4F0E9471869E0125563F4F44E050E0AA
:1013C00068EF78E1CE0183569F4F0E9471869E019F
:1013D00025563F4F44E050E064EF78E1CE0183565C
:1013E0009F4F0E9471869E0125563F4F44E050E07A
:1013F00060EF78E1CE0183569F4F0E94718680E2B4
:1014000090E0CF55DF4F99838883C15AD0409E0129
:1014100025563F4F42E050E0BE016F557F4FCE0151
:1014200083569F4F0E947186C855DF4F1882C85A55
:10143000D04080E2E9EAF2E0DE019D9601900D9253
:101440008A95E1F79E0125563F4F41E050E0BE01ED
:1014500068557F4FCE0183569F4F0E9471869E0133
:1014600025563F4F40E250E0BE01635D7F4FCE0105
:1014700083569F4F0E9471869E0125563F4F41E043
:1014800050E065E476E1CE0183569F4F0E9471865D
:101490002DE3E22E26E1F22E10E0123068F4F7017F
:1014A00080819181A281B381CB57DF4F888399835B
:1014B000AA83BB83C558D0409E0125563F4F44E0C8
:1014C00050E0BE016B577F4FCE0183569F4F0E9465
:1014D00071861F5FF4E0EF0EF11C1530F1F6BE01CE
:1014E000635B7F4F86E1FB0111928A95E9F79E01CC
:1014F00025563F4F46E150E0CE0183569F4F0E9454
:1015000071868CE2E9ECF2E0DE01119601900D9219
:101510008A95E1F79E0125563F4F4CE250E0BE010F
:101520006F5F7F4FCE0183569F4F0E947186BE0131
:1015300061587F4F86E0FB0111928A95E9F79E0181
:1015400025563F4F46E050E0CE0183569F4F0E9404
:101550007186CB57DF4F188219821A821B82C558B9
:10156000D0409E0125563F4F44E050E0BE016B57EE
:101570007F4FCE0183569F4F0E947186BE016D58EA
:101580007F4F8CE0FB0111928A95E9F79E01255669
:101590003F4F4CE050E0CE0183569F4F0E94718632
:1015A000CB57DF4F188219821A821B82C558D04050
:1015B0001CE1115071F09E0125563F4F44E050E070
:1015C000BE016B577F4FCE0183569F4F0E9471869D
:1015D000F0CFCB57DF4F188219821A821B82C55871
:1015E000D04014E0115071F09E0125563F4F44E069
:1015F00050E0BE016B577F4FCE0183569F4F0E9434
:101600007186F0CF95E3E92E96E1F92E10E01230C5
:1016100068F4F70180819181A281B381CB57DF4FBC
:1016200088839983AA83BB83C558D0409E012556E1
:101630003F4F44E050E0BE016B577F4FCE018356D1
:101640009F4F0E9471861F5FF4E0EF0EF11C153072
:10165000F1F68DE2E82E86E1F82E10E0123068F403
:10166000F70180819181A281B381CB57DF4F8883BD
:101670009983AA83BB83C558D0409E0125563F4F0E
:1016800044E050E0BE016B577F4FCE0183569F4F21
:101690000E9471861F5FF4E0EF0EF11C1530F1F629
:1016A0008091D604811167C0C356DF4FE880F9806E
:1016B000CD59D04084E6E81AF108C556DF4F88813D
:1016C0009981CB59D040C756DF4F99838883C95938
:1016D000D04084E690E0C356DF4F99838883CD598C
:1016E000D0409E0125563F4F44E050E065E273E054
:1016F000CE0183569F4F0E9471869E0125563F4F13
:1017000042E050E0BE0167567F4FCE0183569F4FA7
:101710000E947186E4E0F8E584918F010F5F1F4F0E
:10172000882321F00F941E14F801F6CFB70181EB46
:101730009FE00F947623C756DF4F48815981C959DE
:10174000D04060E070E084EA9FE00F943C23E1EA3F
:10175000FFE084918F010F5F1F4F882321F00F94CA
:101760001E14F801F6CFC7010E94F1859091D604AE
:10177000892B8093D60480910A1887FF0F94D1603B
:101780009091D60481E08927C855DF4F0FB6F894B1
:10179000DEBF0FBECDBFDF91CF911F910F91FF90A4
:1017A000EF90DF90CF90BF90AF909F908F907F9001
:1017B0006F905F904F903F902F900895CF93DF935D
:1017C000CDB7DEB72C970FB6F894DEBF0FBECDBFF6
:1017D0008091BC189091BD18A091BE18B091BF180F
:1017E00089839A83AB83BC838091C0189091C11880
:1017F000A091C218B091C3188D839E83AF83B88720
:101800008091C4189091C518A091C618B091C718BE
:1018100089879A87AB87BC870F9417240E943BA5C2
:1018200080E00F94950F81E00F94950F82E00F9464
:10183000950F6091DB157091DC158091DD1590910D
:10184000DE1540E00E94BE7C0F9472254CE050E013
:101850006CEB78E1CE0101960F94BED3892B51F049
:101860002C960FB6F894DEBF0FBECDBFDF91CF919F
:101870000D9476362C960FB6F894DEBF0FBECDBF12
:10188000DF91CF9108952F923F924F925F926F9286
:101890007F928F929F92AF92BF92CF92DF92EF9200
:1018A000FF920F931F93CF93DF93CDB7DEB7C4564C
:1018B000D1090FB6F894DEBF0FBECDBF2DB73EB72E
:1018C000A3963FAF2EAFA39767961FAE1EAE679746
:1018D00084E690E069969FAF8EAF699701E09E0124
:1018E0002B5A3F4F44E050E0BE01655B7F4FCE0175
:1018F000895A9F4F0E9424869E012B5A3F4F42E0F7
:1019000050E0BE01675A7F4FCE01895A9F4F0E9417
:10191000248643E050E0BE01655B7F4F85E293E0A3
:101920000F9414D4892B09F43CC02F968FAD2F97B8
:10193000882339F08FE32C968FAF2C972D961FAE0E
:101940002D97E4E0F8E584918F010F5F1F4F81111F
:1019500003C0EFE9F0E104C00F941E14F801F3CFC7
:1019600084918F010F5F1F4F882321F00F941E1465
:10197000F801F6CFBE01655B7F4F86E990E10F94D9
:101980008E23E8E8F0E184918F010F5F1F4F8823D9
:1019900021F00F941E14F801F6CF81E08093D60455
:1019A000AFC52DB63EB62B961CAE1DAE1EAE1FAEFD
:1019B0002B9767961FAE1EAE679701E09E012B5ACC
:1019C0003F4F41E050E0BE01615A7F4FCE01895A3E
:1019D0009F4F0E94248680E1E5EFF2E0DE019196C0
:1019E00001900D928A95E1F780E1E5E0F3E0DE01F8
:1019F000519601900D928A95E1F780E1E5E1F3E0DF
:101A0000DE01119601900D928A95E1F7A0964FADF7
:101A1000A09750E04D5F5F4F440F551F440F551F77
:101A20008DB79EB7841B950B0FB6F8949EBF0FBE63
:101A30008DBFEDB7FEB731963F0100E09E012B5AF6
:101A40003F4FBF01CE01895A9F4F0E9424869E01BD
:101A50002B5A3F4F44E050E062E575E0CE01895AD1
:101A60009F4F0E942486A096AFACA097B12CF3E0C4
:101A7000AF0EB11CAA0CBB1CAA0CBB1C2DB73EB7E9
:101A80002A193B090FB6F8943EBF0FBE2DBF8DB784
:101A90009EB701967C01EDB7FEB7EA19FB090FB6B8
:101AA000F894FEBF0FBEEDBF2DB73EB72F5F3F4F7F
:101AB00069019E012B5A3F4FA501BC01CE01895AF5
:101AC0009F4F0E9424869E012B5A3F4FA501B601CD
:101AD000CE01895A9F4F0E9424868091DA1588236F
:101AE00009F43FC000E09E012B5A3F4F44E050E014
:101AF00062ED7AE1CE01895A9F4F0E9424869E01B1
:101B00002B5A3F4F44E050E061E278E1CE01895A20
:101B10009F4F0E9424869E012B5A3F4F44E050E085
:101B20006EEC7AE1CE01895A9F4F0E9424869E0175
:101B30002B5A3F4F44E050E06AEA7AE1CE01895ADD
:101B40009F4F0E9424869E012B5A3F4F44E050E055
:101B500066EA7AE1CE01895A9F4F0E94248615E0F9
:101B600074C0A0968FADA09790E002967EEA872E73
:101B70007AE1972EB601AE014F5F5F4FE4EAAE2ED9
:101B8000E8E1BE2ED7017E0131E1E30EF11CFEEB50
:101B9000CF2EFAE1DF2EA5967FAE6EAEA5978E0111
:101BA0000F5D1F4F20E030E0821793072CF0A596C1
:101BB000EEADFFADA59701C0F80140805180628075
:101BC0007380F60141925192619271926F01821776
:101BD000930734F04D905D906D907C90139705C005
:101BE000F7014080518062807380F50141925192EB
:101BF000619271925F018217930714F0FB0101C09B
:101C0000FA014080518062807380F40141925192C8
